:200000000C94D4130C94FF130C94FF130C94FF130C94FF130C94FF130C94FF130C94FF137B
:200020000C94FF130C94FF130C94FF130C94FF130C94FF130C949F4F0C94FF130C94FF1354
:200040000C94FF130C94D74E0C949BC20C94FF130C94284D0C94524D0C94FF130C94FF13C2
:200060000C94FF130C94FF130C94FF130C94FF130C94FF130C94FF130C94FF130C94FF13F0
:200080000C94FF130C94FF130C94FF137B9BA99BD79BDB9CB3ABB3ABB3ABB3ABB3ABB3ABD3
:2000A000B3ABB3ABB3AB069C4B9C929CB3ABB3ABB3ABB3ABB3ABB3ABB3ABB3ABB3ABB3ABC3
:2000C000B3AB629FC39F23A084A0E5A046A1A7A12BA2B4A6AFA227A39FA314A488A4FCA4BC
:2000E00070A5DCA548A6B3ABB3ABB3ABB3ABB3AB309E989EB3AB0BA77FA7EEA764A88CA897
:20010000E2A81FA95CA9BBA91CAA7BAADAAA06ABB4A8B3ABB3ABB3ABB3ABB3ABB3ABB3AB16
:20012000B3ABB3ABB3ABB3ABB3ABC49DF99DB3ABB3ABB3ABB3ABB3ABB3ABB3ABB3ABB3ABA4
:20014000B3AB579EB3ABB3ABB3AB3FAB7CABB3ABB3ABB3ABB3AB6D9BB3ABB3AB1E9D579D36
:20016000A49DFD9E084AD73B3BCE016E84BCBFFDC12F3D6C74319ABD56833DDA3D00C77FC3
:2001800011BED9E4BB4C3E916BAAAABE000000803F05A84CCDB2D44EB93836A9020C50B940
:2001A000918688083CA6AAAA2ABE000000803F000001000F0015000E001200FEFF1600174C
:2001C000000E001300FFFF030002001A001400FFFF1B00FFFF0D000C000400010000000E8A
:2001E00000070006001F00536574204D6963726F7374657070696E670048656174696E6763
:20020000204265640048656174696E67204578747275646572004649524D574152455F4E76
:20022000414D453A414E45545F41385F32303136303532352020687474703A2F2F777777C0
:200240002E616E657433642E636F6D2F2056455253494F4E3A414E45542056312E30204D7B
:20026000414348494E455F545950453A414E45545F41382045585452554445525F434F5522
:200280004E543A31200044656275673A006F6B000D0A004E414E00494E46004572726F725B
:2002A0003A00496E666F3A005761726E696E673A00526573656E643A004563686F3A006F6B
:2002C0006B200057726F6E6720636865636B73756D004D697373696E6720636865636B73A8
:2002E000756D00466F726D6174206572726F7200446F6E65207072696E74696E6720666969
:200300006C6500205800205900205A00204500204600205300205000204900204A002052AE
:200320000053442072656164206572726F72004572726F723A6578706563746564206C6995
:200340006E65200020676F742000736B69702000424C4B2000737461727400506F77657215
:2003600055700045787465726E616C2052657365740042726F776E206F7574205265736523
:2003800074005761746368646F6720526573657400536F6674776172652052657365740027
:2003A000556E6B6E6F776E20636F6D6D616E643A00467265652052414D3A00583A0020584E
:2003C0003A0020593A00205A3A0020453A00543A0020423A0020403A002054002040002025
:2003E00042403A0020524157003A002F00202F0053706565644D756C7469706C793A0046AE
:200400006C6F774D756C7469706C793A0046616E73706565643A005072696E746564206634
:20042000696C616D656E743A005072696E74696E672074696D653A006D20002064617973E6
:20044000200020686F7572732000206D696E00496E76616C696420617263002C00200059E5
:200460003A005A3A0045303A0045313A004D53312C4D53322050696E7300536574206F7596
:2004800074707574200020746F20004820004C2000785F6D696E3A00785F6D61783A007953
:2004A0005F6D696E3A00795F6D61783A007A5F6D696E3A007A5F6D61783A004A65726B3A91
:2004C00000205A4A65726B3A00206C696E6561722073746570733A002071756164726174A6
:2004E00069632073746570733A002C2073706565643D00454550524F4D20757064617465A2
:2005000064006C696E656172204C3A0020717561647261746963204B3A005461726765746C
:2005200045787472005461726765744265643A00504944204175746F74756E6520737461B2
:2005400072740020626961733A200020643A2000206D696E3A2000206D61783A2000204BD5
:20056000753A20002054753A200020436C61737369632050494400204B703A2000204B6981
:200580003A2000204B643A2000504944204175746F74756E65206661696C65642120546507
:2005A0006D706572617475726520746F206869676800504944204175746F74756E652066CB
:2005C00061696C6564212074696D656F757400504944204175746F74756E652066696E69BC
:2005E00073686564202120506C61636520746865204B702C204B6920616E64204B64206330
:200600006F6E7374616E747320696E2074686520436F6E66696775726174696F6E2E6820DA
:200620006F7220454550524F4D004D54454D503A00686561746564206265640065787472BB
:200640007564657220003A2074656D702073656E736F7220646566656374003A20776F72C3
:200660006B696E67005072696E7465722073657420696E746F206472792072756E206D6FC7
:20068000646520756E74696C207265737461727421004175746F6C6576656C696E6720658B
:2006A0006E61626C6564004175746F6C6576656C696E672064697361626C6564005A2D7096
:2006C000726F6265206661696C6564005A2D70726F6265206D61783A005072696E746572CA
:2006E000206865696768743A0077616974004175746F6C6576656C206163746976652028DD
:20070000312F302900436F6E66696775726174696F6E2073746F72656420746F204545501A
:20072000524F4D2E00436F6E66696775726174696F6E206C6F616465642066726F6D204583
:200740004550524F4D2E00436F6E66696775726174696F6E20726573657420746F20646561
:200760006661756C74732E0050726F746F636F6C2076657273696F6E206368616E6765645A
:200780002C20757067726164696E6700457874722E004550523A3020004550523A31200098
:2007A0004550523A3220004550523A33200042617564726174650046696C616D656E7420DA
:2007C0007072696E746564205B6D5D005072696E74657220616374697665205B735D004DC6
:2007E00061782E20696E6163746976652074696D65205B6D732C303D6F66665D0053746FEE
:2008000070207374657070657220616674657220696E6163746976697479205B6D732C30F8
:200820003D6F66665D005820686F6D6520706F73205B6D6D5D005920686F6D6520706F730A
:20084000205B6D6D5D005A20686F6D6520706F73205B6D6D5D0058206D6178206C656E671B
:200860007468205B6D6D5D0059206D6178206C656E677468205B6D6D5D005A206D617820F7
:200880006C656E677468205B6D6D5D0058206261636B6C617368205B6D6D5D005920626185
:2008A000636B6C617368205B6D6D5D005A206261636B6C617368205B6D6D5D004D61782E57
:2008C000206A65726B205B6D6D2F735D004D61782E205A2D6A65726B205B6D6D2F735D00FD
:2008E000582D6178697320737465707320706572206D6D00592D6178697320737465707384
:2009000020706572206D6D005A2D6178697320737465707320706572206D6D00582D61782C
:200920006973206D61782E206665656472617465205B6D6D2F735D00592D61786973206DCB
:2009400061782E206665656472617465205B6D6D2F735D005A2D61786973206D61782E20EC
:200960006665656472617465205B6D6D2F735D00582D6178697320686F6D696E672066651C
:20098000656472617465205B6D6D2F735D00592D6178697320686F6D696E672066656564FD
:2009A00072617465205B6D6D2F735D005A2D6178697320686F6D696E6720666565647261D2
:2009C0007465205B6D6D2F735D00582D6178697320616363656C65726174696F6E205B6DBE
:2009E0006D2F735E325D00592D6178697320616363656C65726174696F6E205B6D6D2F73BF
:200A00005E325D005A2D6178697320616363656C65726174696F6E205B6D6D2F735E325DBF
:200A200000582D617869732074726176656C20616363656C65726174696F6E205B6D6D2F40
:200A4000735E325D00592D617869732074726176656C20616363656C65726174696F6E2023
:200A60005B6D6D2F735E325D005A2D617869732074726176656C20616363656C6572617404
:200A8000696F6E205B6D6D2F735E325D004F5053206F7065726174696F6E206D6F64652064
:200AA0005B303D4F66662C313D436C61737369632C323D466173745D004F5053206D6F760D
:200AC000652061667465722078252072657472616374205B255D004F5053206D696E2E200C
:200AE00064697374616E636520666F722066696C2E2072657472616374696F6E205B6D6D0B
:200B00005D004F50532072657472616374696F6E206C656E677468205B6D6D5D004F5053E5
:200B20002072657472616374696F6E206261636B6C617368205B6D6D5D0042656420486577
:200B40006174204D616E61676572205B302D335D0042656420504944206472697665206DAE
:200B600061780042656420504944206472697665206D696E004265642050494420502D67EA
:200B800061696E004265642050494420492D6761696E004265642050494420442D67616916
:200BA0006E0042656420504944206D61782076616C7565205B302D3235355D00737465708F
:200BC0007320706572206D6D006D61782E206665656472617465205B6D6D2F735D00737432
:200BE000617274206665656472617465205B6D6D2F735D00616363656C65726174696F6E10
:200C0000205B6D6D2F735E325D0068656174206D616E61676572205B302D335D005049440E
:200C2000206472697665206D617800504944206472697665206D696E0050494420502D67B8
:200C400061696E2F646561642D74696D650050494420492D6761696E0050494420442D67DC
:200C600061696E00504944206D61782076616C7565205B302D3235355D00582D6F666673B8
:200C80006574205B73746570735D00592D6F6666736574205B73746570735D0074656D70AA
:200CA0002E2073746162696C697A652074696D65205B735D0074656D702E20666F72207228
:200CC000657472616374696F6E207768656E2068656174696E67205B435D00646973746149
:200CE0006E636520746F2072657472616374207768656E2068656174696E67205B6D6D5D22
:200D000000657874727564657220636F6F6C6572207370656564205B302D3235355D006159
:200D20006476616E6365204B205B303D6F66665D00616476616E6365204C205B303D6F665C
:200D4000665D00534420436172642072656D6F766564005344204361726420696E7365721B
:200D600074656400534420696E6974206661696C006572726F722077726974696E6720742D
:200D80006F2066696C6500426567696E2066696C65206C69737400456E642066696C6520AC
:200DA0006C6973740046696C65206F70656E65643A002053697A653A0046696C65207365B5
:200DC0006C65637465640066696C652E6F70656E206661696C6564005344207072696E74B9
:200DE000696E67206279746520004E6F74205344207072696E74696E67006F70656E206616
:200E000061696C65642C2046696C653A200057726974696E6720746F2066696C653A2000AC
:200E2000446F6E6520736176696E672066696C652E0046696C652064656C657465640044DB
:200E4000656C6574696F6E206661696C6564004469726563746F7279206372656174656470
:200E6000004372656174696F6E206661696C6564005344206572726F72436F64653A00071B
:200E800001061C151C143A00002243141F1FA80E180F6C0FDC0F2C100000000014119C11A8
:200EA000A812F812741300000000A00F5C006009690010097900C0088C007008A2002008E2
:200EC000BD00D007DE008007050130073401E0066D019006B20140060702F0056D02A005B2
:200EE000E80250057B0300052B04B004F8046004EB06C003350920037F0B8002650DE00179
:200F0000B00E40011D0FF000480FC8006C0FA000ED0F60FFFE0F48FE0400801AD8009808B8
:200F2000AC012007800250065403C80528045805FC040005D005B004A40668047807280409
:200F40004C08E8032009B003F4097003C80A38039C0BF802700CB002440D6802180E08023F
:200F6000EC0E8801C00F8800F00F00000400001B54006009640010097400C0088400700807
:200F80009C002008B800D007D8008007000130072C01E00668019006AC0140060002F0056B
:200FA0006802A005E0025005740300052404B004F0046004DC051004E406C003040870031A
:200FC00030092003780B8002600DE001A80E4001680FA000C00F0000E80F60FF0400700DAE
:200FE000D8004804AC0158038002D8025403800228043802FC040002D005C801A406980147
:20100000780770014C08480120091801F409F000C80AC8009C0BA000700C7000440D3800BE
:20102000180E0000EC0EA8FFC00FE8FE380060093B003809400010094600E8084C00C00874
:201040005200980859007008620048086C0020087600F8078000D0079100A8079C00800758
:20106000A8005807BB003007D0000807E300E006F800B806100190062D016806500140063F
:20108000720118069001F005C201C805EC01A0052802780567025005B2022805EE020005DC
:2010A0003E03D8049803B004F20388045E046004BF04380432051004B405E8033A06C0038C
:2010C000D80698036C077003F8074803980820033909F802D409D0026F0AA8020F0B8002FA
:2010E0009F0B58022B0C3002B30C08022F0DE001980DB801FC0D90014C0E68019C0E4001F7
:201100001D0FF000480FC8006C0FA000ED0F60FFFE0F48FE0000401F450060094F00100956
:201120005C00C0086B0070087D0020089200D007AC008007CC003007DE00E00623019006E6
:201140005E014006A601F005FF01A0056D025005F30200059603B0045A0460044005100483
:201160004806C0036E077003A8082003EB09D002230B8002410C3002390DE001040E9001E4
:20118000A20E4001170FF000690FA000A20F5000C60F0000DD0FB0FFEB0F60FF0400681DDD
:2011A0004C00500B94005809DC0050082401A8076C012807B401C006FC017006440228068D
:2011C0008C02F005D402B8051C03880564035805AC033005F40310053C04E8048404C80419
:2011E000CC04A804140590045C057004A4055804EC053804340620047C060804C406F00316
:201200000C07D8035407C8039C07B003E40798032C08800374087003BC08580304094803C1
:201220004C09300394091803DC090803240AF0026C0AE002B40AC802FC0AB002440BA002D5
:201240008C0B8802D40B70021C0C5802640C4002AC0C2802F40C10023C0DF001840DD80150
:20126000CC0DB801140E98015C0E7001A40E4801EC0E1801340FD8007C0F8800C40F08002F
:20128000FC0F00000000000000000000000000000000000000000000000000000000000043
:2012A000000000000000000004000016D800C006AC0178058002C004540348042804E8034C
:2012C000FC049803D0055003A40618037807D8024C08A80220097002F4093802C80A080281
:2012E0009C0BD001700C9001440D5001180EF800EC0E8800C00F00000400401D90006009FE
:201300001C01B007A801D00634023806C002C8054C036805D80318056404D804F0049804EF
:201320007C05600408063004940600042007D003AC07A80338088003C4085803500930031A
:20134000DC090803680AE002F40AB802800B88020C0C6002980C3002240DF801B00DC00184
:201360003C0E8001C80E3001540FB800B40F2800E00F00000400081D900058091C01B007B8
:20138000A801C80634023006C002C0054C036805D80318056404D004F00498047C0560047E
:2013A00008063004940600042007D003AC07A80338088003C408580350093003DC0908038F
:2013C000680AD802F40AB002800B88020C0C6002980C3002240DF801B00DC0013C0E800139
:2013E000C80E3001540FB800B40F2800E00F00005344206572726F7220666978656400538D
:2014000044206572726F7220646964206E6F74207265636F76657221005344205265616412
:20142000204572726F720042696E6172793A00436F6D6D616E6442756666657200000000CA
:201440000000000000000000000000000024F403D950C38EB1C2A23D96828B3582127AE3DC
:2014600072816CCB66A861015DC758EB546151204E1E4B5648C14559431A41013F093D2F3E
:201480003B7139CD374036C93465331432D430A32F802E6B2D632C672B752A8E29B028DCCB
:2014A0002710274B268F25D9242B248223E0224322AC211A218D200420801F001F841E0C0C
:2014C0001E971D261DB81C4E1CE61B821B201BC11A641A0A1AB2195D190A19B9186A181C90
:2014E00018D11788174017FA16B51673163116F115B31576153A150015C7148F1458142282
:2015000014EE13BA13881356132513F612C71299126C1240121512EB11C1119811701148EA
:20152000112111FB10D610B1108D106910461024100210E10FC00FA00F800F610F420F2323
:201540000F060FE80ECB0EAF0E930E770E5C0E410E270E0D0EF30DDA0DC10DA80D900D782D
:201560000D600D490D320D1B0D050DEF0CD90CC30CAE0C990C850C700C5C0C480C350C21E9
:201580000C0E0CFB0BE80BD60BC40BB20BA00B8E0B7D0B6B0B5A0B4A0B390B290B180B0820
:2015A0000BF80AE90AD90ACA0ABB0AAC0A9D0A8E0A800A710A630A550A470A390A2C0A1E01
:2015C0000A110A040AF709EA09DD09D009C409B709AB099F09920987097B096F0963095852
:2015E000094C09410936092B09200915090A090009F508EB08E008D608CC08C208B808AEAB
:2016000008A4089A08900887087D0874086B08610858084F0846083D0834082C0823081A71
:2016200008120809080108F807F007E807E007D807D007C807C007B807B007A807A1070089
:2016400000420FA1071605D0030D038B022E02E801B2018601630145012C0117010401F4CB
:201660000049646C6500486F6D65205A00486F6D65205900486F6D652058005374657070DA
:2016800065722044697361626C6564004B696C6C65640055706C6F6164696E672E2E2E00B9
:2016A0005344207072696E742073746F7070656420627920757365722E0046696E64206915
:2016C0006E69742E672066696C6520696E205344434152442C20737461727420746F207095
:2016E00072696E742E2E2E0000002110422063308440A550C660E770088129914AA16BB1FD
:201700008CC1ADD1CEE1EFF13112100273325222B5529442F772D662399318837BB35AA3F1
:20172000BDD39CC3FFF3DEE36224433420040114E664C774A44485546AA54BB52885099531
:20174000EEE5CFF5ACC58DD55336722611163006D776F6669556B4465BB77AA71997388771
:20176000DFF7FEE79DD7BCC7C448E5588668A7784008611802282338CCC9EDD98EE9AFF9A1
:20178000488969990AA92BB9F55AD44AB77A966A711A500A333A122AFDDBDCCBBFFB9EEBF1
:2017A000799B588B3BBB1AABA66C877CE44CC55C222C033C600C411CAEED8FFDECCDCDDD31
:2017C0002AAD0BBD688D499D977EB66ED55EF44E133E322E511E700E9FFFBEEFDDDFFCCF71
:2017E0001BBF3AAF599F788F8891A981CAB1EBA10CD12DC14EF16FE18010A100C230E3205D
:201800000450254046706760B9839893FBA3DAB33DC31CD37FE35EF3B1029012F322D232F0
:201820003542145277625672EAB5CBA5A89589856EF54FE52CD50DC5E234C324A014810430
:201840006674476424540544DBA7FAB79987B8975FE77EF71DC73CD7D326F2369106B01670
:2018600057667676154634564CD96DC90EF92FE9C899E9898AB9ABA94458654806782768A0
:20188000C018E1088238A3287DCB5CDB3FEB1EFBF98BD89BBBAB9ABB754A545A376A167AF0
:2018A000F10AD01AB32A923A2EFD0FED6CDD4DCDAABD8BADE89DC98D267C076C645C454C30
:2018C000A23C832CE01CC10C1FEF3EFF5DCF7CDF9BAFBABFD98FF89F176E367E554E745E70
:2018E000932EB23ED10EF01E7C3C3E5E2B3D3F2F5B5D3B2C2A225C004E6F206572726F7252
:2019000020666F756E642E0043616E2774206F70656E20726F6F74206469726563746F727E
:20192000792E00496E76616C696420666F726D61742C207265666F726D61742053442E00FF
:201940004E6F20636172642C2077726F6E6720636869702073656C6563742070696E2C2080
:201960006F72205350492070726F626C656D3F0043616E2774206163636573732053442014
:20198000636172642E20446F206E6F74207265666F726D61742E000001FF00FF000001018C
:2019A0000000FF00FF01004B65794E6F203D2000416374696F6E3A256C61000310270200FF
:2019C000831B0310270200871B01000001008B1B02000008008D1B03ED0304009D1B03EE91
:2019E000030400A51B03EF030400AD1B03FA030400B51B03FB030400BD1B03FC030400C5E3
:201A00001B0200000900CD1B0200000600DF1B0200000C00EB1B5265717565737450617593
:201A200073653A004E6F205344204361726400436F6F6C646F776E00507265686561742058
:201A4000414253005072656865617420504C41008025000040380000004B00008070000092
:201A600000960000C0DA000000E10000002C010008B2010000C2010000F40100008403002E
:201A800090D0030000E803000008070020A1070000100E0040420F0060E316000000000019
:201AA0000200000900031C151C1C1C231C2A1C4F6E004F666600596573004E6F0003000441
:201AC000004E2F4100003A002064617973200041380042616E6742616E6700536C6F7742CD
:201AE000616E6700446561642054696D6500504944005072696E74696E672E2E2E0020645D
:201B0000656620000000003FCDCC4C3D0AD7A33B6F12033A4F4D4E49203344205052494ED9
:201B2000544552200057454C434F4D4520544F204F4D4E49004138005072696E74657220FB
:201B400072656164792E0000401454040E15041C000000040A040000000000001F1F1F1FC5
:201B60001F0000001F1111111F0000040A0A0A0E1F1F0E001C1F11111F0000001F15111583
:201B80001F1F00311C381C3F1C461C4D1C4D1C541C5B1C621C691C701C771C7E1C851C8C07
:201BA0001C931C9A1CA11CA81CAF1CB61CBD1CC41CCB1CD21CD91CE01CE71CEE1CF51CFCED
:201BC0001C031D0A1D111D181D1F1D261D4D1C2D1D341D3B1D421D491D501D571D5E1D4DF6
:201BE0001C651D6C1D731D7A1D811D4D1C2D1D881D8F1D961D9D1DA41DAB1DB21DB91DC09A
:201C00001D7A1D4D1CC71D541CCE1DD51DDC1DE31DEA1DF11D0000000400F81D000000044B
:201C200000001E0000000400081E0000000400101E181E0000000000261E00000000003779
:201C40001E0000000000451E0000000000561E03E80300005D1E03F5030102681E03F603A6
:201C60000204741E03540402007F1E03F70304008E1E03F80301009B1E03F9030001A61EA9
:201C800003F4030102B21E0000000000BB1E0000000000CB1E0000000000DB1E00000000BC
:201CA00000DC1E0000000000E51E0000000000F51E0000000000051F0000000000061F00CB
:201CC000000000000F1F00000000001F1F00000000002F1F0000000000301F0000000000FB
:201CE000391F0000000000491F0000000000591F00000000005A1F0000000000631F0000B1
:201D0000000000731F0000000000831F0000000000841F00000000008D1F00000000009DA3
:201D20001F0000000000AD1F0000000000AE1F03FD030010B71F041F040000C91F044804A3
:201D40000000DB1F0337040000E71F0347040000F31F0338040000FC1F03310400100A2019
:201D600003420400101A20043C0400002A20043D0400003A20033A0400004920025820007F
:201D8000005F2003430400006A2003FE030010712003FF030010782003000400107F2002E6
:201DA000EC1900008B2002D7190000962002F3190000A22002DE190000AD2002FA19000020
:201DC000B92002E5190000C42002011A0000D320020F1A0000DC2002081A0000E52002EFF5
:201DE000200000F62002D0190000FE2002082100000F21021D21000024212B2132213921CB
:201E0000402147214E2155215C2163216A21712178217F2186218D21436F6E66696775722B
:201E20006174696F6E0073746F72656420696E20454550524F4D00436F6E66696775726179
:201E400074696F6E006C6F6164656420662E20454550524F4D004261636B20010050726906
:201E60006E742066696C65005061757365205072696E740053746F70205072696E7400437F
:201E80006F6E74696E7565205072696E7400556E6D6F756E742043617264004D6F756E7470
:201EA00020436172640044656C6574652066696C6500583A257830206D6D004D696E206573
:201EC0006E6473746F703A257378004D617820656E6473746F703A2573580000593A257883
:201EE00031206D6D004D696E20656E6473746F703A257379004D617820656E6473746F70E8
:201F00003A25735900005A3A257832206D6D004D696E20656E6473746F703A25737A004D5F
:201F2000617820656E6473746F703A25735A0000583A257830206D6D004D696E20656E64AB
:201F400073746F703A257378004D617820656E6473746F703A2573580000593A2578312083
:201F60006D6D004D696E20656E6473746F703A257379004D617820656E6473746F703A2559
:201F8000735900005A3A257832206D6D004D696E20656E6473746F703A25737A004D617865
:201FA00020656E6473746F703A25735A0000486F6D6520416C6C005370656564204D756CD7
:201FC0002E3A256F6D25252500466C6F77204D756C2E203A256F662525250050726568655E
:201FE000617420504C4100507265686561742041425300436F6F6C646F776E0053657420BF
:20200000746F204F726967696E0044697361626C652073746570706572004265642054659A
:202020006D702E3A25456202430054656D702E203020203A25453002430045787472756461
:2020400065722030204F666600457874722E20706F736974696F6E0003F0030200942153B8
:202060006574204F726967696E00486F6D65205800486F6D65205900486F6D65205A0058A1
:2020800020506F732E2046617374005820506F736974696F6E005920506F732E2046617332
:2020A00074005920506F736974696F6E005A20506F732E2046617374005A20506F736974CD
:2020C000696F6E00517569636B2053657474696E677300506F736974696F6E004578747254
:2020E000756465720046616E2073706565640002000007009821534420436172640044654E
:2021000062756767696E67000200000500A621436F6E66696775726174696F6E00020000B4
:202120000700B021BE210000000000D1210000000000E1210000000000F5210000000000DE
:20214000F9210000000000022200000000000B2200000000001422000000000018220000A4
:20216000000000292200000000002A2200000000003A2200000000003E2200000000004CC0
:20218000220000000000502200000000006122000000000067226E224D1C75227C228322CC
:2021A0008A22912298224D1C9F22A622AD22B4224D1CBB22C222C922D022D722DE22052545
:2021C00065632F25456302072565422F25456202005A3A2578322020427566203A256F4279
:2021E000004D756C3A256F6D20202020466C6F773A256F6600256F7300583A257830206D37
:202200006D00593A257831206D6D005A3A257832206D6D00256F730045313A2565302F25D4
:20222000453002437E256F300000423A2565622F25456202437E256F6200256F73005072BD
:20224000696E74696E672074696D65002555740046696C616D656E74207072696E746564F2
:2022600000255566206D00E5220000000000EE220000000000FD2204520400000E23031A13
:202280000408001B23031B0400002923031C0400003723031D0400004523031E0400005206
:2022A0002303320400005E2303330400006A230334040000762303350400008223028A2316
:2022C00000009123029E230000A52302AE230000B52302BE230000C5230306040000D52344
:2022E0000307040000453A257833206D6D003120636C69636B203D2031206D6D0046616E73
:202300002073706565643A254673252525005475726E2046616E204F66660053657420465A
:20232000616E203235252525005365742046616E203530252525005365742046616E2037CB
:2023400035252525005365742046616E2046756C6C004563686F2020203A25646F00496EFD
:20236000666F2020203A256469004572726F7273203A256465004472792072756E3A2564D0
:20238000640047656E6572616C000200000400E423416363656C65726174696F6E00020042
:2023A000000900EC234665656472617465000200000700FE23457874727564657200020066
:2023C000000F000C2453746F726520746F20454550524F4D004C6F616420662E2045455098
:2023E000524F4D004D1C2A24312438244D1C3F2446244D2454245B246224692470244D1CD9
:2024000077247E2485248C2493249A244D1CA124A824AF24B624BD24C424CB24D224D9245F
:20242000E024E724EE24F524FC240325041004000010250221250000282502362500003D9E
:20244000250408040000492504090400005525040A0400006125040B0400006D25040C04FD
:2024600000007925040D0400008525040E0400009125040F0400009D250414040000A72572
:202480000415040000B1250416040000BB250411040000C6250412040000D125041304001C
:2024A00000DC250429040000E925042C040000F625042B0400000126042A0400000B2604CC
:2024C0002E0400001926044D0400002C26044C0400003D26042D040000492604220400005F
:2024E00056260423040000602604240400006A260425040000782604260400008626042F1B
:2025000004000042617564726174653A256F63005374657070657220496E61637469766528
:2025200000032004020092264D61782E20496E6163746976650003580402009626507269CB
:202540006E7420583A256178005072696E7420593A256179005072696E74205A3A25617A69
:20256000004D6F76652058203A256158004D6F76652059203A256159004D6F7665205A209A
:202580003A25615A004A65726B2020203A25616A005A2D4A65726B203A25614A004D6178A8
:2025A00020583A256678004D617820593A256679004D6178205A3A25667A00486F6D652001
:2025C000583A25665800486F6D6520593A25665900486F6D65205A3A25665A0053746570A8
:2025E000732F4D4D3A2553650053746172742046523A255866004D61782046523A255846CA
:2026000000416363656C3A25584100537461622E54696D653A255877005761697420556EFD
:202620006974733A20255855206D6D00576169742054656D702E20255854024300436F6E55
:2026400074726F6C3A2558680044542F50494420503A2558700050494420493A25586900F9
:2026600050494420443A255864004472697665204D696E3A25586D004472697665204D61D4
:20268000783A25584D00504944204D61783A255844009A26A126A826AF26B626000000009A
:2026A00000C5260000000000CF260000000000DE2600000000004469732E204166746572D6
:2026C0003A256973005B735D20303D4F6666004469732E2041667465723A256970005B7386
:2026E0005D20303D4F66660000002100240027002A0000002200250028002B000000200085
:202700002300260029000202020202020202040404040404040403030303030303030101FD
:202720000101010101010102040810204080010204081020408001020408102040808040D6
:20274000201008040201000000010200000000000000040307060000000000000000000023
:20276000000000000000494E46494E4954594E414ECDCCCC3D0AD7233C17B7D13877CC2BEB
:20278000329595E6241FB14F0A000020410000C84200401C4620BCBE4CCA1B0E5AAEC59D5A
:2027A0007400934E3A79B69911241FBECFEFD0E4DEBFCDBF12E0A0E0B1E0ECE7F4E901E081
:2027C0000BBF02C007900D92A236B107D9F71BBE10E1A2E6B2E001C01D92AD3BB107E1F70B
:2027E00017E2C8EAD7E204C02297FE010E94EEC9C23AD107C9F70E94CAC40C943CCA0C9496
:202800000000CF93DF93BC018230910510F462E070E0A091B910B091BA10ED01E0E0F0E0C6
:2028200040E050E021C0888199818617970769F48A819B81309719F09383828304C09093B3
:20284000BA108093B910FE0134C06817790738F44115510519F08417950708F4AC01FE0120
:202860008A819B819C01E9012097E9F641155105A9F1CA01861B970B049708F4BA01E0E0AE
:20288000F0E02AC08D919C91119784179507F9F46417750781F412968D919C911397309797
:2028A00019F09383828304C09093BA108093B910FD0132964CC0CA01861B970BFD01E80F92
:2028C000F91F6193719302978D939C9340C0FD01828193819C01D9011097A1F68091B7105E
:2028E0009091B810892B41F480911401909115019093B8108093B710409116015091170103
:202900004115510541F44DB75EB78091120190911301481B590B2091B7103091B810CA01D1
:20292000821B930B8617970780F0AB014E5F5F4F8417950750F0420F531F5093B8104093F2
:20294000B710F9016193719302C0E0E0F0E0CF01DF91CF910895CF93DF93009709F450C0B7
:20296000EC0122971B821A82A091B910B091BA10109709F140E050E0AC17BD0708F1BB83C4
:20298000AA83FE0121913191E20FF31FAE17BF0779F48D919C911197280F391F2E5F3F4FFF
:2029A0003983288312968D919C9113979B838A834115510571F4D093BA10C093B91020C0AE
:2029C00012968D919C911397AD01009711F0DC01D3CFFA01D383C28321913191E20FF31F88
:2029E000CE17DF0769F488819981280F391F2E5F3F4FFA01318320838A819B81938382834E
:202A0000DF91CF910895A0E0B0E0E9E0F5E10C940BCAEC015B016115710519F0FB019183D7
:202A20008083F9908F2D90E00E94F2C9892BC9F7FDE2FF1621F4F990EE24E39405C02BE220
:202A4000F21609F4F990EE248E0101501040C80166E677E243E050E00E949217892B01F5F0
:202A60008E010E5F1F4FC80169E677E245E050E00E949217892B19F48E01095F1F4FA11400
:202A8000B10419F0F50111830083E0FC04C070E090E080E814C070E090E080E86FEF08C180
:202AA000C8016EE677E243E050E00E949217892B69F4A114B10429F470E090E080EC6FE7E8
:202AC000F7C02296F501D183C083F6CF8824992440E050E060E070E0EF2DE053EA30A0F5EE
:202AE000F2E0EF2A8E2D90E09C0128703070E2FE06C0232B79F50894811C911C2BC0232B6A
:202B000019F0089481089108DB01CA0112E0880F991FAA1FBB1F1A95D1F7480F591F6A1F94
:202B20007B1F440F551F661F771F4E0F511D611D711D483929E9520729E9620729E1720758
:202B400048F084E0E82A06C0EE3F31F4E3FC39C098E0E92AF990C0CFE53311F0E53189F587
:202B600029912D3219F4E0E1EE2A05C02B3219F081E090E003C0299182E090E0E22FE053C7
:202B8000EA3018F0C81BD90B1CC020E030E0FCE020383F075CF4C901880F991F880F991F2E
:202BA000280F391F220F331F2E0F311DE991E053EA3068F3E4FE03C0309521953F4F820E18
:202BC000931ECE2CDD24E1FE07C0A114B10421F02197F501D183C083CB01BA010E946AC68A
:202BE0007B018C01F3E0CF22DD2423E0C216D10421F417FB109517F9109557016801C8014C
:202C0000B70120E030E040E050E00E94CAC5882309F44AC097FE0DC025E8E22E27E2F22E11
:202C20009094819491089394C0E2D0E000E010E012C09DE9E92E97E2F92EF6CFF7012591F7
:202C4000359145915491C601B5010E947AC85B016C018C1A9D0A8C169D0684F7D595C795F6
:202C60000F5F1F4F0630110529F08CEF9FEFE80EF91EF1CFC501D6017C018D018C2D880F45
:202C80008D2D881F8F3F51F0C601B50120E030E040E050E00E94CAC5882331F482E290E012
:202CA0009093BC108093BB107E2D9F2D802F612F272F392F482F562FB901CA01CDB7DEB739
:202CC000ECE00C9427CA2F923F925F926F927F928F929F92AF92BF92CF92DF92EF92FF923A
:202CE0000F931F93CF93DF938C011B01EA016115710519F0FB0191838083209749F0CE0151
:202D00000297839728F020E030E040E050E0F6C0F801A1908F018A2D90E00E94F2C9892BE0
:202D2000B9F7FDE2AF1631F4F801A1908F015524539407C0FBE2AF1619F4F801A1908F01D0
:202D40005524209719F0C031D105C1F4F0E3AF1679F4F8018081883711F0883549F4F8010C
:202D6000A1800E5F1F4FF2E05F2AC0E1D0E006C0209721F480E3A816E9F427C0C830D10566
:202D800031F1C930D10524F4C230D10531F50CC0CA30D10589F0C031D105F9F4C12CD12C89
:202DA000E12CB8E0FB2E28C0C12CD12CE12CA0E4FA2E22C0CAE0D0E0FCECCF2EFCECDF2EA4
:202DC000FCECEF2EFCE0FF2E17C0C8E0D0E0C12CD12CE12CE0E1FE2E0FC09E01442737FDC5
:202DE0004095542F60E070E080E090E80E94A3C9C901DA016C017D0120E030E040E050E015
:202E000060E03E01882477FC8094982C70EDB72EBA0CE9E0EB1570F48A2D81548A3118F4B4
:202E200099ECB92E06C08A2D81568A3150F589EAB82EBA0C8B2D90E08C179D0714F56F3F8D
:202E4000E1F0C216D306E406F506B0F0CA01B901A40193010E9450C99B01AC012B0D311D23
:202E6000411D511D2130F0E03F07F0E04F07F0E85F0710F461E001C06FEFF801A1908F019D
:202E8000C5CF2114310481F0662331F001501040F1011183008308C051FE1AC002501040DC
:202EA000F1011183008314C067FF12C050FC05C02FEF3FEF4FEF5FE704C020E030E040E028
:202EC00050E882E290E09093BC108093BB1016C050FE08C050954095309521953F4F4F4FCC
:202EE0005F4F0CC057FF0AC082E290E09093BC108093BB102FEF3FEF4FEF5FE7B901CA0142
:202F0000DF91CF911F910F91FF90EF90DF90CF90BF90AF909F908F907F906F905F903F900D
:202F20002F900895FB01DC014150504088F08D9181341CF08B350CF4805E659161341CF0AF
:202F40006B350CF4605E861B611171F3990B0895881BFCCFFB01DC0102C001900D92415091
:202F60005040D8F70895FB01DC010D900020E9F7119701900D920020E1F70895FC01819163
:202F8000861721F08823D9F7992708953197CF010895FB01DC018D91019080190110D9F378
:202FA000990B0895FB01DC0101900D920020E1F70895FB01DC014150504048F001900D92D0
:202FC0000020C9F701C01D9241505040E0F70895FC0181E090E00190061609F4CF010020A4
:202FE000D1F701970895A0E0B0E0E9EFF7E10C940FCA7C01EB018A01690109C0CE012196EE
:20300000F6010995F70181937F010150104001151105A1F7CDB7DEB7E8E00C942BCABF9263
:20302000CF92DF92EF92FF920F931F937B018C01FB010995B82EC8010196F7010995C82EE3
:20304000C8010296F7010995D82EC8010396F7010995982F6B2D7C2D8D2D1F910F91FF90DA
:20306000EF90DF90CF90BF900895DF92EF92FF920F931F937B018C01FB010995D82EC801CE
:203080000196F7010995982F8D2D1F910F91FF90EF90DF900895A0E0B0E0E1E5F8E10C94C9
:2030A0000FCAEC017B018A01690109C0CE012196F70161917F01F6010995015010400115D4
:2030C0001105A1F7CDB7DEB7E8E00C942BCABF92CF92DF92EF92FF920F931F93D52EC62E4C
:2030E000B72E79018C01642FF9010995C80101966D2DF7010995C80102966C2DF701099599
:20310000C80103966B2DF70109951F910F91FF90EF90DF90CF90BF900895DF92EF92FF9284
:203120000F931F93D72E7A018C01FA010995C80101966D2DF70109951F910F91FF90EF90A7
:20314000DF9008959C01F999FECF32BD21BDF89A80B5089508956091180170911901809163
:203160001A0190911B016817790744F470931B0160931A0181EB93E00E94C4290895BC01CB
:20318000893191051CF469E170E005C0893C910514F068EC70E07093710C6093700C8FEF00
:2031A00093E00E94C4290895EF92FF920F931F93CF93DF93EC01893191051CF4C9E1D0E08F
:2031C00006C081E0C53FD80714F0C4EFD1E0BE01882777FD8095982F0E946CC67B018C01E2
:2031E00060916E0C70916F0C882777FD8095982F0E946CC69B01AC01C801B7010E94D1C513
:203200009B01AC0160916A0C70916B0C80916C0C90916D0C0E947AC860936A0C70936B0C9C
:2032200080936C0C90936D0CD0936F0CC0936E0C80EF93E0BE010E94C429DF91CF911F910C
:203240000F91FF90EF9008950E9447509C0180911801909119012817390724F43093190174
:203260002093180108950E94E34C08952F923F924F925F926F927F928F929F92AF92BF921D
:20328000CF92DF92EF92FF920F931F93DF93CF93CDB7DEB728970FB6F894DEBF0FBECDBF03
:2032A000A090CB0BB090CC0BC090CD0BD090CE0B2090CF0B3090D00B4090D10B5090D20B02
:2032C0008091D30B9091D40BA091D50BB091D60B89839A83AB83BC832091F30B3091F40BC7
:2032E0004091F50B5091F60B6090F70B7090F80B8090F90B9090FA0B8091FB0B9091FC0BAE
:20330000A091FD0BB091FE0B8D839E83AF83B8878091870B882359F40F2EF0E0EF2EF0E0F3
:20332000FF2EF0E80F2FFFE31F2FF02D0AC00F2EF0E7EF2EF2E4FF2EF1E20F2FFDE31F2FC0
:20334000F02DC601B5010E9404C5A80197010E947AC8AB01BC018BEB93E022E00E94FF2A24
:203360008091870B882359F40F2EF0E0EF2EF0E0FF2EF0E80F2FFFE31F2FF02D0AC00F2E21
:20338000F0E7EF2EF2E4FF2EF1E20F2FFDE31F2FF02DC201B101A40193010E9404C5A80118
:2033A00097010E947AC8AB01BC0182EC93E022E00E94FF2A8091870B882359F40F2EF0E0D2
:2033C000EF2EF0E0FF2EF0E80F2FFFE31F2FF02D0AC00F2EF0E7EF2EF2E4FF2EF1E20F2F61
:2033E000FDE31F2FF02D69817A818B819C812D813E814F8158850E9404C5A80197010E940C
:203400007AC8AB01BC0186EC93E022E00E94FF2A2091C70B3091C80B4091C90B5091CA0BDD
:20342000A090940BB090950BC090960BD090970B8091870B882359F40F2EF0E0EF2EF0E055
:20344000FF2EF0E80F2FFFE31F2FF02D0AC00F2EF0E7EF2EF2E4FF2EF1E20F2FFDE31F2F9F
:20346000F02DCA01B9010E946CC6A60195010E947AC8A80197010E947AC8AB01BC018AECB1
:2034800093E022E00E943B2B28960FB6F894DEBF0FBECDBFCF91DF911F910F91FF90EF907C
:2034A000DF90CF90BF90AF909F908F907F906F905F904F903F902F9008950F931F9303E222
:2034C00014E0C8016DE00E94624EC8016AE00E94624E1F910F9108956F927F928F929F92DA
:2034E000AF92BF92CF92DF92EF92FF920F931F93DF93CF9300D000D0CDB7DEB76091880CF0
:203500007091890C80918A0C90918B0C2FE632E143E85AE30E947AC87B018C01CE010196D3
:2035200061E870E044E050E022EA38E10E94F317C801B70129813A814B815C810E9404C5D3
:20354000AB01BC0187E194E022E00E94FF2A88E394E00E94A129E091CC01F091CD01638599
:2035600074858585968520E030E040E751E40E94D8C718160CF47AC06624772443018DE73B
:2035800090E062EA78E10E940F187B018C01E60CF71C081D191DC801B70120E831E541E024
:2035A00050E00E94C5C9922E832E742E652E622F732F842F952F20E83EEA4EEF5FEF0E94FE
:2035C00050C95B016C01AE0CBF1CC01ED11E89E294E0492D582D672D762D0E94EB29C60119
:2035E000B50120E13EE040E050E00E94C5C9122F032FF42EE52E8BE394E0422F502F6F2D60
:203600007E2D0E94EB29612F702F8F2D9E2D20EF31EF4FEF5FEF0E9450C9A60EB71EC81EAE
:20362000D91EC601B5012CE330E040E050E00E94C5C982E494E0BA01A9010E94EB298AE414
:2036400094E00E94282A0F900F900F900F90CF91DF911F910F91FF90EF90DF90CF90BF903B
:20366000AF909F908F907F906F9008950E94E3C22091840C3091850C4091860C5091870C61
:20368000621B730B840B950B28EE33E040E050E00E94A3C9C901DA013C014D0170CF1F9358
:2036A000182FE0917502F091760244A555A566A577A58EEC93E022E00E94FF2AE091750236
:2036C000F091760240A951A962A973A98DEE93E020E00E94FF2A0E942338AB01BC0181ED5A
:2036E00093E022E00E94FF2A409196015091970160919801709199018DEE93E020E00E94F4
:20370000FF2A112391F084EE93E061E070E00E94FC296CEF7FE080918E0190918F01681B00
:20372000790B89EE93E00E94FC29E0918B01F0E0E85BFB4F60818FED93E070E00E94FC2913
:20374000E0911E01EF3F29F4E0917502F0917602E081F0E0E85BFB4F608185ED93E070E0D9
:203760000E94FC290E945D1A1F910895809164028823C1F0109264020E94364180911D01F9
:20378000815080931D01882349F480911C01833010F40E94F53A85E080931D018EE89FE0FE
:2037A0000E9428C0089508C00E94C8490E94B61B8EE89FE00E94B5998091810B8823A1F72F
:2037C0000895CF93DF9397FD10C0EC018F3F910521F01CF0CFEFD0E002C0009731F08091AD
:2037E000010C88608093010C07C08091010C877F8093010CC0E0D0E0662311F00E94D31B3F
:2038000080914B0490E0C817D90729F08DE094E0BE010E94C429C0934B04DF91CF910895C2
:203820002F923F924F925F926F927F928F929F92AF92BF92CF92DF92EF92FF920F931F93F6
:20384000DF93CF93CDB7DEB7E0970FB6F894DEBF0FBECDBF6C0180912702282F84FF19C063
:20386000D6018C9182FD09C081FF13C016968D919C9117978F36910561F00E94E3C260932E
:2038800040047093410480934204909343040C949F28F6010081118102FF75C38085918514
:2038A0008431910509F42DC28531910558F48430910520F4029708F040C020C0049709F0D6
:2038C00056C3E1C18A35910509F465C28B35910540F48531910509F418C24C9709F047C321
:2038E00017C28C35910509F45DC28C35910508F455C28C39910509F03AC30EC312FF12C00D
:20390000F601878D90A1A1A1B2A12091000C0097A105B10519F0822F806202C0822F8F7D0B
:203920008093000CC6010E944D6F882309F41FC381E061E00E9499651AC38091CB0B909192
:20394000CC0BA091CD0BB091CE0B89879A87AB87BC878091CF0B9091D00BA091D10BB09192
:20396000D20B8D879E87AF87B88B8091D30B9091D40BA091D50BB091D60B898B9A8BAB8B27
:20398000BC8BC6010E944D6F882309F4F0C2FE01319688E0DF011D928A95E9F7F6018281AB
:2039A00080FD05C020E030E040E050E007C0D60197962D913D914D915C919A978091870B6F
:2039C000882351F0CA01B90123E333E34BEC51E40E947AC89B01AC0129833A834B835C83AB
:2039E000F601828181FD05C020E030E040E050E007C0D6019B962D913D914D915C919E97CF
:203A00008091870B882351F0CA01B90123E333E34BEC51E40E947AC89B01AC012D833E836C
:203A20004F835887FE01759680E1DF011D928A95E9F78091CB0B9091CC0BA091CD0BB091B3
:203A4000CE0B8D8B9E8BAF8BB88F8091CF0B9091D00BA091D10BB091D20B898F9A8FAB8F3E
:203A6000BC8F8091D30B9091D40BA091D50BB091D60B8D8F9E8FAF8FB8A36091EF0B70910B
:203A8000F00B8091F10B9091F20B0E946CC62091940B3091950B4091960B5091970B0E94E4
:203AA0007AC869A37AA38BA39CA3F601828182FFC7C087A490A8A1A8B2A88091870B8823D8
:203AC00051F0C501B40123E333E34BEC51E40E947AC84B015C016D897E898F89988D29852D
:203AE0003A854B855C850E9403C56DA77EA78FA798AB698D7A8D8B8D9C8D2D853E854F85B3
:203B000058890E9403C52B013C01C501B40120E030E040E850E40E947AC8A50194010E9449
:203B20007AC87B018C016DA57EA58FA598A99B01AC010E947AC89B01AC01C801B7010E94F7
:203B400003C57B018C01C301B201A30192010E947AC89B01AC01C801B7010E9403C50E942C
:203B6000E7C87B018C016DA57EA58FA598A9A30192010E94E5C79B01AC0117FB109517F94E
:203B80001095C801B7010E94D1C57B018C01A80197010E9434C9882329F08FE494E00E9491
:203BA0002D2AE5C1D60118968D919C911997039721F417FB109517F91095C501B40120E0F2
:203BC00030E040E050E00E94CAC5882344F417FB109517F91095B7FAB094B7F8B094C30159
:203BE000B201A80197010E947AC89B01AC016DA57EA58FA598A90E9403C520E030E040E060
:203C00005FE30E947AC869837A838B839C836DA57EA58FA598A9A80197010E947AC89B01FD
:203C2000AC01C301B2010E9404C520E030E040E05FE30E947AC86D837E838F8398870CC0B1
:203C400069817A818B819C812D813E814F8158850E94E5C74B015C01E0E0D60118968D91E2
:203C60009C911997029709F4E1E0CE010996BE016B5E7F4FAE014F5F5F4F95018401EE2E0A
:203C80000E94445674C10E94D31BF6018081918193FD04C0EE24FF24870107C0D601939641
:203CA000ED90FD900D911C91969792FF0DC0F601678D70A181A192A128EE33E040E050E05A
:203CC0000E9450C97B018C010E94E3C25B016C01AE0CBF1CC01ED11E04C00E94C8490E9495
:203CE000B61B0E94E3C2A6019501261B370B480B590BDA01C90180509449A543B74768F3A2
:203D000036C181E08093870B32C11092870B2FC1C80188739070892B11F080E008C0C80125
:203D200056E0969587955A95E1F78095817006FF08C01092C70B1092C80B1092C90B10926B
:203D4000CA0B882321F041E051E061E01DC0D6012D913C91C90188739070892BC1F0C9010C
:203D600043E0969587954A95E1F7582F5170C90134E0969587953A95E1F7682F617025FD84
:203D800002C040E001C041E0852F0E94017480E00E94986AECC01092B90BE9C081E0809361
:203DA000B90BE5C0A090F30BB090F40BE090F50BF090F60B6090F70B7090F80B8090F90B33
:203DC0009090FA0B2090FB0B3090FC0B4090FD0B5090FE0B03FF21C0F6012285338544857E
:203DE00055858091870B882351F0CA01B90123E333E34BEC51E40E947AC89B01AC01CA0155
:203E0000B9012091CB0B3091CC0B4091CD0B5091CE0B0E9403C55B017C0104FF23C0D60166
:203E20001E962D913D914D915C9151978091870B882351F0CA01B90123E333E34BEC51E4F3
:203E40000E947AC89B01AC01CA01B9012091CF0B3091D00B4091D10B5091D20B0E9403C5B4
:203E60003B014C0105FF21C0F60122893389448955898091870B882351F0CA01B90123E3B1
:203E800033E34BEC51E40E947AC89B01AC01CA01B9012091D30B3091D40B4091D50B50912D
:203EA000D60B0E9403C51B012C01B501C7019301A401710182010E94776AD6018C9186FFC6
:203EC00056C056962D913D914D915C9159978091870B882351F0CA01B90123E333E34BEC32
:203EE00051E40E947AC89B01AC01CA01B9012091E7013091E8014091E9015091EA010E946F
:203F00007AC80E9439C66093C70B7093C80B8093C90B9093CA0B2BC080E061E040E00E94F6
:203F2000017400D000D020915A0C30915B0C40915C0C50915D0C8091FF0190910002A09145
:203F40000102B0910202EDB7FEB781839283A383B48360E87FE483EC97E47B018C015B0150
:203F60006C010E94BA720F900F900F900F900E94E3C2609340047093410480934204909348
:203F800043040C949F2801FD02C00C948D28D60116968D919C9117978237910509F4C9C607
:203FA0008337910508F081C08A32910509F47EC18B329105C8F58931910509F427C18A31EA
:203FC0009105C8F48631910509F404C18731910548F48431910509F4F3C0459711F00C947E
:203FE0009F28F3C08731910509F4F9C0489711F00C949F2806C18C31910509F42BC18D313B
:20400000910548F48A31910509F406C14B9711F00C949F281AC18E31910509F427C1809743
:2040200011F00C949F2831C18336910509F427C684369105D8F48435910509F49AC585356C
:20404000910550F48235910509F48CC58335910511F00C949F2889C58535910509F4A5C530
:204060008C35910511F00C949F28C0C58A36910509F45CC58B36910550F48836910509F49C
:204080005DC18936910511F00C949F2807C28D36910509F40DC28F36910509F430C68B3648
:2040A000910511F00C949F2853C58E3C910509F468C78F3C9105E8F58E3B910509F4E9C318
:2040C0008F3B9105D8F48537910509F435C68637910550F48337910509F424C6843791054B
:2040E00011F00C949F287DC48737910509F435C68C38910511F00C949F2896C18B3C910555
:2041000009F4E3C68C3C910550F4893C910509F450C68A3C910511F00C949F2890C68C3C07
:20412000910509F4E5C68D3C910511F00C949F2825C7B1E080399B0709F498C7E1E08139CB
:204140009E07E0F48D3D910509F480C78E3D910550F48F3C910509F418C78C3D910511F000
:204160000C949F2861C7F1E08F329F0709F4AAC48E55914011F00C949F28CAC731E0843F8C
:20418000930709F4ACC741E0853F940750F451E08139950709F46DC78259914009F0CFC75E
:2041A0006BC7B1E0863F9B0709F4AFC7E1E0863F9E0708F49CC7875F914009F0C0C7DEC6FD
:2041C00082EF9CE00E94B37ABAC782EF9CE00E94557EB5C782EF9CE00E94FB78B0C717FF35
:2041E000AEC782EF9CE060E00E947189D601D3966D917C91D49782EF9CE040E00E941C7A86
:204200009EC782EF9CE00E94137999C782EF9CE060E00E94877D93C712FF91C7F601478D5D
:2042200050A161A172A180915C0D882309F487C74093530D5093540D6093550D7093560DD6
:2042400082E39DE00E9402877AC782EF9CE00E94F77975C717FF73C7D601D3966D917C913A
:20426000D49782EF9CE00E94B87969C717FF67C782EF9CE060E00E947189F60163A974A9B6
:2042800082EF9CE00E9469795AC717FF58C782EF9CE060E00E947189D601D3966D917C9143
:2042A000D49782EF9CE00E943F7949C712FF47C713FF45C7F601878D90A1A1A1B2A1B7FD7A
:2042C0003EC78F3F9105A105B10511F00CF037C703A114A120E030E0F901EE0FFF1FE1556A
:2042E000FE4FE4918E2F90E08017910709F427C72F5F3F4F2833310579F717FD20C7802FEE
:2043000061E00E941AC4802FD6015F966C910E9497C4F601678D70A1802F0E949CC38AE74A
:2043200094E0B8010E94FC29D6015F966D917C91909786E894E00E94C42901C70E94A73ACF
:20434000882309F0FCC60E94E3C2609340047093410480934204909343048091270283FDB4
:20436000EEC6F6018081918193FD0AC092FF0AC0878D90A1A1A1B2A10097A105B10511F4F8
:204380000E94D31BD6018D919C91119792FFD7C65F968D909D90AD90BC9092979C01207077
:2043A000317091FF1EC05E960C91232B11F410E00FC010E0F601628D738D848D958D20E042
:2043C00030E040E050E00E94D8C718160CF411E0C501B4010E946CC6402F212F0E94F73E38
:2043E000AEC6E0917502F09176020081232B11F410E011C010E0D6015A966D917D918D91F2
:204400009C915D9720E030E040E050E00E94D8C718160CF411E0C501B4010E946CC6402FFD
:20442000212F0E94F73E8BC60E94A73A882309F086C60E94E3C260934004709341048093B8
:204440004204909343048091270283FD78C6F6018081918192FF73C6E78CF0A001A112A188
:2044600090FD02C0BB2412C0BB24D6015A966D917D918D919C915D9720E030E040E050E0EB
:204480000E94D8C7181614F4BB24B394C801B7010E946CC64B2D0E94303B51C683E0169580
:2044A00007958A95E1F7802F81700E944F1B47C60E94A73A882309F042C60E94E3C2609347
:2044C00040047093410480934204909343048091270283FD34C68EE89FE065E072E040E02D
:2044E0000E94BB988EE89FE00E9491B60E94D31B8090750290907602F6012081318131FFC0
:2045000007C0868D882321F41FE1812E11E0912E32FF27C0D6015F96ED90FD900D911C9169
:204520009297F401A08030FD02C0BB2412C0BB24D6015A966D917D918D919C915D9720E0AC
:2045400030E040E050E00E94D8C7181614F4BB24B394C801B7010E946CC64A2D2B2D0E9498
:20456000F73EF40164A575A586A597A520A931A942A953A90E9403C57B018C0120E030E07A
:2045800040E050E00E94D8C718165CF4C801B70120E030E040E050E40E94CAC5882364F4F3
:2045A000CEC5C801B70120E030E040E050EC0E94D8C718160CF4C3C53324D4019A962D916A
:2045C0003C919B9798968D919C9199978217930714F4332433940E94E3C269A77AA78BA730
:2045E0009CA744245524320110E00E94E3C26DA37EA38FA398A7DC01CB0129A53AA54BA545
:204600005CA5821B930BA40BB50B895E9340A040B04058F080E00E944F1B8DA19EA1AFA1F4
:20462000B8A589A79AA7ABA7BCA70E94B61B80917502909176028816990609F067C0D40131
:204640009396ED90FC9094971E141F040CF05EC0112309F05BC0332009F458C091966D91B9
:204660007C919297882777FD8095982F0E946CC69B01AC01F40164A575A586A597A50E94C7
:20468000D8C718160CF042C000D000D000D00DB71EB70F5F1F4F662777276E197F09882781
:2046A00077FD8095982F0E946CC62091E7013091E8014091E9015091EA010E947AC80E9486
:2046C00039C65B016C01F40187859089A189B289F80180839183A283B3831482158260E0BB
:2046E00070E080E090E020E030E040E050E0EE24FF2487010E94726911E02DB73EB72A5FAD
:204700003F4F0FB6F8943EBF0FBE2DBF411451046104710409F053C03320C9F0D401D0962D
:204720006D917D918D919C91D39720E030E040E85FE30E9403C59B01AC01F40164A575A573
:2047400086A597A50E94D8C787FF1AC04ECFD401D0966D917D918D919C91D39720E030E028
:2047600040E85FE30E9404C59B01AC01F40164A575A586A597A50E94CAC518160CF435CF39
:20478000D4015F966D917C919097882777FD8095982F28EE33E040E050E00E9450C92B01BE
:2047A0003C012DA13EA14FA158A5420E531E641E751E411451046104710409F416CFD30112
:2047C000C2012DA13EA14FA158A5821B930BA40BB50B80509449A543B74708F406CF11233A
:2047E00009F44AC080917502909176028816990609F042C000D000D000D00DB71EB70F5FE2
:204800001F4FD40193966D917C919497882777FD8095982F0E946CC62091E7013091E801E0
:204820004091E9015091EA010E947AC80E9439C65B016C01F40187859089A189B289F8012B
:2048400080839183A283B3831482158260E070E080E090E020E030E040E050E0EE24FF24C4
:2048600087010E9472692DB73EB72A5F3F4F0FB6F8943EBF0FBE2DBF1092CE0F0E94E3C276
:204880006093400470934104809342049093430456C423FD54C48EE89FE069EF71E040E0C6
:2048A0000E94BB988EE89FE00E9491B60E94D31BD6018D919C91119792FF21C05F96ED90E7
:2048C000FD900D911C91929790FD02C0BB2410C0BB24F601628D738D848D958D20E030E0D1
:2048E00040E050E00E94D8C7181614F4BB24B394C801B7010E946CC64B2D0E94303B609100
:204900009201709193018091940190919501209196013091970140919801509199010E94EA
:2049200003C57B018C0120E030E040E050E00E94D8C718165CF4C801B70120E030E040E4D2
:2049400050E40E94CAC5882364F4F9C3C801B70120E030E040E450EC0E94D8C718160CF4D3
:20496000EEC30E94E3C27B018C0114C00E94E3C26E197F09800B910B695E734080409040DB
:2049800038F080E00E944F1B0E94E3C27B018C010E94B61B60919201709193018091940101
:2049A0009091950120E030E040E05FE30E9404C520919601309197014091980150919901DD
:2049C0000E94CAC587FDD2CF1092CE0F0E94E3C26093400470934104809342049093430479
:2049E000AEC323FDACC30E94E3C24B015C010E94E3C2681979098A099B09695E734080400C
:204A0000904038F080E00E944F1B0E94E3C24B015C010E94B61BC090CC01D090CD01D601AD
:204A20001B96ED90FD900D911C911E97C801B70120E030E040EF51E40E94D8C71816A4F4BF
:204A4000C801B701F60127813085418552850E9403C59F7720E030E040E85FE30E94D8C7A9
:204A6000181614F4772402C077247394C090CE01D090CF01D6011B96ED90FD900D911C91D5
:204A80001E97C801B70120E030E040EF51E40E94D8C718169CF4C801B701F6012781308598
:204AA000418552850E9403C59F7720E030E040E85FE30E94D8C718160CF499CF772009F4F4
:204AC00096CF3DC312FD03C026E930E005C0D6015F962D913C91909713FD03C0CC24DD2479
:204AE0000AC0F601C3A0D4A0F2E0CF16D1041CF0B2E0CB2ED12CF601EE0FFF1FE453FE4F68
:204B0000E080F180B901882777FD8095982F0E946CC6AB01BC01E3E016950795EA95E1F76D
:204B20000170C7012C2D0E94973B09C312FD03C08FEF90E005C0D6015F968D919C919097E0
:204B4000612F66956695669561700E94E11BF7C2612F669566956695617080E090E00E94E8
:204B6000E11BEDC21092BA0BEAC281E08093BA0BE6C212FF14C0F601678D70A181A192A160
:204B800028EE33E040E050E00E9450C96093D1017093D2018093D3019093D401D0C20E9433
:204BA000D31B81E00E942F75CAC212FF16C0D6015F966D917D918D919C91929728EE33E078
:204BC00040E050E00E9450C960934404709345048093460490934704B2C210924404109278
:204BE00045041092460410924704A9C203FF0DC0F60182859385A485B5858093DB019093CE
:204C0000DC01A093DD01B093DE01D6018C9184FF0EC01E968D919D910D90BC91A02D809375
:204C2000DF019093E001A093E101B093E201F601808185FF0CC082899389A489B589809368
:204C4000E3019093E401A093E501B093E6010E94D975D6018C9186FF72C2E0917502F0911F
:204C6000760256962D913D914D915C915997218732874387548780810E94BD3F60C212FDB3
:204C800007C040E1842E47E2942EA12CB12C0DC0F601678D70A181A192A128EE33E040E07E
:204CA00050E00E9450C94B015C0103FD5E9A04FD5E9A05FD159A0E94E3C27B018C01E80C7A
:204CC000F91C0A1D1B1D02C00E947D750E94E3C2A8019701261B370B480B590BDA01C901A3
:204CE000805A9648A140B04078F3D6013C9133FD5E9834FD5E9835FF22C2159820C212FF17
:204D000004C0F601878D809327028091270283FF16C260E070E080E090E040E020E00E94D2
:204D2000F73E0DC286E192E00E94282A0E946C1A06C20E94361903C217FF01C2D601D396E3
:204D40006D917C91D4978EE89FE040E00E94E7988EE89FE00E9491B6F2C10E94D31B81E91C
:204D600094E00E94A129329B03C08EE894E002C08BE894E00E94A1298FE994E00E94A1296C
:204D8000339B03C08EE894E002C08BE894E00E94A1298DEA94E00E94A129349B03C08EE824
:204DA00094E002C08BE894E00E94A1290E945D1AC6C103FF0DC0F60182859385A485B58582
:204DC0008093070290930802A0930902B0930A02D6018C9184FF0EC01E968D919D910D901B
:204DE000BC91A02D80930B0290930C02A0930D02B0930E02F601808185FF0CC08289938944
:204E0000A489B58980930F0290931002A0931102B0931202D6018C9186FF0EC056968D91E0
:204E20009D910D90BC91A02D8093130290931402A0931502B09316020E94D97580C103FF54
:204E40000DC0F60182859385A485B5858093170290931802A0931902B0931A02D6018C9102
:204E600084FF0EC01E968D919D910D90BC91A02D80931B0290931C02A0931D02B0931E0204
:204E8000F601808185FF0CC082899389A489B58980931F0290932002A0932102B093220202
:204EA000D6018C9186FF0EC056968D919D910D90BC91A02D8093230290932402A0932502E1
:204EC000B09326020E94D9753AC112FF38C1F601278D30A141A152A11216130614061506AB
:204EE0001CF020931C012BC181E080931C0127C1809175029091760212FD03C0FC01B59636
:204F000010C0F601878D90A1A1A1B2A1B7FD17C10097A105B10519F4E4E4F1E002C0EBE836
:204F2000F1E003FF0BC0D6011A962D913D914D915C911D97228F338F448F558FD6018C9123
:204F400084FF0AC01E962D913D914D915C915197268F378F40A351A3D6018C9185FF0AC07D
:204F600052962D913D914D915C91559722A333A344A355A3CF010E94D737E1C00E946C2C31
:204F8000DEC0C6010E947735DAC003FF0DC0F60182859385A485B5858093720C9093730C49
:204FA000A093740CB093750CD6018C9186FF11C0E0917502F091760256962D913D914D91F9
:204FC0005C915997278B308F418F528F80810E94BD3FF601808185FF0CC082899389A48997
:204FE000B5898093760C9093770CA093780CB093790C4091720C5091730C6091740C709198
:20500000750C8BEB94E022E00E94FF2A4091760C5091770C6091780C7091790C81EC94E0C5
:2050200022E00E943B2B8BC012FD05C024E630E040E050E007C0D6015F962D913D914D91E0
:205040005C919297C9010E94D41879C012FD05C024E630E040E050E005C0F601278D30A12A
:2050600041A152A1C9010E94BF1869C00E94D31B66C00E94666B63C010FF08C0D6015A9605
:20508000CD90DD90ED90FC905D9708C0C0906A0CD0906B0CE0906C0CF0906D0CB80134E036
:2050A000769567953A95E1F76170A80125E0569547952A95E1F74170980196E0369527951E
:2050C0009A95E1F7217083E0169507958A95E1F7802F8170870176010E94957430C080E0FD
:2050E0000E94EC2E85E097E00E94472A28C00E940932E0917502F091760280810E94BD3FC0
:2051000085E297E00E94472A1AC00E94F23517C087EE91E00E94282A12C011FF07C00E94FF
:20512000D31BF601868D0E94BD3F09C022FF07C080EA93E00E94A129C6010E946544E09657
:205140000FB6F894DEBF0FBECDBFCF91DF911F910F91FF90EF90DF90CF90BF90AF909F904F
:205160008F907F906F905F904F903F902F900895CF93DF930E94C8490E945444EC018EE8E5
:205180009FE00E94B5992097D1F080915D0D882381F0888181FF04C08E819F814D9791F0B0
:2051A00082EF9CE0BE010E94597BCE010E94BE4803C0CE010E94101CCE010E94CF480E94CC
:2051C0007D75D8CF82EF9CE00E949879EECFCF93DF9320C080915D0D882381F0888181FF05
:2051E00004C08E819F814D9739F182EF9CE0BE010E94597BCE010E94BE4803C0CE010E94E1
:20520000101CCE010E94CF480E94B61B8EE89FE00E94B5998091810B882329F40E945444E3
:20522000EC01009771F00E94C8498EE89FE00E94B599209779F6E8CF82EF9CE00E94987974
:20524000D9CFDF91CF910895CF93DF93EC0105C0219683E294E00E94624E68816623C1F7A7
:20526000DF91CF910895AF92BF92CF92DF92EF92FF920F931F93DF93CF93CDB7DEB72B9748
:205280000FB6F894DEBF0FBECDBFC62ED92E1B869BE0A92EB12CAC0EBD1E6C2D9D2D2AE0FA
:2052A00030E040E050E00E94A3C9D52E7901042F152F80E3C80EC801B7012AE030E040E098
:2052C00050E00E9450C9C61AF501C2925F01CE2C7F2D802FE114F10401051105F1F6CF0147
:2052E0000E9424292B960FB6F894DEBF0FBECDBFCF91DF911F910F91FF90EF90DF90CF90BB
:20530000BF90AF900895EF92FF920F931F937B018C0197FF0DC083E294E06DE20E94624E16
:2053200010950095F094E094E11CF11C011D111DC801B7010E9433291F910F91FF90EF9008
:205340000895CF93DF93EC0104C083E294E00E94624EFE01649121966623B9F7DF91CF914C
:205360000895EF92FF920F931F937A018B010E94A129C801B7010E9433290E945D1A1F916F
:205380000F91FF90EF900895EF92FF920F931F937B010E94A1290027F7FC0095102FC801BD
:2053A000B7010E9483290E945D1A1F910F91FF90EF900895EF92FF920F931F937A018B0166
:2053C0000E94A129C801B7010E9433291F910F91FF90EF900895EF92FF920F931F937A0106
:2053E0008B010E94A129C801B7010E9483291F910F91FF90EF900895EF92FF920F931F9385
:205400007B010E94A1290027F7FC0095102FC801B7010E9483291F910F91FF90EF900895EC
:205420000F931F938B010E94A129C8010E9424291F910F9108950F931F938B010E94A1292F
:20544000C8010E9424290E945D1A1F910F9108950E94A1290E945D1A08950F931F938C018B
:205460008BE992E00E94A129C8010E94282A1F910F9108950F931F938C0182EA92E00E94CF
:20548000A129C8010E94282A1F910F9108950F931F938C0182EA92E00E94A129C8010E9402
:2054A000A1291F910F9108959F92AF92BF92CF92DF92EF92FF920F931F93CF93DF937B01EA
:2054C0008C01942EA80197010E9434C9882319F083E992E020C0C0E0D0E057016801E8949E
:2054E000D7F8C601B5012FEF3FEF4FE75FE70E9434C9882351F4C601B5012FEF3FEF4FE70A
:205500005FE70E94CAC5181614F0C1E0D0E0219729F087E992E00E94A12965C0C801B701CC
:2055200020E030E040E050E00E94CAC588234CF483E294E06DE20E94624E17FB109517F9AE
:20554000109520E030E040E05FE3DD240BC0CA01B90120E030E040E251E40E94D1C59B01A8
:20556000AC01D394D91498F3C801B7010E9404C55B016C010E943EC67B018C010E9433293D
:20558000992029F083E294E06EE20E94624EC801B7010E946AC69B01AC01C601B5010E9403
:2055A00003C51FC020E030E040E251E40E947AC87B018C010E9439C65B016C01CC24B7FCE3
:2055C000C094DC2CC601B5010E948329C601B5010E946CC69B01AC01C801B7010E9403C51F
:2055E0009A949920F9F6DF91CF911F910F91FF90EF90DF90CF90BF90AF909F900895DF920E
:20560000EF92FF920F931F937A018B01D22E0E94A129C801B7014D2D0E94542A1F910F9146
:20562000FF90EF90DF900895EF92FF920F931F93CF93DF93162F072FE42EF22E0E94A129FD
:20564000212F302FC901EC0110E00AC049915991699179918DE594E02F2D0E94FF2A1F5FD7
:205660001E15A0F30E945D1ADF91CF911F910F91FF90EF900895DF92EF92FF920F931F93A9
:205680007A018B01D22E0E94A129C801B7014D2D0E94542A0E945D1A1F910F91FF90EF9005
:2056A000DF9008959C01F999FECF32BD21BDF89A80B508959C01F999FECF1FBA32BD21BD0F
:2056C00060BD0FB6F894FA9AF99A0FBE0895885C904022E08835920778F464E670E00E9417
:2056E0007CC96F5F7F4F8CE897E00E94FC2983E294E060E20E94624E08950F931F93CF9357
:20570000DF93EC018B0182E997E0BE010E94FC2983E294E060E20E94624EF999FECFD2BDDB
:20572000C1BDF89A60B570E0882777FD8095982F0E94832983E294E060E20E94624ECE016B
:205740000E94672BC8010E94282ADF91CF911F910F910895CF92DF92EF92FF920F931F9363
:205760008C016B0189E997E0B8010E94FC2983E2E82E84E0F82EC70160E20E94624EC8019D
:2057800062E57BE20E943518AA2797FDA095BA2FBC01CD010E948329C70160E20E94624EBE
:2057A000C8010E94672BC6010E94282A1F910F91FF90EF90DF90CF900895CF92DF92EF9215
:2057C000FF920F931F938C016B0180EA97E0B8010E94FC2993E2E92E94E0F92EC70160E259
:2057E0000E94624EC80162E57BE20E940F180E948329C70160E20E94624EC8010E94672B7A
:20580000C6010E94282A1F910F91FF90EF90DF90CF900895F999FECF12BC11BCF89A80B543
:20582000823071F48BE490E062E57BE20E940F186093D5017093D6018093D7019093D8017B
:205840000895DF93CF9300D000D0CDB7DEB7BC01CE01019644E050E022E53BE20E94F317D7
:2058600029813A814B815C81B901CA010F900F900F900F90CF91DF910895BF92CF92DF9289
:20588000EF92FF920F931F938C016B01B42E87EA97E0B8010E94FC2923E2E22E24E0F22E26
:2058A000C70160E20E94624EC8010E94212C4B2D0E94542AC70160E20E94624EC8010E9475
:2058C000672BC6010E94282A1F910F91FF90EF90DF90CF90BF9008958BE490E06EEA77E0D5
:2058E0000E94DD2B81E890E067EB77E043E00E943D2C8DE790E06CEC77E00E94DD2B8FE49E
:2059000090E06FED77E00E94DD2B83E590E06DEF77E00E94DD2B83E090E060EE78E044E0E8
:205920000E943D2C87E090E064EF78E044E00E943D2C8BE090E068E079E044E00E943D2C00
:205940008FE090E06CE179E043E00E943D2C83E190E068E379E043E00E943D2C87E190E016
:2059600064E579E043E00E943D2C8BE190E060E779E043E00E943D2C8FE190E06EE879E01E
:2059800043E00E943D2C83E290E06CEA79E043E00E943D2C87E290E06CEB78E043E00E94DA
:2059A0003D2C8FE290E06DEC78E043E00E943D2C85E890E066E278E043E00E943D2C89E8A2
:2059C00090E066E378E043E00E943D2C8DE890E066E478E043E00E943D2C81E990E066E5AE
:2059E00078E043E00E943D2C85E990E068E678E043E00E943D2C89E990E06AE778E043E0C1
:205A00000E943D2C83E390E06AEC79E043E00E943D2C87E390E067EE79E043E00E943D2C12
:205A20008BE390E064E07AE043E00E943D2C8FE390E061E27AE043E00E943D2C83E490E038
:205A400065E47AE043E00E943D2C87E490E069E67AE043E00E943D2C80E793E06EEE76E037
:205A60000E947D2B8AE690E06AE37BE00E947D2B8BE690E061E57BE00E947D2B8CE790E05B
:205A800063E67BE00E947D2B8CE690E065E77BE043E00E943D2C80E790E064E87BE043E0C0
:205AA0000E943D2C84E790E063E97BE043E00E943D2C88E790E062EA7BE00E947D2B88ECE7
:205AC00090E06CEB7BE043E00E943D2C8CEC90E069EC7BE043E00E943D2C80ED90E06EED78
:205AE0007BE043E00E943D2C84ED90E064EF7BE043E00E943D2C88ED90E06AE07CE00E9433
:205B00007D2B89ED90E06DE17CE00E947D2B85EF90E06BE27CE00E947D2B8AED90E069E3F9
:205B20007CE044E00E943D2C8EED90E06EE47CE044E00E943D2C82EE90E069E57CE044E064
:205B40000E943D2C86EE90E064E67CE00E947D2B87EE90E06AE77CE00E94DD2B8BEE90E041
:205B60006BE87CE00E94DD2B8FEE90E06CE97CE00E94AA2B8AEF90E065EB7CE00E94AA2BAB
:205B80008CEF90E06BED7CE00E94AA2B8EEF90E061E07DE00E947D2B0895DF93CF9300D0D9
:205BA00000D0CDB7DEB749835A836B837C83BE016F5F7F4F44E050E02AE53BE20E944B1886
:205BC0000F900F900F900F90CF91DF91089588E293E040E050E060E272E40E94CD2D8CE20D
:205BE00093E040E050E060E070E40E94CD2D88E493E040E050E066E173E40E94CD2D80E2E7
:205C000093E040E050E060E070E00E94CD2D84E293E040E050E060E070E00E94CD2D80E3DD
:205C200093E040E050E060EA71E40E94CD2D84E393E040E050E060EA71E40E94CD2D88E396
:205C400093E040E050E060E273E40E94CD2D8CE393E040E050E060EA71E40E94CD2D80E47B
:205C600093E040E050E068EC72E40E94CD2D84E493E040E050E060E273E40E94CD2D81EA50
:205C800093E040E050E060E271E40E94CD2D0895EF92FF920F931F936091880C7091890CF0
:205CA00080918A0C90918B0C20E030E040E050E00E94CAC5882309F48AC00E94E3C220910A
:205CC000840C3091850C4091860C5091870C621B730B840B950B28EE33E040E050E00E94C6
:205CE000A3C979018A018DE790E062E57BE20E940F18E60EF71E081F191F8DE790E0B801DD
:205D0000A7012AE53BE20E94671881E890E00E94212C7B018C016091880C7091890C809191
:205D20008A0C90918B0C2FE632E143E85AE30E947AC89B01AC01C801B7010E9404C5AB01C0
:205D4000BC0181E890E00E94CD2D80E090E0A0E0B0E08093880C9093890CA0938A0CB093C6
:205D60008B0C0E94E3C26093840C7093850C8093860C9093870C20E030E040E0283631050F
:205D800039F0F999FECF32BD21BDF89A80B5480F2F5F3F4F88E02030380781F7F999FECFA6
:205DA00088E690E092BD81BDF89A80B5481769F0F999FECF1FBA88E690E092BD81BD40BD59
:205DC0000FB6F894FA9AF99A0FBE0E946C1A1F910F91FF90EF900895FF920F931F93CF9314
:205DE000DF93F82E4091D5015091D6016091D7017091D8018BE490E02AE53BE20E946718DD
:205E0000409144045091450460914604709147048FE490E02AE53BE20E9467184091D101E5
:205E20005091D2016091D3017091D40183E590E02AE53BE20E9467184091DB015091DC0183
:205E40006091DD017091DE0183E090E00E94CD2D4091DF015091E0016091E1017091E201FA
:205E600087E090E00E94CD2D4091E3015091E4016091E5017091E6018BE090E00E94CD2DFE
:205E80004091EB015091EC016091ED017091EE018FE090E00E94CD2D4091EF015091F0019A
:205EA0006091F1017091F20183E190E00E94CD2D4091F3015091F4016091F5017091F60121
:205EC00087E190E00E94CD2D4091FB015091FC016091FD017091FE018BE190E00E94CD2D3C
:205EE0004091FF015091000260910102709102028FE190E00E94CD2D4091030250910402BC
:205F0000609105027091060283E290E00E94CD2D4091720C5091730C6091740C7091750C6D
:205F200087E290E00E94CD2D4091760C5091770C6091780C7091790C8FE290E00E94CD2DBD
:205F400040910702509108026091090270910A0283E390E00E94CD2D40910B0250910C0234
:205F600060910D0270910E0287E390E00E94CD2D40910F02509110026091110270911202AC
:205F80008BE390E00E94CD2D40911702509118026091190270911A028FE390E00E94CD2DFB
:205FA00040911B0250911C0260911D0270911E0283E490E00E94CD2D40911F02509120025B
:205FC000609121027091220287E490E00E94CD2D20919E01F999FECF1FBA8AE690E092BD5A
:205FE00081BD20BD0FB6F894FA9AF99A0FBE2091A301F999FECF1FBA8BE690E092BD81BD46
:2060000020BD0FB6F894FA9AF99A0FBE2091A401F999FECF1FBA8CE790E092BD81BD20BD83
:206020000FB6F894FA9AF99A0FBE4091A5015091A6016091A7017091A8018CE690E00E9455
:20604000CD2D4091A9015091AA016091AB017091AC0180E790E00E94CD2D4091AD01509121
:20606000AE016091AF017091B00184E790E00E94CD2D2091B101F999FECF1FBA88E790E02D
:2060800092BD81BD20BD0FB6F894FA9AF99A0FBE4091560C5091570C6091580C7091590C1F
:2060A00085E890E00E94CD2D40915E0C50915F0C6091600C7091610C89E890E00E94CD2D98
:2060C0004091660C5091670C6091680C7091690C8DE890E00E94CD2D4091520C5091530C5E
:2060E0006091540C7091550C81E990E00E94CD2D40915A0C50915B0C60915C0C70915D0C35
:2061000085E990E00E94CD2D4091620C5091630C6091640C7091650C89E990E00E94CD2D25
:206120008DE990E040E050E060E070E00E94CD2D81EA90E040E050E060E070E00E94CD2DA6
:2061400085EA90E040E050E060E070E00E94CD2D2091FF0BF999FECF1FBA80E793E092BDC8
:2061600081BD822F90E045E0969587954A95E1F7817080BD0FB6F894FA9AF99A0FBE02E048
:206180001CE0C0E0D0E0CE01880F991F880F991FF80141915191619171918F01845B9C4F4B
:2061A0000E94CD2D2196C930D10569F7409128015091290160912A0170912B0188EC90E02B
:2061C0000E94CD2D40912E0150912F0160913001709131018CEC90E00E94CD2D4091360131
:2061E00050913701609138017091390180ED90E00E94CD2D40913201509133016091340169
:206200007091350184ED90E00E94CD2D20915701F999FECF1FBA88ED90E092BD81BD20BD3A
:206220000FB6F894FA9AF99A0FBE20915C01F999FECF1FBA89ED90E092BD81BD20BD0FB6BE
:20624000F894FA9AF99A0FBE20915D01F999FECF1FBA85EF90E092BD81BD20BD0FB6F894D8
:20626000FA9AF99A0FBE40915E0150915F0160916001709161018AED90E00E94CD2D4091B0
:2062800062015091630160916401709165018EED90E00E94CD2D40916601509167016091A0
:2062A00068017091690182EE90E00E94CD2D20916A01F999FECF1FBA86EE90E092BD81BDC9
:2062C00020BD0FB6F894FA9AF99A0FBE4091200150912101609122017091230187EE90E089
:2062E0002AE53BE20E946718409124015091250160912601709127018BEE90E02AE53BE2FE
:206300000E94671860913E0170913F018FEE90E04AE55BE20E948D186091400170914101D6
:206320008AEF90E04AE55BE20E948D1860914201709143018CEF90E04AE55BE20E948D18AA
:2063400020918901F999FECF1FBA8EEF90E092BD81BD20BD0FB6F894FA9AF99A0FBE81EFBE
:2063600090E040E050E060E070E00E94CD2D86EF90E040E050E060E070E00E94CD2DFF20B1
:20638000A1F08DE790E040E050E060E070E02AE53BE20E94671881E890E040E050E060E0F2
:2063A00070E00E94CD2D0E94E72DF999FECF1FBA89E690E092BD81BD87E080BD0FB6F894A2
:2063C000FA9AF99A0FBE20E030E040E02836310539F0F999FECF32BD21BDF89A80B5480F92
:2063E0002F5F3F4FF8E020303F0781F7F999FECF1FBA88E690E092BD81BD40BD0FB6F894AA
:20640000FA9AF99A0FBEDF91CF911F910F91FF900895DF92EF92FF920F931F93CF93DF9391
:20642000F999FECF89E690E092BD81BDF89AD0B48BE490E062E57BE20E940F186093D50166
:206440007093D6018093D7019093D8018FE490E062E57BE20E940F186093440470934504A4
:20646000809346049093470483E590E062E57BE20E940F186093D1017093D2018093D3018A
:206480009093D40183E090E00E94212C6093DB017093DC018093DD019093DE0187E090E0C9
:2064A0000E94212C6093DF017093E0018093E1019093E2018BE090E00E94212C6093E3019A
:2064C0007093E4018093E5019093E6018FE090E00E94212C6093EB017093EC018093ED0133
:2064E0009093EE0183E190E00E94212C6093EF017093F0018093F1019093F20187E190E0FD
:206500000E94212C6093F3017093F4018093F5019093F6018BE190E00E94212C6093FB01D0
:206520007093FC018093FD019093FE018FE190E00E94212C6093FF0170930002809301024B
:206540009093020283E290E00E94212C6093030270930402809305029093060287E290E031
:206560000E94212C6093720C7093730C8093740C9093750C8FE290E00E94212C6093760CBD
:206580007093770C8093780C9093790C83E390E00E94212C6093070270930802809309024A
:2065A00090930A0287E390E00E94212C60930B0270930C0280930D0290930E028BE390E09F
:2065C0000E94212C60930F027093100280931102909312028FE390E00E94212C6093170279
:2065E000709318028093190290931A0283E490E00E94212C60931B0270931C0280931D02E8
:2066000090931E0287E490E00E94212C60931F02709320028093210290932202F999FECF58
:206620008AE690E092BD81BDF89A80B580939E01F999FECF8BE690E092BD81BDF89A80B5E0
:206640008093A301F999FECF8CE790E092BD81BDF89A80B58093A4018CE690E00E94212C64
:206660006093A5017093A6018093A7019093A80180E790E00E94212C6093A9017093AA013F
:206680008093AB019093AC0184E790E00E94212C6093AD017093AE018093AF019093B001B7
:2066A000F999FECF88E790E092BD81BDF89A80B58093B10185E890E00E94212C6093560C62
:2066C0007093570C8093580C9093590C89E890E00E94212C60935E0C70935F0C8093600C3B
:2066E0009093610C8DE890E00E94212C6093660C7093670C8093680C9093690C81E990E062
:206700000E94212C6093520C7093530C8093540C9093550C85E990E00E94212C60935A0CBA
:2067200070935B0C80935C0C90935D0C89E990E00E94212C6093620C7093630C8093640CC1
:206740009093650C82E08D1508F050C002E01CE07801C0E0D0E0CE01880F991F880F991F85
:20676000845B9C4F0E94212CF70161937193819391937F012196C930D10569F72091020C13
:206780003091030C4091040C5091050CCA01B9010E9434C98823A1F0CCE4D3E0CE01880F2D
:2067A000991F880F991F0E94212CF80161937193819391938F012196F3E0C535DF0771F758
:2067C000F999FECF80E793E092BD81BDF89A80B590E0811191E0892F0E94B66B82EA92E060
:2067E00062E07CE049E026E00E94142B88EC90E00E94212C609328017093290180932A0191
:2068000090932B018CEC90E00E94212C60932E0170932F01809330019093310180ED90E087
:206820000E94212C6093360170933701809338019093390184ED90E00E94212C6093320165
:20684000709333018093340190933501F999FECF88ED90E092BD81BDF89A80B5809357015D
:20686000F999FECF89ED90E092BD81BDF89A80B580935C01F999FECF85EF90E092BD81BD3F
:20688000F89A80B580935D018AED90E00E94212C60935E0170935F0180936001909361013C
:2068A0008EED90E00E94212C6093620170936301809364019093650182EE90E00E94212C71
:2068C00060936601709367018093680190936901F999FECF86EE90E092BD81BDF89A80B553
:2068E00080936A0187EE90E062E57BE20E940F186093200170932101809322019093230112
:206900008BEE90E062E57BE20E940F18609324017093250180932601909327018FEE90E06E
:2069200062E57BE20E94351890933F0180933E018AEF90E062E57BE20E943518909341012E
:20694000809340018CEF90E062E57BE20E943518909343018093420181E08D1570F4F999AF
:20696000FECF8EEF90E092BD81BDF89A80B580938901E7E0DE1609F46EC088E697E00E94FF
:206980003A2AF2E0FD1508F458C088E293E040E050E060E272E40E94CD2D8CE293E040E039
:2069A00050E060E070E40E94CD2D88E493E040E050E066E173E40E94CD2D80E293E040E019
:2069C00050E060E070E00E94CD2D84E293E040E050E060E070E00E94CD2D80E393E040E010
:2069E00050E060EA71E40E94CD2D84E393E040E050E060EA71E40E94CD2D88E393E040E0C9
:206A000050E060E273E40E94CD2D8CE393E040E050E060EA71E40E94CD2D80E493E040E0AD
:206A200050E068EC72E40E94CD2D84E493E040E050E060E273E40E94CD2D86E08D1540F048
:206A400081EA93E040E050E060E271E40E94CD2D80E00E94EC2E0E94D9750E941E38DF9161
:206A6000CF911F910F91FF90EF90DF9008950F931F9320E030E010E02836310539F0F999A9
:206A8000FECF32BD21BDF89A80B5180F2F5F3F4F88E02030380781F7F999FECF88E690E0A6
:206AA00092BD81BDF89A00B5F999FECF12BC11BCF89A80B5823029F4011719F40E94093270
:206AC00013C0F999FECF1FBA12BC11BC82E080BD0FB6F894FA9AF99A0FBE0E94E72D80E016
:206AE000011381E00E94EC2E1F910F910895FC018081918191FF42C093FF40C0268D213040
:206B0000D9F0213030F0223011F1233009F036C02BC092FF33C023A134A145A156A1878DAC
:206B2000F999FECF1FBA32BD21BD80BD0FB6F894FA9AF99A0FBE22C092FF20C0678D70A176
:206B400083A194A14AE55BE20E948D1817C092FF15C0478D50A161A172A183A194A12AE5AA
:206B60003BE20E9467180AC083FF08C0428553856485758583A194A10E94CD2D20E030E03C
:206B800040E02836310539F0F999FECF32BD21BDF89A80B5480F2F5F3F4F88E020303807BB
:206BA00081F7F999FECF88E690E092BD81BDF89A80B5481769F0F999FECF1FBA88E690E0FE
:206BC00092BD81BD40BD0FB6F894FA9AF99A0FBE0E940932E0917502F091760280810E9485
:206BE000BD3F0895EF92FF920F931F9380E092ECA1E0B0E08093D5019093D601A093D701B9
:206C0000B093D8011092440410924504109246041092470480E49EE7A5E0B0E08093D101C7
:206C20009093D201A093D301B093D4010F2EF0E0EF2EF0E0FF2EF8EC0F2FF2E41F2FF02DB5
:206C4000E092DB01F092DC010093DD011093DE01E092DF01F092E0010093E1011093E201E4
:206C600020E030E048EC53E42093E3013093E4014093E5015093E60180E090E0A0E8BFE3DD
:206C80008093E7019093E801A093E901B093EA012093EB013093EC014093ED015093EE01C0
:206CA0002093EF013093F0014093F1015093F20180E090E0A0E0B1E48093F3019093F401DE
:206CC000A093F501B093F601E092FB01F092FC010093FD011093FE01E092FF01F09200023B
:206CE000009301021093020280E090E0A0E8B0E48093030290930402A0930502B0930602A5
:206D00000F2EF0E0EF2EF0E0FF2EF0EA0F2FF1E41F2FF02DE092720CF092730C0093740CF0
:206D20001093750C8AE999E9A9E9BEE38093760C9093770CA093780CB093790C2093070291
:206D4000309308024093090250930A0220930B0230930C0240930D0250930E0220930F026F
:206D600030931002409311025093120220931702309318024093190250931A0220931B02FB
:206D800030931C0240931D0250931E0220931F0230932002409321025093220210929E0126
:206DA0002FEF2093A30180E58093A40180E090E0A4E4B3E48093A5019093A601A093A701F4
:206DC000B093A80180E090E0A4E0B2E48093A9019093AA01A093AB01B093AC0180E090E0B3
:206DE000A1E9B3E48093AD019093AE01A093AF01B093B0012093B10180E090E0AAE7B3E4AB
:206E00008093520C9093530CA093540CB093550C80E090E0A4E6B3E480935A0C90935B0C54
:206E2000A0935C0CB0935D0C80E090E0A0E7B3E48093620C9093630CA093640CB093650CB3
:206E400080E090E0A0E0B0E08093560C9093570CA093580CB093590C80935E0C90935F0C0D
:206E6000A093600CB093610C8093660C9093670CA093680CB093690C80E090E0AEEBB2E44A
:206E80008093280190932901A0932A01B0932B0180E090E0A8E4B2E480932E0190932F0115
:206EA000A0933001B0933101E0923601F0923701009338011093390180E090E0AAE7B4E4F4
:206EC0008093320190933301A0933401B093350183E08093570186EE80935C0182E380930A
:206EE0005D0180E090E0A0EEB0E480935E0190935F01A0936001B093610180E090E0A0E0C4
:206F0000B0E48093620190936301A0936401B093650180E090E0A0E2B2E48093660190931A
:206F20006701A0936801B093690120936A0180EE9CEFAFEFBFEF8093240190932501A09389
:206F40002601B093270188E494EFAFEFBFEF8093200190932101A0932201B093230181E0CD
:206F600090E090933F0180933E0186E990E0909341018093400110924301109242012093D6
:206F800089010E94E72D0E94D975E0917502F091760280810E94BD3F0E941E3887E497E067
:206FA0000E94472A1F910F91FF90EF900895EF92FF920F931F93CF93DF93EC018B898130D7
:206FC000B1F5EE8CFF8C08A119A1C801B70120E030E040E050E00E94CAC5882341F1688DBF
:206FE00070E080E090E00E946AC620E030E040E251E40E947AC8A80197010E94D1C56FA3C9
:2070000078A789A79AA7698D70E080E090E00E946AC620E030E040E251E40E947AC8A80104
:2070200097010E94D1C56BA77CA78DA79EA7DF91CF911F910F91FF90EF9008958BE891E023
:207040000E94D7370895E091CE01F091CF012781308541855285B901CA0108952F923F92A4
:207060004F925F926F927F928F929F92AF92BF92CF92DF92EF92FF920F931F93CF93DF933C
:207080001C01DC0111964C91453338F44233F8F4842F81508C3058F50AC0443628F4413609
:2070A00030F44C3321F513C0443609F510C0D1011296EC911297F0E0EE0FFF1FE159FD4FEB
:2070C000208131818CEF9FE0821B930B0BC0D1011296EC911297F0E0EE0FFF1FE159FD4F4C
:2070E0008081918114969C938E93139705C08FEF9FE0F10194838383D1011396ED90FC9084
:207100001497453348F4423308F053C0842F81508C3008F000C107C04C3309F4C9C0443651
:2071200009F0F9C0DEC090E0FC01EE57F14F4491440FFC01EE0FFF1FE257F14F25913491D9
:20714000F90145905490F9013296659074900CEF1FE00E191F0982E029C0E82FF0E0EE0F49
:20716000FF1FE20FF31F859094908F5FE82FF0E08150EE0FFF1FE20FF31FC591D491081519
:2071800019058CF4B301882777FD8095982F0E946CC65B016C01B80164197509882777FD2A
:2071A0008095982F44C08E5F3E0124018417A8F273C04E52842F90E0FC01EE57F14F44911C
:2071C000440FFC01EE0FFF1FE257F14F25913491F90145905490F90132966590749082E080
:2071E00058C0E82FF0E0EE0FFF1FE20FF31F859094908F5FE82FF0E08150EE0FFF1FE20F87
:20720000F31FC591D491E814F9040CF03FC0B301882777FD8095982F0E946CC65B016C015D
:20722000E418F508B701882777FD8095982F0E946CC67B018C01C619D709BE01882777FD20
:207240008095982F0E946CC69B01AC01C801B7010E947AC87B018C0184189508B40188272A
:2072600077FD8095982F0E946CC69B01AC01C801B7010E94D1C59B01AC01C601B5010E9480
:2072800004C520E030E040E05EE323C08E5F3E012401841708F4A5CFBE01882777FD80957E
:2072A000982F0E946CC620E030E040E05EE32AC0B701882777FD8095982F0E946CC620E04D
:2072C00030E04AE754E40E947AC820E030E040E859E30E947AC8F101678370878187928705
:2072E0001AC0B701882777FD8095982F0E946CC620E030E040EF53E40E947AC820E030E0BF
:2073000040E859E30E947AC8D10117966D937D938D939C931A97DF91CF911F910F91FF90E7
:20732000EF90DF90CF90BF90AF909F908F907F906F905F904F903F902F900895CF92DF924B
:20734000EF92FF920F931F93CF93DF936C01FC014387548765877687CB01BA0120E030E064
:2073600040E051E40E947AC80E9439C6DB01F6018181853340F4823308F068C081508C3010
:2073800008F0DCC007C08C3309F4B2C0843609F0D5C0BFC090E0FC01EE57F14F1491110FE6
:2073A000FC01EE0FFF1FE257F14F65917491FB0125913491FB013296E590F49082E03BC0B0
:2073C000E82FF0E0EE0FFF1FE60FF71F459154918F5FE82FF0E08150EE0FFF1FE60FF71F19
:2073E000C591D491CA17DB071CF50CEF1FE0021B130B241B350BB901882777FD8095982F91
:2074000097012A1B3B0B442737FD4095542F0E9450C9EC1AFD0A9701442737FD4095542FFB
:207420000E94C5C9020F131FF6011683058386C08E5F7E019A01811708F4C2CF8CEF9FE055
:20744000841B950BF6019683858378C08E5290E0FC01EE57F14F6491660FFC01EE0FFF1F49
:20746000E257F14F45915491FA01E590F490FA0132960591149182E037C0E82FF0E0EE0FA9
:20748000FF1FE40FF51F259134918F5FE82FF0E08150EE0FFF1FE40FF51FC591D491AC1706
:2074A000BD07FCF4B701621B730B882777FD8095982F98012A1B3B0B442737FD4095542F4B
:2074C0000E9450C90C1B1D0B9801442737FD4095542F0E94C5C9E20EF31EF601F682E5820B
:2074E0002DC08E5F8E017901861708F4C6CF23C0BD01882777FD8095982F3CE0660F771FB4
:20750000881F991F3A95D1F728EE33E040E050E010C0BD01882777FD8095982F2CE0660FEE
:20752000771F881F991F2A95D1F724EF31E040E050E00E94C5C9F60136832583DF91CF9103
:207540001F910F91FF90EF90DF90CF900895EF92FF920F931F938091FF0B82FD02C080E040
:207560003FC0E091CC01F091CD01E780F084018512858CE396E060E070E00E94FC29C80182
:20758000B7010E9439C6665F7F4F6D52714018F48BE596E002C086E496E00E94282AE09196
:2075A000CE01F091CF01E780F0840185128581E396E00E94A129C801B7010E9439C6665F86
:2075C0007F4F6D52714018F086E496E002C08BE596E00E94282A85E696E00E942D2A81E0AE
:2075E0001F910F91FF90EF900895EF92FF920F931F930E94E3C2AB01BC018AE296E00E94F6
:20760000EB29E0911C01F0E0EE0FFF1FE453FE4F008111813DE5E32E34E0F32EF80147811D
:20762000508561857285C70122E00E94FF2AF8014385548565857685C70120E00E94FF2AF1
:20764000F8018081E8E4F4E0E80FF11D6081C70170E00E94C4291F910F91FF90EF90089508
:20766000DF92EF92FF920F931F937B018C01D42E20E030E040EF52E40E94D8C718165CF4F4
:207680000F2EF0E0EF2EF0E0FF2EF0EF0F2FF2E41F2FF02D14C0C801B70120E030E040E0E0
:2076A00050E00E94CAC5882354F40F2EF0E0EF2EF0E0FF2EF0E00F2FF0E01F2FF02D609115
:2076C0009601709197018091980190919901A80197010E94CAC5882321F18BE891E0B80149
:2076E000A7010E949E39DD2079F0C801B70120E030E040EF51E40E94D8C718162CF480916E
:20770000CB0181608093CB014091960150919701609198017091990185E295E020E00E9459
:207720003B2B1F910F91FF90EF90DF9008952F923F924F925F926F927F928F929F92AF9270
:20774000BF92CF92DF92EF92FF920F931F93DF93CF93CDB7DEB7AE970FB6F894DEBF0FBEB3
:20776000CDBF9EA78DA74B8F5C8F6D8F7E8F2F8F08A30E94E3C26D8B7E8B8F8B988FADA5F2
:20778000BEA596968C9190E0959587959C01442737FD4095542F29873A874B875C8780E36A
:2077A00095E00E943A2AE091CC01F091CD011682158280E090E0A0E0B0E083879487A58761
:2077C000B687E081F0E0E85BFB4F1082E091CE01F091CF011682158283879487A587B687CE
:2077E000E081F0E0E85BFB4F10823F8D30931E01ADA5BEA5EC91F0E0E85BFB4F96968C91B3
:207800008083332321F48091890180938A012D893E894F89588D298B3A8B4B8B5C8B7901D7
:207820008A0149855A856B857C854D835E836F8378871A8E198E9924939460E070E080EA50
:2078400091E469837A838B839C835B016C018DA59EA50E942E38ADA5BEA51796BC91B9A748
:20786000EDA5FEA5F085FAA7ADA5BEA51996BC91BBA7EDA5FEA5F285FCA70E94E3C21B01F8
:207880002C0169817A818B819C8129A53AA54BA55CA50E94CAC5882344F489A59AA5ABA53E
:2078A000BCA589839A83AB83BC83C601B50129A53AA54BA55CA50E94CAC587FD06C089A50D
:2078C0009AA5ABA5BCA55C016D01992009F441C069A57AA58BA59CA52B8D3C8D4D8D5E8D52
:2078E0000E94D8C718160CF096C1A20191012E193F09400B510B6F8D662329F484EC99E0D0
:20790000A0E0B0E004C08CED95E0A0E0B0E082179307A407B50708F07EC1ADA5BEA5EC9192
:207920006E2F70E0685B7B4F8985BD818B1BFB0180832D873E874F87588B298A3A8A4B8A5E
:207940005C8A2B8D3C8D4D8D5E8D29833A834B835C8369A57AA58BA59CA52B8D3C8D4D8DEC
:207960005E8D0E94CAC588230CF054C1A201910169897A898B899C89261B370B480B590B92
:207980007F8D772329F088EB9BE0A0E0B0E004C088E893E1A0E0B0E082179307A407B507D8
:2079A00008F038C1898D9A8D892B09F418C16D847E848F849888620E731E841E951E6D85A1
:2079C0007E858F859889621B730B840B950B2D813E814F8158850E9450C9A40193010E9495
:2079E000C5C969857A858B859C85260F371F481F591F24313105410551054CF484E190E035
:207A0000A0E0B0E089879A87AB87BC8718C0ADA5BEA596968C9190E044977C010027F7FCF8
:207A20000095102F29873A874B875C87E216F3060407150724F4E986FA860B871C87EDA566
:207A4000FEA526A1822F869590E0A0E0B0E049855A856B857C8584179507A607B7072CF014
:207A60004D835E836F83788714C0822F90E001979C01442737FD4095542F69857A858B8546
:207A80009C85261B370B480B590B2D833E834F83588783E495E049855A856B857C850E944D
:207AA000EB298BE495E04D815E816F8178850E94EB2980E595E0B601A50122E00E94FF2A7A
:207AC00087E595E049815A816B817C8122E00E943B2B898D9A8D03970CF481C06D817E8128
:207AE0008F8198850E946CC620E030E040E850E40E947AC87B018C0169817A818B819C811E
:207B0000A60195010E9403C520ED3FE049E450E40E947AC89B01AC01C801B7010E94D1C54B
:207B20007B018C01C401B3010E946CC620E030E04AE754E40E94D1C55B016C018EE595E08D
:207B4000B801A70122E00E94FF2A84E695E0B601A50122E00E943B2BC801B7012AE939E9FB
:207B600049E15FE30E947AC83B014C01A40193010E9404C5A60195010E94D1C57B018C010A
:207B80006DA3FEA20FA318A7C401B301A60195010E947AC820E030E040E05EE30E947AC8D5
:207BA0005B016C0169A3BAA2CBA2DCA28AE695E00E94282A87E795E0B401A30122E00E94F0
:207BC0003B2B8DE795E0A701B80122E00E943B2B83E895E0A501B60122E00E943B2BADA552
:207BE000BEA5EC912E2F30E0285B3B4F8D81B9858B0FF9018083298D3A8D2F5F3F4F3A8FE6
:207C0000298F82017101AB8CBC8CCD8CDE8C9924939401C099246B8D7C8D8D8D9E8D20E0CD
:207C200030E040EA51E40E9404C59B01AC0169A57AA58BA59CA50E94D8C718161CF489E893
:207C400095E031C0D201C1014D895E896F89788D841B950BA60BB70B895E9340A040B04033
:207C600038F080E00E944F1B2D8A3E8A4F8A588E220C331C441C551C69897A898B899C89B6
:207C8000261A370A480A590A2E183F08400A510A71E827167FE4370672E1470670E05706F9
:207CA00050F182EB95E00E942D2AE091CC01F091CD011682158280E090E0A0E0B0E0838702
:207CC0009487A587B687E081F0E0E85BFB4F1082E091CE01F091CF011682158283879487EB
:207CE000A587B687E081F0E0E85BFB4F10828FEF80931E0156C0898D9A8D06970CF448C023
:207D00008FEC95E00E943A2AE091CC01F091CD011682158280E090E0A0E0B0E083879487AC
:207D2000A587B687E081F0E0E85BFB4F1082E091CE01F091CF011682158283879487A58779
:207D4000B687E081F0E0E85BFB4F10828FEF80931E0198A1992329F12DA13EA14FA158A53D
:207D6000C901DA01EDA5FEA5868F978FA0A3B1A329A13AA14BA15CA1C901DA0182A393A3C9
:207D8000A4A3B5A381E0838B80E00E94EC2E09C08EE89FE00E94B5998EE89FE00E9428C08C
:207DA00056CDAE960FB6F894DEBF0FBECDBFCF91DF911F910F91FF90EF90DF90CF90BF90CA
:207DC000AF909F908F907F906F905F904F903F902F900895E0917502F091760260E08685E3
:207DE000882309F461E085850E9497C408959F92AF92BF92CF92DF92EF92FF920F931F93FB
:207E0000CF93DF937B018C01942EA22EE091CC01F091CD01638574858585968520E030E050
:207E200040E751E40E94D8C7181614F4BB2402C0BB24B394C801B70120E030E849E853E4A7
:207E40000E94D8C718165CF40F2EF0E0EF2EF0E8FF2EF9E80F2FF3E41F2FF02D14C0C80136
:207E6000B70120E030E040E050E00E94CAC5882354F40F2EF0E0EF2EF0E0FF2EF0E00F2F91
:207E8000F0E01F2FF02DC92CDD24F601EE0FFF1FE453FE4FC081D181CE01B801A7010E94B6
:207EA0009E39AA2081F0C801B70120E030E040EF51E40E94D8C7181634F4FE01E05CFF4F9B
:207EC000808181608083C801B70120E030E040EA50E40E94D8C788237CF08CE690E0C89E2E
:207EE000F001C99EF00DD89EF00D1124E15EFE4FE659FF4F81918083692D70E080E090E0A1
:207F00000E946AC6AB01BC018AE195E020E00E94FF2A89EE93E0B801A70120E00E943B2B28
:207F2000E091CC01F091CD01638574858585968520E030E040E751E40E94D8C718162CF0B7
:207F4000BB2079F40E94482E0CC0BB2051F00E94E3C26093840C7093850C8093860C9093B3
:207F6000870CDF91CF911F910F91FF90EF90DF90CF90BF90AF909F9008952F923F924F92A5
:207F80005F926F927F928F929F92AF92BF92CF92DF92EF92FF920F931F93DF93CF9300D01E
:207FA00000D0CDB7DEB78091C70B9091C80BA091C90BB091CA0BE0917502F0917602838FF3
:207FC000948FA58FB68FEFE1CE2EE1E0DE2ED0927602C09275028093EF0B9093F00BA0936B
:207FE000F10BB093F20BE0902801F090290100912A0110912B01E092E701F092E801009321
:20800000E9011093EA0160E070E080E89FE3A80197010E94D1C56093940B7093950B8093AD
:20802000960B9093970B80912E0190912F01A0913001B09131018093F7019093F801A0931A
:20804000F901B093FA0160913201709133018091340190913501609323027093240280939E
:2080600025029093260260931302709314028093150290931602A80197010E947AC80E9441
:208080003EC66093A40B7093A50B8093A60B9093A70B6093B40B7093B50B8093B60B909382
:2080A000B70BC60185960E94D737A090CB0BB090CC0BC090CD0BD090CE0B6090CF0B709024
:2080C000D00B8090D10B9090D20B2090D30B3090D40B4090D50B5090D60B80916A0C909196
:2080E0006B0CA0916C0CB0916D0C89839A83AB83BC830091750210917602D80111966D9171
:208100007D918D919C91149790958095709561957F4F8F4F9F4F0E946CC62091880B3091B3
:20812000890B40918A0B50918B0B0E947AC860937A0C70937B0C80937C0C90937D0CF801A7
:20814000658176818781908590958095709561957F4F8F4F9F4F0E946CC620918C0B309179
:208160008D0B40918E0B50918F0B0E947AC860937E0C70937F0C8093800C9093810C809133
:20818000000C80FF26C000D000D08091FB019091FC01A091FD01B091FE01EDB7FEB78183D7
:2081A0009283A383B483C601B501A4019301820171010F2EF0E8AF2EFFE4BF2EF3ECCF2E04
:2081C000F7E4DF2EF02D0E94BA720F900F900F900F9089819A81AB81BC8180936A0C909316
:2081E0006B0CA0936C0CB0936D0C80E00E94986A0F900F900F900F90CF91DF911F910F9101
:20820000FF90EF90DF90CF90BF90AF909F908F907F906F905F904F903F902F9008958FE12F
:2082200091E09093760280937502209A219A80912C0161E00E941AC480912D01882329F42D
:2082400080912C0161E00E9497C40E94E3C260935301709354018093550190935601549AEB
:208260005C980E941E380E94E94C08952F923F924F925F926F927F928F929F92AF92BF9244
:20828000CF92DF92EF92FF920F931F93DF93CF93CDB7DEB72B970FB6F894DEBF0FBECDBFB0
:2082A0000CEC11E01C830B8389E891E09A8389831F821E8292E39D8380911E01AE81A817A9
:2082C00009F452C2EB81FC8180809180C4010E942E38FE81FF2329F5D40117966D917D9179
:2082E0008D919C911A9720E030E040EA50E40E94CAC5882394F4F4016385748585859685B5
:2083000020E030E040EA50E40E94CAC588232CF4A981BA8111961C9204C0E981FA8180818F
:208320008183D090FF0BD2FC2DC0D4011796ED90FD900D911C911A97C801B70120E030E0FB
:2083400040E251EC0E94CAC587FD0AC0C801B70120E030E041E953E40E94D8C7181694F456
:20836000809177028F5F809377028B3018F4B1E0BF8308C0E4E0DE2AD092FF0B0E94A73ADC
:20838000F1E0FF838091FF0B82FDEEC12224D40113962D913C91149715968D919C911697A4
:2083A000281739071CF4222423940FC08401005C1F4FF801808180FF08C08D8163E00E94DF
:2083C000D396D8018C918E7F8C93F40187A5E82FF0E03C96EE0FFF1FEE0FFF1FE80DF91DF7
:2083E000D4011796AD90BD90CD90DC901A97A082B182C282D382382E3394B3E03B22F401F7
:2084000037A68389813009F0DAC0E384F48405851685C801B70120E030E040EA51E40E9499
:20842000CAC587FDC4C0C801B701A60195010E9403C52B013C0120E030E040EA51E40E9403
:20844000D8C7181624F4D40196966C91B1C0C301B20120E030E040EA51EC0E94CAC587FD25
:20846000A6C0D4015A96ED90FD900D911C915D97E886F9860A871B87C301B20154962D9149
:208480003D914D915C9157970E9404C57B018C01F401A3A4B4A4C5A4D6A4A60195010E948B
:2084A000CAC587FD11C0D4019796AD90BD90CD90DC909A97C801B701A60195010E94D8C753
:2084C000181614F057016801F401A48AB58AC68AD78A688579858A859B85A30192010E94A3
:2084E0007AC87B018C01C601B501D4015E962D913D914D915C9191970E947AC82DEC3CEC47
:208500004CEC5DE30E947AC89B01AC01C801B7010E9404C57B018C01F40186A1C82EDD24AE
:20852000E7A5F0E03C96EE0FFF1FEE0FFF1FE80DF91D6081718182819381D40117962D91A2
:208540003D914D915C911A970E9403C5F40122A133A144A155A10E947AC82FED3FE445E5B3
:2085600050E40E947AC89B01AC01C801B7010E9404C57B018C01B601882777FD8095982FEF
:208580000E946CC69B01AC01C801B7010E947AC829E23FEF4FE75BE30E947AC80E9439C627
:2085A00077FD05C0C616D7061CF4B60101C060E0D401EC91F0E0E85BFB4F6083B5C0833047
:2085C00009F07DC0F4014384548465847684C301B20120E030E040EA51E40E94CAC587FD53
:2085E0006AC0C301B201A60195010E9403C57B018C0120E030E040EA51E40E94D8C718164C
:2086000024F4D40196968C9157C0C801B70120E030E040EA51EC0E94CAC587FD4CC0F4015F
:20862000648975898689978920E030E040E450E40E947AC87B018C01E32DF0E03C96EE0F1C
:20864000FF1FEE0FFF1FE80DF91DC601B50120813181428153810E9403C52FED3FE445E59C
:2086600050E40E947AC89B01AC01C801B7010E9404C520E030E040E85EE30E947AC8D4017B
:2086800054966D937D938D939C9357975A962D913D914D915C915D970E947AC8A601950147
:2086A0000E9404C5A30192010E94D8C718161CF0F401808D01C080E0D401EC9131C0823085
:2086C00041F50E94E3C29B01AC01F40187859089A189B28979018A01E81AF90A0A0B1B0B10
:2086E000D801C70189589341A040B040E8F0E081222011F480E001C08FEFF0E0E85BFB4FD8
:208700008083D4011F962D933D934D935C9352970BC0D401EC91222011F480E001C08FEF81
:20872000F0E0E85BFB4F8083F401678170858185928520E030E849E853E40E94D8C71816FB
:2087400034F4D401EC91F0E0E85BFB4F1082809175029091760285968816990629F42220D8
:2087600011F0149A01C01498BE81BF5FBE83ED81EE5CED830B811C810E5F1F4F1C830B83E6
:2087800089819A8184599F4F9A838983B23009F093CD9F81992339F480917702882319F03E
:2087A0008150809377028091FF0B82FF17C0E091CC01F091CD01E081F0E0E85BFB4F10820C
:2087C000E091CE01F091CF01E081F0E0E85BFB4F1082809127028860809327022B960FB6D4
:2087E000F894DEBF0FBECDBFCF91DF911F910F91FF90EF90DF90CF90BF90AF909F908F901F
:208800007F906F905F904F903F902F900895FC018081918180FD02C024E001C026E083FDB7
:208820002C5F84FD2C5F85FD2C5F86FD2C5F90FD2C5F91FD2F5F92FD2C5F93FD2C5FAC0170
:208840004270507094FF19C02E5F3281452B09F02E5F82FD2E5F30FD2C5F31FD2C5F32FD58
:208860002C5F97FF11C0848190E001968135910514F080E590E0280F07C0452B09F02F5FE0
:2088800082FD2F5F97FD205F822F08958091E30290E00196817090708093E302809152031E
:2088A0008F5F80935203089580915203882319F420E030E008C09091E20285E3989F90019A
:2088C000112428583D4FC9010895CF93DF93EC01888181FF12C083E294E06DE40E94624E58
:2088E0006E817F81882777FD8095982F0E94832983E294E060E20E94624E888182FF12C073
:2089000083E294E067E40E94624E68857985882777FD8095982F0E94832983E294E060E28E
:208920000E94624E8881998191FF12C083E294E064E50E94624E6E8D70E0882777FD809569
:20894000982F0E94832983E294E060E20E94624E888183FF09C04A855B856C857D8583E03C
:2089600093E022E00E94FF2A888184FF09C04E855F856889798986E093E022E00E94FF2A12
:20898000888185FF09C04A895B896C897D8989E093E022E00E94FF2A888186FF09C04E89F8
:2089A0005F89688D798D8CE093E024E00E94FF2A8881998190FF09C04A8D5B8D6C8D7D8DE9
:2089C0008FE093E022E00E94FF2A8881998192FF08C04F8D58A169A17AA182E193E00E94FA
:2089E000EB298881998193FF08C04BA15CA16DA17EA185E193E00E94EB298A8180FF09C0EE
:208A00004FA158A569A57AA588E193E022E00E94FF2A8A8181FF09C04BA55CA56DA57EA519
:208A20008BE193E022E00E94FF2A8A8182FF09C04FA558A969A97AA98EE193E022E00E9485
:208A4000FF2A8881998197FF04C08BA99CA90E9424290E945D1ADF91CF9108950F931F932E
:208A6000CF93DF93EC018B01709148037250F80140E050E020E030E01FC0672F763108F02E
:208A800065E1DF01962F8D91480F511D4F3F510510F04F5F5040240F351F2F3F310510F0BB
:208AA0002F5F3040915079F76150862F90E06F5F0196E80FF91F761B7723F9F68181281BBE
:208AC00031098081481B5109242B352B232B51F08091270282FF04C083EC92E00E942D2A07
:208AE00080E0CDC0F801219131913983288334FF0CC0D80112968D919C9113979B838A8315
:208B0000329637FF04C0419103C01B821A8240E1888180FF0EC0819191919D838C83A0E06B
:208B2000B0E080934E0390934F03A0935003B0935103888199819C012270307094FF0EC05C
:208B4000232B21F0819191919F838E83888182FF10C081919191998788870BC0232B19F070
:208B600081918E831F82888182FF03C0819188871986888183FF08C081919191A191B19129
:208B80008A879B87AC87BD87888184FF08C081919191A191B1918E879F87A88BB98B888174
:208BA00085FF08C081919191A191B1918A8B9B8BAC8BBD8B888186FF08C081919191A1914B
:208BC000B1918E8B9F8BA88FB98F8881998190FF08C081919191A191B1918A8F9B8FAC8FF1
:208BE000BD8F8881998191FF02C081918E8F8881998192FF08C081919191A191B1918F8F43
:208C000098A3A9A3BAA38881998193FF08C081919191A191B1918BA39CA3ADA3BEA38A8122
:208C200080FF08C081919191A191B1918FA398A7A9A7BAA78A8181FF08C081919191A1916A
:208C4000B1918BA79CA7ADA7BEA78A8182FF08C081919191A191B1918FA798ABA9ABBAAB76
:208C60008881998197FF08C0FCABEBABE40FF11D108281E0809349031092570381E0DF9116
:208C8000CF911F910F910895EF92FF920F931F93DF93CF9300D0CDB7DEB77C018B01CB018F
:208CA000BE016F5F7F4F0E940315FC0189819A810817190751F4D70112968D919C91139784
:208CC000906813969C938E931297CF010F900F90CF91DF911F910F91FF90EF900895EF92A0
:208CE000FF920F931F93DF93CF9300D0CDB7DEB77C018B01CB01BE016F5F7F4F4AE050E048
:208D00000E9463169C0189819A810817190731F4F70182819381906893838283C9010F9087
:208D20000F90CF91DF911F910F91FF90EF900895EF92FF920F931F93CF93DF938C017B0186
:208D4000DC0111961C921E9213961C921E921297CB016EE470E00E94BE17BC010097B1F0A7
:208D60006F5F7F4FC8010E946F4660934E0370934F038093500390935103F80180819181B5
:208D8000816091838083CB0164839583C7016DE470E00E94BE17BC010097D1F06F5F7F4F7F
:208DA000C8010E946F46D80117967C936E9316978D919C9111979C01226011963C932E9307
:208DC0006F3F710529F020F0826090618D939C93F801808181FFC5C18681978187319105B7
:208DE00099F08C31910581F08D31910569F08E31910551F08032910539F08537910509F027
:208E0000B0C102C0319601C0F70180818D34D1F701C0319680818032E1F701C03196808179
:208E20008032E1F3D801D396EC93D397D496FC930DC0D80116968D919C91179785379105EB
:208E400011F0203231F02A3221F031962081222381F7108281E080934903F80180819181AE
:208E6000906834C16F5F7F4FC8010E946F46D80119967C936E9318978D919C9111979C0172
:208E8000246011963C932E936F3F710529F020F0846090618D939C93C70168E570E00E949F
:208EA000BE17BC01009779F06F5F7F4FC8010E944446F80162877387848795878081918179
:208EC000886091838083C70169E570E00E94BE17BC01009791F06F5F7F4FC8010E94444650
:208EE000D8011E966D937D938D939C9351978D919C91119780618D939C93C7016AE570E014
:208F00000E94BE17BC01009779F06F5F7F4FC8010E944446F801628B738B848B958B808178
:208F20009181806291838083C70165E470E00E94BE17BC01009791F06F5F7F4FC8010E9472
:208F40004446D80156966D937D938D939C9359978D919C91119780648D939C93C70166E43B
:208F600070E00E94BE17BC01009779F06F5F7F4FC8010E944446F801628F738F848F958FB9
:208F800080819181916091838083C70164E570E00E94BE17BC01009779F06F5F7F4FC801BC
:208FA0000E946F46D8015E966C935E978D919C91119792608D939C93C70163E570E00E9463
:208FC000BE17BC01009779F06F5F7F4FC8010E946F46F801678F70A381A392A380819181D5
:208FE000946091838083C70160E570E00E94BE17BC01009791F06F5F7F4FC8010E946F4601
:20900000D80193966D937D938D939C9396978D919C91119798608D939C93C70169E470E023
:209020000E94BE17BC010097A1F06F5F7F4FC8010E944446F80167A370A781A792A78281C5
:20904000938181609383828380819181906191838083C7016AE470E00E94BE17BC010097B4
:20906000D9F06F5F7F4FC8010E944446D8019B966D937D938D939C939E9712968D919C9105
:209080001397826013969C938E9312978D919C91119790618D939C93C70162E570E00E946E
:2090A000BE17BC010097A1F06F5F7F4FC8010E944446F80167A770AB81AB92AB82819381C3
:2090C00084609383828380819181906191838083C7016AE270E00E94BE17EC010097D9F04E
:2090E000BC016F5F7F4FC8010E946F4690E004C0D7018D917D019827EC16FD06C9F796171E
:2091000051F08091270282FF04C083EC92E00E942D2A90E01EC0F8018281938197FD06C0FD
:209120008081918186709270892B29F5809157038F5F809357038091270282FF04C083EE9C
:2091400092E00E942D2A90E080915703833008F091E0892FDF91CF911F910F91FF90EF90C7
:209160000895C70167E470E00E94BE17BC01009709F078CE91CE10925703EACFCF93DF93FD
:20918000EC018091270280FF07C089EB92E00E94A129CE010E946544DF91CF9108959C01EC
:2091A00080915203882389F0C9010E94BE488091E2028F5F8093E202823011F41092E2029C
:2091C00080915203815080935203089583E294E00E94544E1092440380914503882311F048
:2091E0008EE101C08EE08093D0010E945D1A40914A0350914B0360914C0370914D034F5F48
:209200005F4F6F4F7F4F81EB92E00E94B1298DE892E00E94282A0895CF92DF92EF92FF925E
:209220000F931F93CF93DF93EC01888181FF38C08E819F818E369105A9F480914E039091EF
:209240004F03A0915003B091510380934A0390934B03A0934C03B0934D038DE892E00E9434
:20926000282A8AC08037910511F40E9433198E819F818A599240A1F480914A0390914B03CC
:20928000A0914C03B0914D030196A11DB11D80934A0390934B03A0934C03B0934D036FC085
:2092A000888180FF57C000914A0310914B0320914C0330914D03680179010894C11CD11CE8
:2092C000E11CF11C40914E0350914F036091500370915103D701C60184279527A627B727E5
:2092E000892B81F1C801841B950B889700F18091D00187FF19C08091270282FF12C08FE2F1
:2093000093E0B701A6010E94DA2940914E0350914F03609150037091510384E493E00E946B
:20932000B1290E94E6482BC081508093D001109244038AE493E00E94B1298DE892E00E9414
:20934000282A1DC040934A0350934B0360934C0370934D030E94464440914E0350914F0377
:2093600060915003709151038FEB92E00E94B12980914503809346038FEF8093D001DF9165
:20938000CF911F910F91FF90EF90DF90CF900895BF92CF92DF92EF92FF920F931F93CF93B9
:2093A000DF9380915203823008F02DC280914903882309F401C280915203882309F4FCC1A9
:2093C00022C28091D00187FF04C0809144038823B1F08091530390915403A0915503B09130
:2093E0005603A7019601281B390B4A0B5B0B293C31054105510518F00E94E6481FC0809194
:209400005203882309F0ACC08091530390915403A0915503B0915603A7019601281B390B1F
:209420004A0B5B0BDA01C901895E9340A040B04008F496C089EE96E00E94282AC092530367
:20944000D0925403E0925503F092560389C09091D00197FD0FC080914603882359F08091B1
:20946000E402882321F491509093D0014DC0B092D0014AC08091E402882309F445C08823F8
:20948000880F880B80238093450380914503882309F1113009F467C0812F8450823030F4E7
:2094A00084EE92E00E9407448093480380914803181709F04EC09091E30285E3989FE00165
:2094C0001124C858DD4FCE0164EE72E041E00E942E452BC0A12FB0E01197FD01EC51FD4FE8
:2094E000E081EE2351F0EA3041F0ED3031F080914703882319F5EA3309F5AC51BD4F1C924A
:2095000010924703113019F4109244032CC09091E30285E3989FE0011124C858DD4FCE0166
:2095200064EE72E041E00E949846882321F0CE010E940C4908C10E94E64805C1EB3311F4E2
:209540000093470380914703882319F011501093440380914403803631F40E94E64853C1BD
:2095600001E09EE1B92E83E294E00E94084E181619060CF030C110914403103608F02BC187
:20958000C0925303D0925403E0925503F092560383E294E00E94354EE12FF0E0EC51FD4F5E
:2095A00080831F5F10934403113009F06ECF4FCF80914403882309F4D5C025C10E94E3C2E9
:2095C0006093530370935403809355039093560382E39DE00E94838EEC014FEF8F3F9407D8
:2095E00061F581E293E00E94282A8EE89FE069E174E141E00E94BB984091530D5091540D2E
:209600006091550D7091560D82E39DE00E94028782E39DE00E94838EEC015FEF8F3F95074C
:2096200029F48FEF93E10E942D2AB6C08EE89FE060EF73E141E00E94BB982091530D30912C
:20964000540D4091550D5091560D2F5F3F4F4F4F5F4F2093530D3093540D4093550D50937B
:20966000560D80914403E82FF0E0EC51FD4FC083182F1F5F10934403113041F4109245036D
:209680008091E40287FF02C01093450380914503882301F1123008F465C0812F8450823011
:2096A00030F484EE92E00E9407448093480380914803181709F056C08091E30225E3829F9E
:2096C000C001112488589D4F64EE72E040E00E942E4535C0C12FD0E0BE0161507040FB013E
:2096E000EC51FD4FE081EA3071F0ED3009F079C00AC080914703882311F4EA3321F01F355F
:2097000008F07DC023C06C517D4FFB01108203C0CC51DD4F188210924703113019F4109298
:20972000440320C08091E30225E3829FC001112488589D4F64EE72E040E00E949846882332
:2097400011F00E944644109244035DC0EB3319F481E08093470380914703882319F011507D
:209760001093440320914F0D3091500D4091510D5091520D8091530D9091540DA091550DDF
:20978000B091560D82179307A407B50728F480914403803608F412CF10925B0D80EF92E099
:2097A0000E94282A10924403109247038091010C8D7F8093010C27C0109249030E94E3C27A
:2097C0006B017C0183E294E00E94084E181619060CF4C6CEF6CD80915B0D882309F0E8CE58
:2097E00012C080914F0D9091500DA091510DB091520D82179307A407B50709F07ACFEA3384
:2098000009F086CF80CFDF91CF911F910F91FF90EF90DF90CF90BF9008954F925F92AF92B0
:20982000BF92CF92DF92EF92FF920F9320E28030920708F079C022E08030920708F04AC088
:209840008A30910510F48AE090E0A12C24E2B22E24EFC22ED12CEE24FF18DD20A1F4CC2080
:2098600009F012C001E1AA1CBB1C0A9509F431C0EE1CFF1CE81AF90A20F4E80EF91E8894AA
:20988000F2CF0894F0CF12C009E1AA1CBB1CCC1C0A9509F41EC0EE1CFF1CE81AF90A20F4B3
:2098A000E80EF91E8894F1CF0894EFCF01E2AA1CBB1CCC1CDD1C0A9509F40BC0EE1CFF1C78
:2098C000E81AF90A20F4E80EF91E8894F0CF0894EECF51C0EDE3F4E1282F2F71969587953A
:2098E0009695879596958795969587958E7FE80FF91FA590B59025010590401805905008FD
:20990000249DC001259D900DE12D880F991FEE1F880F991FEE1F880F991FEE1FA91ABE0AB9
:20992000CC24DD24112427C0EFE3F6E19C013F709695969596959E7FE90FF11DA590B59007
:2099400025010590401805905008249DC001359DE02D259D900DE11D349D900DE11D907FCE
:209960009295E2958E2F807F982BEF70A91ABE0ACC24DD241124B501C6010F91FF90EF908F
:20998000DF90CF90BF90AF905F904F90089514BC80E488BDEEE6F0E0808184608083109259
:2099A000800010928200EFE6F0E0108289E0809381008CED9FEF9093890080938800808180
:2099C000826080830895E0915803F09159030995089580E480937C00109265021092690218
:2099E000109268021092700210926F021092660210926B0210926A021092720210927102E2
:209A00001092670210926D0210926C02109274021092730287EC80937A0080917A0086FDDD
:209A2000FCCF8091780090917900E0916E02F0E0E158F14FE49180917C00E770807EE82BA4
:209A4000E0937C0080917A00806480937A0008951F920F920FB60F920BB60F9211242F936D
:209A60008F939F93EF93FF932091C6009091DF039F5F9F778091E003981741F0E091DF03C9
:209A8000F0E0E15AFC4F20839093DF03FF91EF919F918F912F910F900BBE0F900FBE0F9035
:209AA0001F9018951F920F920FB60F920BB60F9211248F939F93EF93FF939091210480913C
:209AC0002204981731F48091C1008F7D8093C1000EC0E0912204F0E0EF51FC4F90818091F8
:209AE00022048F5F8F73809322049093C600FF91EF919F918F910F900BBE0F900FBE0F905B
:209B00001F901895AF92BF92DF92EF92FF920F931F93CF93DF93EC017A018B01DD24403047
:209B200081EE580780E0680780E0780711F0DD24D394E1E0AE2EB12CEC85FD85DD2069F07D
:209B4000C5010E8802C0880F991F0A94E2F7808360E079E08DE390E005C0108260E874E8AA
:209B60008EE190E0A80197010E94A3C92150304040405040569547953795279580E12030C6
:209B8000380720F0DD2011F0DD24D6CFE885F9853083EA85FB852083EE85FF85408121E0E9
:209BA00030E0C9010A8802C0880F991F0A94E2F7482B4083EE85FF854081C9010B8802C0A4
:209BC000880F991F0A94E2F7482B4083EE85FF854081C9010C8802C0880F991F0A94E2F7EB
:209BE000482B4083EE85FF8580810D8802C0220F331F0A94E2F7209528232083DF91CF9173
:209C00001F910F91FF90EF90DF90BF90AF900895DC011496ED91FC911597E058FF4F2191D6
:209C2000808130E020583F4F281B31092F773070C9010895DC011496ED91FC911597E0586D
:209C4000FF4F9081E058F040DF01AF57BF4F8C91981719F42FEF3FEF06C08C91E80FF11D3C
:209C60008081282F30E0C9010895DC011496ED91FC911597E058FF4F9081E058F040DF01F8
:209C8000AF57BF4F8C91981719F42FEF3FEF0AC08C91E80FF11D90818C918F5F8F778C935E
:209CA000292F30E0C9010895FC0186819781DC01A05CBF4FFC01EF5BFF4F9C918081981760
:209CC000E1F70895CF93DF93EC01EE81FF81E05CFF4F9081E054F0409F5F9F73DF01AF5B66
:209CE000BF4F8C919817E9F3E05CFF4F8081E054F040E80FF11D6083EE81FF81E05CFF4F5E
:209D00009083EE85FF85208181E090E00D8802C0880F991F0A94E2F7282B208381E090E0E3
:209D2000DF91CF910895109226041092250485E592E090932404809323048FE593E09093B4
:209D400028048093270481EE93E090932A048093290485EC90E090932C0480932B0484EC40
:209D600090E090932E0480932D0480EC90E09093300480932F0481EC90E090933204809318
:209D8000310486EC90E0909334048093330484E08093350483E08093360487E080933704F2
:209DA00085E08093380481E08093390408951F920F920FB60F920BB60F9211242F933F93BE
:209DC0004F935F936F937F938F939F93AF93BF93CF93DF93EF93FF9388B5805C88BD90914C
:209DE0003E04992369F4809148048C7F80933A0481115D9A8091490480933B0481115C9A8E
:209E000070913F04772331F480914B0480933D0481112C9A80913A04891719F49C3F09F063
:209E20005D9880913D04871719F47F3F09F02C9880913B04891719F49C3F09F05C987894E4
:209E40008091620290916302019690936302809362028658914038F010926302109262028D
:209E600081E08093640280917A0086FD43C060916E02862F90E04091780050917900DC01F1
:209E8000AA0FBB1FED01C859DD4F28813981420F531F59834883FC01EB59FD4F80818F5FAB
:209EA0008083803210F183E0569547958A95E1F7A159BD4F11965C934E9319821882108287
:209EC000862F8F5F80936E02833010F010926E02E0916E02F0E0E158F14FE49180917C006B
:209EE000E770807EE82BE0937C0080917A00806480937A0072FF04C08EE89FE00E94B799F3
:209F000080913F048F5F80933F0480913E048C5F80933E04FF91EF91DF91CF91BF91AF91A6
:209F20009F918F917F916F915F914F913F912F910F900BBE0F900FBE0F901F9018951F92E1
:209F40000F920FB60F920BB60F9211242F933F934F935F936F937F938F939F93AF93BF93FF
:209F6000EF93FF9380915A03882309F07DC080E070915D03772381F470915C03772319F4A7
:209F800060915B0391F0709389006093880010925B0310925C0308C060915C036058704069
:209FA00060935C0370935D0381E0882309F05CC081E080935A0388E49EEE90938900809343
:209FC00088008091810B882309F42FC00E94DD51F8948823E1F47F3FD1F010925B031092C8
:209FE0005C0310925D03809184009091850024E6820F911D6817790728F4909389008093A2
:20A00000880012C070938900609388000DC07058804060935B0370935C0380935D0390E8EC
:20A0200090938900109288001DC080914C0490914D04892B49F080914C0490914D04019742
:20A0400090934D0480934C0410925B0310925C0310925D0310925E038CED9FEF9093890070
:20A060008093880010925A03FF91EF91BF91AF919F918F917F916F915F914F913F912F91E6
:20A080000F900BBE0F900FBE0F901F901895FF920F931F93FFB6F89484E090E00E94011440
:20A0A0008C010E94AB142DB73EB7FFBE201B310BC9011F910F91FF9008951F9384B7182F2B
:20A0C00010FF04C08BE593E00E943A2A11FF04C083E693E00E943A2A12FF04C082E793E05D
:20A0E0000E943A2A13FF04C082E893E00E943A2A15FF04C081E993E00E943A2A14BE1F9164
:20A1000008952F923F924F925F926F927F928F929F92AF92BF92CF92DF92EF92FF920F93C2
:20A120001F93CF93DF93EC01888180FDE2C0898180FDDFC029C02E5F3F4FC901A0E0B0E080
:20A14000841B950BA60BB70BB595A79597958795BC018816990608F4C401881A990AF2018C
:20A1600091828082FE01E15AFF4F408151819B014617570708F49A01421B530B518340836F
:20A18000888181608883B5C0ED96E880F9800A811B81ED97FE01E35BFF4FC801B701208199
:20A1A0003181428153810E947AC83B014C014BE6242E312C2C0E3D1EC759DF4F4880598085
:20A1C000B20180E090E00E946AC65B016C01A097C801B701288139814A815B810E947AC8BB
:20A1E0009B01AC01C601B5010E947AC80E943EC67B018C01F10171836083A496C601B50186
:20A20000A40193010E947AC80E943EC63B014C0179836883CD56D040C201889F5001999F65
:20A220006001899F8827B00CC11CD81EB00CC11CD81E11249701229FC001339FD001239F14
:20A240002227900DA11DB21F900DA11DB21F11243DE5432E512C4C0E5D1EA6019501281BC3
:20A26000390B4A0B5B0BCA01B901CF59DF4FE880F9800A811B81EE0CFF1C001F111FA801EF
:20A2800097010E94A3C949010894811C911CF201918280829301229FC001339FD001239F65
:20A2A0002227900DA11DB21F900DA11DB21F1124A81AB90ACA0ADB0AC601B501A8019701CC
:20A2C0000E94A3C92F5F3F4F3A932A93280D391D6096488159816A817B81CF56D040C901C0
:20A2E000A0E0B0E084179507A607B7070CF023CF47CFDF91CF911F910F91FF90EF90DF900B
:20A30000CF90BF90AF909F908F907F906F905F904F903F902F900895FF920F931F93282FBF
:20A32000162F8091810B882309F042C080914C0490914D04892BE1F52223D1F134E0A3E793
:20A34000B0E0FF24F39407E048EA51E660E070E031502091800B822F90E08A9FF0018B9FC1
:20A36000F00D9A9FF00D1124E25BFB4FF18200831086832F810F828343835483658376839D
:20A380002F5F2093800B203110F01092800B8091010C80618093010C9FB7F8948091810BD5
:20A3A0008F5F8093810B9FBF332391F681E001C080E01F910F91FF900895BF92CF92DF92B4
:20A3C000EF92FF920F931F93CF93DF9380917E0B90917F0B892B09F048C18091820B482F33
:20A3E00050E083E790E0489FE001499FD00D589FD00D1124C25BDB4FD0937F0BC0937E0BAD
:20A40000898187FD3FC078948FEF9FEF9093DA018093D9018091270285FF21C08091820B6F
:20A420008F5F8093820B803110F01092820B10927F0B10927E0BF8948091810B815080934A
:20A44000810B8091810B882329F48091010C8F7E8093010C28EE33E040E050E0B5C383E765
:20A4600090E0489FF001499FF00D589FF00D1124E25BFB4F818180FF30C09091810B8281DE
:20A48000891748F010927F0B10927E0B20ED37E040E050E099C323813481458156818091B6
:20A4A000820B8F5F8093820B803110F01092820B10927F0B10927E0BF8948091810B815050
:20A4C0008093810B8091810B882309F07DC38091010C8F7E8093010C77C36085262F64FD3C
:20A4E0005E9825FD5E9826FD159867FD5E9883E790E0489FF001499FF00D589FF00D112464
:20A50000E25BFB4F808186608083789483E790E0489F9001499F300D589F300D1124F901E4
:20A52000E25BFB4F8781843079F4E281F0E0EE0FFF1FEE0FFF1FE20FF31FE25BFB4F818572
:20A540009285A385B48512C0E281F0E0EE0FFF1FEE0FFF1FE20FF31FE25BFB4F81859285A1
:20A56000A385B485880F991FAA1FBB1F8093830B9093840BA093850BB093860B83E790E0C4
:20A58000489FF001499FF00D589FF00D1124E25BFB4F808180FD03C0CE010E948150E0915A
:20A5A0007E0BF0917F0BE559FF4F80819181EB56F0409093830C8093820C10922E0C109226
:20A5C0002F0C1092300C1092310C10922A0C10922B0C10922C0C10922D0CF8948085282F35
:20A5E00030E0C90181719070419711F4459A01C04598C90182729070829711F4479A01C0B7
:20A600004798C901847490708434910511F42A9801C02A9A287830702838310511F4289A62
:20A6200001C0289880918C0C97818823C1F0943009F0D6C210928C0C8091260C9091270C56
:20A64000A091280CB091290C9C01AD01220F331F441F551F280F391F4A1F5B1FB5C29430CD
:20A6600009F4BEC281E080938C0C7894E0917E0BF0917F0BD78086E0C82ECD2024E0D216B4
:20A6800019F083E08D198783F894CC20F1F0818184FF12C09085892F8171803121F432999E
:20A6A00002C09F7E90879085892F8272803221F4339902C09F7D90879085892F84748034E2
:20A6C00021F4349902C09F7B908780912802E159FF4FE080F18002811381282F30E040E073
:20A6E00050E0E216F3060407150714F4A8019701B22E1E141F04100611060CF002C210E0B7
:20A70000A7C0112321F081E090E00E944AC3E0917E0BF0917F0B808587FF23C025A136A1FD
:20A7200047A150A585899689A789B08D281B390B4A0B5B0B25A336A347A350A757FF11C0B7
:20A74000299A8091830B9091840BA091850BB091860B280F391F4A1F5B1F25A336A347A357
:20A7600050A7808584FF23C0218D328D438D548D81859285A385B485281B390B4A0B5B0B99
:20A78000218F328F438F548F57FF11C05F9A8091830B9091840BA091850BB091860B280F5A
:20A7A000391F4A1F5B1F218F328F438F548F808585FF23C0258D368D478D50A1858596856D
:20A7C000A785B089281B390B4A0B5B0B258F368F478F50A357FF11C0469A8091830B9091C9
:20A7E000840BA091850BB091860B280F391F4A1F5B1F258F368F478F50A3808586FF23C016
:20A8000021A132A143A154A181899289A389B489281B390B4A0B5B0B21A332A343A354A384
:20A8200057FF11C02B9A8091830B9091840BA091850BB091860B280F391F4A1F5B1F21A314
:20A8400032A343A354A329985F9846982B981F5F1B1508F456CF85E0D82209F426C17894CF
:20A86000C0917E0BD0917F0BC35ADF4F88819981CD55D040A0E0B0E020912E0C30912F0C7C
:20A880004091300C5091310C82179307A407B50708F460C020912A0C30912B0C40912C0CEF
:20A8A00050912D0CCB59DF4F88819981AA81BB81BA01A901589F212D5A9F302D412D599F3C
:20A8C000200D311D4B1F689F200D311D4B1F699F300D411D789F300D411D6A9F400D799FE4
:20A8E000400D4695379527954695379527951124269688819981820F931F9093830C809329
:20A90000820CFE01329122912817390720F43093830C2093820C2091820C3091830C8EE20F
:20A92000213E380790F08DE5213C380740F084E080932802369527953695279509C082E0E1
:20A94000809328023695279503C081E080932802C90158C0FE01E159FF4FC15ADF4F888117
:20A960009981CF55D040A0E0B0E0208131814281538182179307A407B5077CF0898182FD00
:20A9800038C110922A0C10922B0C10922C0C10922D0C8981846089832CC1C759DF4F88811A
:20A9A0009981C956D0402EE2813E920708F04BC06BC0C359DF4FE881F9810AC0C359DF4F77
:20A9C00088819981E61BF70BE817F90708F4FC018EE2E13EF80790F02DE5E13CF20740F0F3
:20A9E00084E080932802F695E795F695E79509C082E080932802F695E79503C081E0809302
:20AA00002802CF010E940D4C9B01AC012093260C3093270C4093280C5093290C80912A0CB7
:20AA200090912B0CA0912C0CB0912D0C820F931FA41FB51F80932A0C90932B0CA0932C0CF3
:20AA4000B0932D0C32C0FE01E75AFF4F815C9D4578F084E08093280280819181A281B381C8
:20AA6000F2E0880F991FAA1FBB1FFA95D1F715C082E08093280280819181A281B381880F46
:20AA8000991FAA1FBB1F09C081E080932802C75ADF4F88819981AA81BB818093260C9093B3
:20AAA000270CA093280CB093290CCC2051F12B2D30E040E050E080912E0C90912F0CA091C6
:20AAC000300CB091310C820F931FA41FB51F80932E0C90932F0CA093300CB093310CE091D7
:20AAE0007E0BF0917F0BE159FF4F80819181A281B381821B930BA40BB50B80839183A283EA
:20AB0000B383E0917E0BF0917F0B87812091260C3091270C4091280C5091290C843039F023
:20AB200079018A0116950795F794E79402C079018A01CC2009F446C0E159FF4F8081918172
:20AB4000A281B381EF56F040181619061A061B061CF48085807FB1F58091820B8F5F809342
:20AB6000820B803110F01092820B10927F0B10927E0BF8948091810B81508093810B809167
:20AB8000810B882329F48091010C8F7E8093010C8091810B882339F48EE89FE061E676E10E
:20ABA00040E00E94BB98A801970155954795379527952093260C3093270C4093280C50932C
:20ABC000290C02C0A8019701B901CA01DF91CF911F910F91FF90EF90DF90CF90BF900895D0
:20ABE0002091260C3091270C4091280C5091290CEBCF20912A0C30912B0C40912C0C5091E0
:20AC00002D0CCB59DF4F88819981AA81BB81C556D040389F612D3A9F702D212D399F600D86
:20AC2000711D2B1F489F600D711D2B1F499F700D211D589F700D211D4A9F200D599F200D80
:20AC40002695779567952695779567951124E091820CF091830CE617F70708F4AACEAECE3F
:20AC6000CF93DF93C82FD0E004C00E94C8490E94B61B8091810B9E01280F311D2131310526
:20AC8000A4F7DF91CF9108952F923F924F925F926F927F928F929F92AF92BF92CF92DF9280
:20ACA000EF92FF920F931F93DF93CF93CDB7DEB7EF970FB6F894DEBF0FBECDBF4C017EABFE
:20ACC0006DAB58AF4FAB09AF1AAF2BAF3CAFEDAEDA01AD90BD90CD90DD90BCABABABC601C7
:20ACE000B501F40120813181428153810E9404C56BA37CA38DA39EA3AFA9B8AD1496ED90D2
:20AD0000FD900D911C911797C801B701F40124813581468157810E9404C56F8F78A389A38D
:20AD20009AA32091EF0B3091F00B4091F10B5091F20B2FA738AB49AB5AAB8091C70B90910E
:20AD4000C80BA091C90BB091CA0B8BA79CA7ADA7BEA72091940B3091950B4091960B5091D3
:20AD6000970B2FA338A749A75AA7D601C501B0588B8F9C8FAD8FBE8FA801970150582F8B79
:20AD8000388F498F5A8FADA9BEA96D917D918D919C912BA13CA14DA15EA10E9403C55B01BB
:20ADA0006C01EDA9FEA964817581868197812F8D38A149A15AA10E9403C53B014C016B8D8A
:20ADC0007C8D8D8D9E8DA40193010E947AC87B018C016F89788D898D9A8DA60195010E94E6
:20ADE0007AC89B01AC01C801B7010E9403C51B012C016B8D7C8D8D8D9E8DA60195010E946F
:20AE00007AC87B018C016F89788D898D9A8DA40193010E947AC89B01AC01C801B7010E9424
:20AE200004C59B01AC01C201B1010E9477C55B016C0120E030E040E050E00E94CAC58823A8
:20AE400054F4C601B5012BED3FE049EC50E40E9404C55B016C01FDADFF2351F0C601B501CF
:20AE60002BED3FE049EC50E40E9403C55B016C01C601B5019F7729AD3AAD4BAD5CAD0E940C
:20AE80007AC83B014C012FE632E143E85AE30E94CAC587FDE5C1E0906A0CF0906B0C00918E
:20AEA0006C0C10916D0CC801B70120E030E040E752E40E94D8C71816F4F4C801B7012DE825
:20AEC0003AE748E85CE30E947AC80E9439C69B016430710514F023E030E0B901882777FDC3
:20AEE0008095982F0E946CC69B01AC01C401B3010E94D1C502C0C401B3010E94A7C60E94BC
:20AF00003EC67E8B6D8B2D893E89232B21F441E050E05E8B4D8BAD89BE89BD0180E090E02F
:20AF20000E946AC67B018C01C601B501A80197010E94D1C5698B7A8B8B8B9C8B2FA538A955
:20AF400049A95AA98BA59CA5ADA5BEA5281B390B4A0B5B0B2FA738AB49AB5AABCA01B9015D
:20AF60000E946CC62FA138A549A55AA50E947AC8A80197010E94D1C56D877E878F87988BD4
:20AF800069897A898B899C8920E030E040E05FEB0E947AC829893A894B895C890E947AC813
:20AFA00020E030E040E85FE30E9404C569877A878B879C876BA57CA58DA59EA50E946CC60C
:20AFC0002FA138A549A55AA50E947AC869837A838B839C83A1E0B0E0BFAFAEAF99240DC176
:20AFE000892D992787FD909583709070892B41F40E94C8490E94B61B8EE89FE00E94B5994B
:20B00000B8E1B9150CF446C06B8D7C8D8D8D9E8D29893A894B895C890E947AC87B018C0162
:20B020006F89788D898D9A8D29853A854B855C850E947AC89B01AC01C801B7010E9404C59F
:20B040007B018C016B8D7C8D8D8D9E8D29853A854B855C850E947AC85B016C016F89788DD9
:20B06000898D9A8D29893A894B895C890E947AC89B01AC01C601B5010E9403C56B8F7C8F4C
:20B080008D8F9E8F9394C701D8018F8B988FA98FBA8F61C0EEADFFADBF0180E090E00E9443
:20B0A0006AC629893A894B895C890E947AC87B018C01C8010E94CEC56D837E838F83988725
:20B0C000B701C8010E94DDC83B014C01AFA9B8ADED90FD900D911C9117FB109517F91095A1
:20B0E000EBA9FCA92080318042805380C801B7012D813E814F8158850E947AC85B016C01E9
:20B10000C201B101A40193010E947AC89B01AC01C601B5010E9404C56B8F7C8F8D8F9E8F1E
:20B12000C801B701A40193010E947AC87B018C01C201B1012D813E814F8158850E947AC8F5
:20B140009B01AC01C801B7010E9403C56F8B788F898F9A8F992469817A818B819C812D85FC
:20B160003E854F8558890E9404C569837A838B839C8300D000D0CDB6DEB60894C11CD11CB9
:20B180006BA17CA18DA19EA12B8D3C8D4D8D5E8D0E9404C57B018C016F8D78A189A19AA1E5
:20B1A0002F89388D498D5A8D0E9404C59B01AC0180E89FE4A3ECB7E4F60180839183A28359
:20B1C000B383C801B7010F2EF0E8EF2EFFE4FF2EF3EC0F2FF7E41F2FF02DA980BA80CB8065
:20B1E000DC800E94BA722EAD3FAD2F5F3F4F3FAF2EAF0F900F900F900F904EAD5FAD8D89DE
:20B200009E894817590708F4EBCE00D000D0ADA9BEA96D917D918D919C91139714962D91CD
:20B220003D914D915C9117971C96AD90BD90CD90DC901F970F2EF0E8EF2EFFE4FF2EF3ECEB
:20B240000F2FF7E41F2FF02DEDB7FEB7E182F282038314830E94BA720F900F900F900F90D3
:20B26000EF960FB6F894DEBF0FBECDBFCF91DF911F910F91FF90EF90DF90CF90BF90AF9078
:20B280009F908F907F906F905F904F903F902F9008952F923F924F925F926F927F928F92C2
:20B2A0009F92AF92BF92CF92DF92EF92FF920F931F93DF93CF93CDB7DEB761970FB6F8945D
:20B2C000DEBF0FBECDBF3090800B232D30E03F872E8783E790E0289FA001299F500D389F14
:20B2E000500D1124425B5B4F5C874B877FB7F8946091820B5091800B5D87651729F06F30FC
:20B3000011F460E001C06F5F20E030E040E050E003E710E018C0862F90E0809FF001819FF2
:20B32000F00D909FF00D1124E25BFB4F83819481A581B6816F3011F460E001C06F5F280F08
:20B34000391F4A1F5B1F283C8FEA380780E0480780E0580730F49D856917E9F602C03A94F3
:20B3600002C023E730E0361699F0832D90E0829FF001839FF00D929FF00D1124E25BFB4FE1
:20B38000808181FD05C0332051F70FE0302EEBCFAD853A16B1F0232D30E083E790E0289FA3
:20B3A000F001299FF00D389FF00D1124E25BFB4F808181FF06C0BFE03B1611F4332401C0F3
:20B3C0003394ED853E16F9F483E790E02E853F85289F8001299F100D389F100D1124025BEF
:20B3E0001B4FD80111968C911197806811968C9311977FBF8C9184608C938B859C850E9417
:20B400008150F801D5C5232D30E03A87298783E790E0289FF001299FF00D389FF00D112497
:20B42000E25BFB4F8181806881837FBF3D85332311F40FE002C00D850150402F50E0598B25
:20B44000488B83E790E0489FF001499FF00D589FF00D1124E25BFB4F2281AE85BF85A89F71
:20B46000F001A99FF00DB89FF00D1124223031F4E25BFB4F8281823031F431C0E25BFB4FBD
:20B480008281823061F503E710E028893989209FF001219FF00D309FF00D1124E25BFB4F5F
:20B4A0008081826080834E855F85409FF001419FF00D509FF00D1124E25BFB4F80818460B5
:20B4C00080838B859C850E94815089859A85809FF001819FF00D909FF00D112467C583E774
:20B4E00090E0AE85BF85A89F7001A99FF00CB89FF00C1124EEE4F4E0EE0EFF1E28893989AF
:20B50000289F8001299F100D389F100D11240E0F1F1FD70199966D917D918D919C919C97E9
:20B52000F80121A532A543A554A50E9403C55B016C01D7019D966D917D918D919C91D09798
:20B54000F80125A536A547A550A90E9403C57B018C01C601B501A60195010E947AC85B01FB
:20B560006C01C801B701A80197010E947AC89B01AC01C601B5010E9404C50E94E7C84B01EA
:20B580005C01C090720CD090730CE090740CF090750CA70196010E94D8C718164CF020E0C6
:20B5A00030E040E85FE32B833C834D835E830AC0C701B601A50194010E94D1C56B837C834A
:20B5C0008D839E8383E790E04E855F85489FD001499FB00D589FB00D1124A25BBB4F1896AE
:20B5E0002C91189730E048895989489FF001499FF00D589FF00D1124E25BFB4F808590E03A
:20B60000282B392B26FF32C0D1966D917D918D919C91D49721A932A943A954A90E9403C53B
:20B620004B015C01E894B7F8C090760CD090770CE090780CF090790CC501B401A7019601CE
:20B640000E94D8C7181694F4C701B601A50194010E94D1C52B013C016B817C818D819E8182
:20B66000A30192010E94CAC5882324F44B805C806D807E8083E790E0EE85FF85E89FD001E4
:20B68000E99FB00DF89FB00D1124A25BBB4F28893989289FF001299FF00D389FF00D1124DC
:20B6A000E25BFB4FD5966D917D918D919C91D89725A936A947A950AD0E9403C54B015C0125
:20B6C000E894B7F8E0917502F0917602C788D08CE18CF28CC501B401A70196010E94D8C7CD
:20B6E000181684F4C701B601A50194010E94D1C56B017C01C301B201A70196010E94CAC5E2
:20B70000882314F47301620103E710E048895989409FF001419FF00D509FF00D1124E25B07
:20B72000FB4FC701B60121AD32AD43AD54AD0E947AC86B017C018E859F85809FF001819F6E
:20B74000F00D909FF00D1124E25BFB4F11AD02ADB3ACA4ACC701B601212F302F4B2D5A2DBB
:20B760000E94CAC587FD06C0812F902FAB2DBA2D6C017D0183E790E0A889B989A89FF001B0
:20B78000A99FF00DB89FF00D1124E25BFB4FEB5BFF4FC082D182E282F382E554F04030E0D9
:20B7A0008085807F803809F431E020E083E790E04E855F85489FF001499FF00D589FF00D7D
:20B7C0001124E25BFB4F8085807F803809F421E0321761F103E710E088899989809FF0013B
:20B7E000819FF00D909FF00D1124E25BFB4F808182608083AE85BF85A09FF001A19FF00D7A
:20B80000B09FF00D1124E25BFB4F8081846080838B859C850E94815029853A85209FF00177
:20B82000219FF00D309FF00D1124C0C34D85242F30E083E790E0289F5001299FB00C389F45
:20B84000B00C11248EE494E0A80EB91EADE4B0E0AA0EBB1EF501C080D180E280F38023EB68
:20B860003FEFA20EB31E4F833F81332319F44FE04F8303C05F8151505F838F81882E99247A
:20B88000D50111968C91119781FF0CC0D9964C90D997DA965C90DA97DB966C90DB97DC9641
:20B8A0007C9013C0C701B601A70196010E947AC8F501EF5BFF4F20813181428153810E94ED
:20B8C00004C50E94E7C82B013C0123E730E0829EF001839EF00D929EF00D1124E25BFB4FB3
:20B8E000EB5BFF4F10810181F280D380E554F040F98BE88BB201C301212F302F4F2D5D2D50
:20B900000E94D8C788230CF4A1C0E889F989E35BFF4F6081718182819381212F302F4F2D46
:20B920005D2D0E94CAC5882391F1A889B9898C918E7F8C93E889F989EF5AFF4FC0807180A8
:20B9400062805380E02E0D2D6C2D772D862D952D212F3E2D4F2D5D2D0E94CAC587FD04C0FE
:20B960001C2DE72CF62C052D23E730E0829EF001839EF00D929EF00D1124E556FB4F812F37
:20B980009E2DAF2DB02F80839183A283B38343E750E0849EF001859EF00D949EF00D1124BE
:20B9A000ED56FB4FE080F18002811381F501E75BFF4F60817181828193819701A8010E94BF
:20B9C000CAC5882399F181E590E0A80EB91ED501DC901196CC90119712967C90129713964D
:20B9E0006C90EFEAFFEFAE0EBF1E6D2D7C2D872D962D9701A8010E94CAC587FD04C0ED2C5E
:20BA0000FC2C072D162D29E430E0A20EB31EC701D801F50180839183A283B38327EB3FEFA0
:20BA2000A20EB31ED5018C918E7F8C9323E730E0829EF001839EF00D929EF00D1124E55680
:20BA4000FB4FC080D180E280F38066C041E550E0A40EB51ED5011C911196EC90119712963F
:20BA6000FC90129713960C91EFEAFFEFAE0EBF1E612F7E2D8F2D902F9201A3010E94CAC5CD
:20BA8000882324F4142DE52CF62C072D29E430E0A20EB31E812F9E2DAF2DB02FF50180836E
:20BAA0009183A283B38327EB3FEFA20EB31E43E750E0849EF001859EF00D949EF00D112465
:20BAC000E156FB4FC080D180E280F380B201C301A70196010E94CAC587FD04C0C201D301B9
:20BAE0006C017D0183E790E0889EF001899EF00D989EF00D1124E25BFB4FE35BFF4FC08289
:20BB0000D182E282F382ED54F04080818E7F8083D5018C918E7F8C93BF81B31571F0E3E725
:20BB2000F0E08E9E50018F9EB00C9E9EB00C11242EE434E0A20EB31E97CE83E790E04985EE
:20BB40005A85489F7001499FF00C589FF00C11248EE494E0E80EF91EA9E4B0E0EA0EFB1E81
:20BB6000F701608071808280938027EB3FEFE20EF31E3F81388748854F3011F4188603C075
:20BB800058855F5F58878885282E3324E3E7F0E02E9ED0012F9EB00D3E9EB00D1124A25BE5
:20BBA000BB4FBA83A983D70111968C91119781FF0CC0D9961C91D997DA964C90DA97DB96C8
:20BBC0005C90DB97DC960C9115C0C401B301A40193010E947AC8F701EF5BFF4F20813181AA
:20BBE000428153810E9404C50E94E7C8162F472E582E092FF701E35BFF4FF98BE88B612F6F
:20BC0000742D852D902F20813181428153810E94D8C7F701EF5AFF4F18160CF0A8C0A080A6
:20BC2000B180C280D380C401B301A60195010E94CAC587FD03C06401530118C0C601B50102
:20BC4000A60195010E947AC8F701EF5BFF4F20813181428153810E9404C50E94E7C8A8895C
:20BC6000B9896D937D938D939C931397E9E4F0E0EE0EFF1ED701AD92BD92CD92DD927D0111
:20BC8000CC901196DC90119712960C91129713961C91E8EFFFEFEE0EFF1ED701BC901196A0
:20BCA000AC90119712969C90129713968C90EBEBFFEFEE0EFF1EB601C8012B2D3A2D492DCC
:20BCC000582D0E94CAC587FD04C0CB2CDA2C092D182D23E730E0229EF001239EF00D329E95
:20BCE000F00D1124E156FB4F6080718082809380B601C801A40193010E94CAC587FD04C079
:20BD0000C601D8013C014D0143E750E0249E8001259E100D349E100D1124025B1B4F075B2E
:20BD20001F4FD8016D927D928D929C92139709541040F701E35BFF4FD701AB5BBF4F6081B9
:20BD40007181828193812D913D914D915C910E94CAC5882341F4F701808182608083D801BB
:20BD60008C9184608C93F70180818E7FB4C0D7018C9186608E7F8C93A080B180C280D3803C
:20BD8000C601B501A40193010E94D8C718161CF06401530115C0C601B501A60195010E9488
:20BDA0007AC8F701EF5BFF4F20813181428153810E9404C50E94E7C8162F472E582E092F93
:20BDC000E9E4F0E0EE0EFF1ED701AD92BD92CD92DC921397E8E0F0E0EE0EFF1ED701DC90DB
:20BDE0001196CC9011971296BC9012971396AC90EFEAFFEFEE0EFF1E6D2D7C2D8B2D9A2D74
:20BE0000212F342D452D502F0E94CAC587FD04C01D2D4C2C5B2C0A2D2DE430E0E20EF31E65
:20BE2000812F942DA52DB02FF70180839183A283B38328EF3FEFE20EF31ED701DC90119645
:20BE4000CC9011971296BC9012971396FC90612F742D852D902F2D2D3C2D4B2D5F2D0E9401
:20BE6000CAC587FD04C01D2D4C2C5B2C0F2D23E730E0229EF001239EF00D329EF00D1124DB
:20BE8000E156FB4F6080718082809380612F742D852D902FA40193010E94CAC587FD06C0E5
:20BEA000812F942DA52DB02F3C014D0143E750E0249EF001259EF00D349EF00D1124E25BC7
:20BEC000FB4FE75BFF4F6082718282829382E954F04080818460808358858D85581719F0DE
:20BEE000E980FA8048CEE981FA81EF5AFF4F10810181F280E380612F702F8F2D9E2DA4018A
:20BF000093010E94CAC587FD06C0812F902FAF2DBE2D3C014D01E981FA81E75BFF4F6082FA
:20BF200071828282938213E7E12EF12CAF818A2F90E08E9D80018F9D100D9E9D100D1124F4
:20BF4000025B1B4FC8010E9481502FB7F894F80181818F778183FF81FF3011F41F8203C04F
:20BF60003F813F5F3F834F81842F90E08E9DF0018F9DF00D9E9DF00D1124E25BFB4F818173
:20BF8000806881832FBF8091800B481779F68B859C850E94815083E790E0AE85BF85A89F21
:20BFA000F001A99FF00DB89FF00D1124E25BFB4F81818F77818361960FB6F894DEBF0FBE7D
:20BFC000CDBFCF91DF911F910F91FF90EF90DF90CF90BF90AF909F908F907F906F905F9000
:20BFE0004F903F902F9008952F923F924F925F926F927F928F929F92AF92BF92CF92DF920B
:20C00000EF92FF920F931F93DF93CF93CDB7DEB76B970FB6F894DEBF0FBECDBF4C011B011B
:20C020004B8F25E530E0820E931ED401AD90BD90CD90DC90EBEAFFEF8E0E9F1ED401189604
:20C040008C91807320916A0C30916B0C40916C0C50916D0C8823D9F07090320C6090330CED
:20C060005090340C4090350CC901DA017C018D01672D762D852D942DA80197010E94CAC5C3
:20C0800087FD09C0872D962DA52DB42D02C0C901DA017C018D01C601B50120E034E244E7F9
:20C0A0005BE40E947AC8A80197010E94D1C52B013C018091FF0B90E0E6E096958795EA9564
:20C0C000E1F7B82FB170BC8B8091810B8A30C0F5C301B20120E034E244E758E40E94CAC508
:20C0E000882374F5E090810B60E074E284E798E4A30192010E9403C520E030E040E450E4AA
:20C100000E947AC85B016C01FF240894E11CF11C0027F7FC0095102FC801B7010E946CC666
:20C120009B01AC01C601B5010E94D1C59B01AC01C301B2010E9404C52B013C01E1E0EC8B35
:20C14000C301B2010E9439C6D40113966D937D938D939C9316978EE89FE00E94B599F40163
:20C16000E159FF4F60817181828193810E946CC66F8B788F898F9A8FC301B2012F89388D43
:20C18000498D5A8D0E94D1C50E9439C65B016C01F4016084762C64FE30C0D1016D917D9195
:20C1A0008D919C919F7720E034E244E75BE40E947AC87B018C016F89788D898D9A8D2091C6
:20C1C000EB013091EC014091ED015091EE010E947AC89B01AC01C801B7010E94D1C50E94AE
:20C1E00039C669837A838B839C836A157B058C059D053CF05B016C0104C019821A821B826B
:20C200001C8275FE30C0F10164817581868197819F7720E034E244E75BE40E947AC87B013B
:20C220008C016F89788D898D9A8D2091EF013091F0014091F1015091F2010E947AC89B01CD
:20C24000AC01C801B7010E94D1C50E9439C66D837E838F8398876A157B058C059D053CF057
:20C260005B016C0104C01D821E821F82188676FE32C0D10118966D917D918D919C911B97C4
:20C280009F7720E034E244E75BE40E947AC87B018C016F89788D898D9A8D2091F30130917B
:20C2A000F4014091F5015091F6010E947AC89B01AC01C801B7010E94D1C50E9439C6698773
:20C2C0007A878B879C876A157B058C059D053CF05B016C0104C019861A861B861C8667FE56
:20C2E00030C0F10164857585868597859F7720E034E244E75BE40E947AC87B018C016F89D7
:20C30000788D898D9A8D2091F7013091F8014091F9015091FA010E947AC89B01AC01C801DB
:20C32000B7010E94D1C50E9439C66D877E878F87988B6A157B058C059D053CF05B016C0113
:20C3400004C01D861E861F86188AC601B5016139F1E07F07F0E08F07F0E09F0724F461E9DF
:20C3600071E080E090E029E530E0820E931ED4016D937D938D939C931397E7EAFFEF8E0E04
:20C380009F1E0E946CC67B018C01F401E159FF4F60817181828193810E946CC69B01AC017F
:20C3A000C801B7010E947AC86B017C0160E074E284E79BE4A70196010E94D1C52B013C01CF
:20C3C000D40118968C911897082F10E084FF2DC019966D917D918D919C911C970E946CC6EA
:20C3E0009B01AC01C701B6010E94D1C50E9439C669837A838B839C83C301B201F10120817C
:20C400003181428153810E947AC8D40199966D937D938D939C939C97017110700031110520
:20C4200069F4DC01CB01B05804C080E090E0A0E0B0E0F40181A792A7A3A7B4A7D4011896CC
:20C440008C911897082F10E085FF2DC01D966D917D918D919C9150970E946CC69B01AC016A
:20C46000C701B6010E94D1C50E9439C66D837E838F839887C301B201F101248135814681B7
:20C4800057810E947AC8D4019D966D937D938D939C93D097027210700032110569F4DC019C
:20C4A000CB01B05804C080E090E0A0E0B0E0F40185A796A7A7A7B0ABD40118968C911897AE
:20C4C000082F10E086FF2DC051966D917D918D919C9154970E946CC69B01AC01C701B601FE
:20C4E0000E94D1C50E9439C669877A878B879C87C301B201F10120853185428553850E9438
:20C500007AC8D401D1966D937D938D939C93D497047410700034110569F4DC01CB01B05883
:20C5200004C080E090E0A0E0B0E0F40181AB92ABA3ABB4ABD40118961C91189717FF2FC068
:20C5400055966D917D918D919C9158970E946CC69B01AC01C701B6010E94D1C50E9439C635
:20C560006D877E878F87988BC301B201F10124853585468557850E947AC8D401D5966D93F2
:20C580007D938D939C93D8971878103841F4DC01CB01B058F40185AB96ABA7ABB0AFF40103
:20C5A000EB5AFF4F6081718182819381A30192010E947AC8D401D9966D937D938D939C9340
:20C5C000DC9718968C91E82FF0E0FB8BEA8BCF01887890708838910529F028EA3BE03E8B06
:20C5E0002D8B04C088E99BE09E8B8D8B79EA272E6FE5362E53E6452E48E5542E66247724A2
:20C60000AA24BB2480E190E0062C02C0880F991F0A94E2F7AA89BB898A239B23892B41F11A
:20C62000E1E0F0E0EC0FFD1FEA0DFB1D60817181828193810E946CC67B018C01ED89FE897F
:20C64000EA0DFB1D60817181828193810E946AC69B01AC01C801B7010E947AC86B017C0178
:20C66000B101C201A70196010E94CAC5882324F4C101D2016C017D010894611C711CE4E028
:20C68000F0E0AE0EBF1EF4E06F16710429F0D701C60116012D01B6CFD4011296BC900B2DE0
:20C6A00010E0000F111F000F111FF401E00FF11F81859285A385B485B595A79597958795CC
:20C6C000F40181A392A3A3A3B4A3858F968FA78FB0A3818F928FA38FB48F60E070E080E80F
:20C6E0009FE321AD32AD43AD54AD0E94D1C52DE330E0820E931ED4016D937D938D939C934D
:20C7000013970C0F1D1FF80161817281838194810E946CC69B01AC01C701B6010E94D1C55D
:20C720000E943EC624E230E0820E931ED4016D937D938D939D934D010E946AC620E030E097
:20C7400040E858E40E947AC820E034E244E75BE40E94D1C50E943EC6F40160837183828362
:20C7600093832BE93FEF820E931E84010F5B1F4F85E590E0880E991ED4012D913D914D915D
:20C780005C91EBEAFFEF8E0E9F1ECA01B9010E9404C5A70196010E947AC8D401D9962D917B
:20C7A0003D914D915C91DC970E947AC820E034E244E75BE40E94D1C5F801608371838283FC
:20C7C00093836091720C7091730C8091740C9091750C20E030E040E05FE30E947AC81B01AF
:20C7E0002C01D4011896BC91B98B6B2E7724B6FF5AC0F401E1A8F2A803A914A9F2E0BF16CD
:20C80000F9F46091760C7091770C8091780C9091790C20E030E040E05FE30E947AC8D401CE
:20C82000D9962D913D914D915C91DC970E947AC8A80197015F770E94D1C57B018C0135C08E
:20C8400057016801E894D7F86091760C7091770C8091780C9091790C20E030E040E05FE328
:20C860000E947AC87B018C01C601B501A80197010E94D8C71816BCF4C801B701F40121ADAA
:20C8800032AD43AD54AD0E947AC8A60195010E94D1C57B018C01C201B101A80197010E940E
:20C8A000CAC5882314F482017101F989F7FF3CC020E762227724E0917502F0917602672837
:20C8C00031F16789708D818D928D20E030E040E05FE30E947AC8D401D9962D913D914D9118
:20C8E0005C91DC970E947AC8F40125A936A947A950AD5F770E94D1C55B016C01C801B7010D
:20C90000A60195010E94CAC587FD0EC00FC06789708D818D928D20E030E040E05FE30E945A
:20C920007AC85B016C0102C057016801D40112968C91823048F4E090320CF090330C0091E3
:20C94000340C1091350C0AC0823081F4E090360CF090370C0091380C1091390CC801B70113
:20C96000A60195010E94CAC5882314F486017501F401D1ACC2ACB3ACA4ACC801B7012D2D2F
:20C980003C2D4B2D5A2D0E94CAC587FD06C08D2D9C2DAB2DBA2D7C018D0121E530E0820EC1
:20C9A000931ED401ED92FD920D931C931397F40112930293F292E292DF011E930E93FE9201
:20C9C000EE924D01E7EBFFEF8E0E9F1ED401D996AD90BD90CD90DC90DC97C801B701A8013C
:20C9E00097010E947AC8F401EF5BFF4F20813181428153810E9404C57B018C01C601B50153
:20CA0000A60195010E947AC89B01AC01C801B7010E94D8C7882324F0F4018181826081834E
:20CA20008401075A1F4FD8012D913D914D915C9160E074E284EF90E00E94A3C9E9E6F0E04C
:20CA40008E0E9F1ED4012D933C93E7E9FFEF8E0E9F1E8EE89FE00E94B5990E944959F801E0
:20CA600080819181A281B3818F5C9740A040B04018F02C89222329F084E0D40117968C939A
:20CA800020C081E0F4018783E281F0E0EE0FFF1FEE0FFF1FE80DF91D81859285A385B48564
:20CAA000F40185A396A3A7A3B0A781A392A3A3A3B4A3858F968FA78FB0A3818F928FA38F64
:20CAC000B48FFB8DFF2331F086E490E090934D0480934C048091800B8F5F8093800B8031BE
:20CAE00010F01092800B8091010C80618093010C9FB7F8948091810B8F5F8093810B9FBF80
:20CB00006B960FB6F894DEBF0FBECDBFCF91DF911F910F91FF90EF90DF90CF90BF90AF9043
:20CB20009F908F907F906F905F904F903F902F9008952F923F924F925F926F927F928F9209
:20CB40009F92AF92BF92CF92DF92EF92FF920F931F93DF93CF93CDB7DEB7A1970FB6F89464
:20CB6000DEBF0FBECDBF182F6A8F8091FF0B8E7F8093FF0B81E00E9430568A8D60E00E94B8
:20CB80008C518B8B8091800B282E3324112371F083E790E0289EF001299EF00D389EF00D9C
:20CBA0001124E25BFB4F80E181830CC083E790E0289EF001299EF00D389EF00D1124E25BEE
:20CBC000FB4F118283E790E0289EF001299EF00D389EF00D1124E25BFB4F10822A8D222306
:20CBE00011F482E0808383E790E0289E7001299EF00C389EF00C11248701025B1B4FD801C8
:20CC000018961C920E941B6AE091700CF091710CFD8BEC8B2BEB3BE03A8B298B87E5682EFB
:20CC200084E0782E6E0C7F1C44245524AA24BB24085F1F4F4801C8010D969D8F8C8FCF01A6
:20CC4000A0E0B0E08E8F9F8FA8A3B9A34B8EF501ED51F44F80819181A281B3818E8B9F8BD5
:20CC6000A88FB98FE989FA8980819181A281B3812E893F89488D598D281B390B4A0B5B0B5A
:20CC8000D3012D933D934D935C93139757FD0DC021E030E0042C02C0220F331F0A94E2F799
:20CCA000F4018081822B80830CC088279927DC01821B930BA40BB50BF30180839183A283DC
:20CCC000B383F3E04F1649F52C893D892436310521F1AC8DBD8D6D917D918D919C910E940F
:20CCE0006CC67B018C016E8D7F8D88A199A10E946AC69B01AC01C801B7010E947AC82AE005
:20CD000037ED43E25CE30E947AC80E9439C6EC8DFD8D6083718382839383D301ED90FD9033
:20CD20000D911C91B1E0CB2ED12CCC0EDD1ECA0CDB1CC801B7010E946CC6F501E857F44FB2
:20CD400020813181428153810E947AC8F6016083718382839383E114F1040105110561F0C5
:20CD600020E130E00B8C02C0220F331F0A94E2F7D4018C91822B8C93E989FA898E899F895D
:20CD8000A88DB98D81939193A193B193FA8BE98B0894411C511C24E030E0A20EB31E620E04
:20CDA000731E30E1A316B10409F050CF83E790E0289E8001299E100D389E100D1124025BC1
:20CDC0001B4FD80118968C91807F59F4BB89BB2309F41BC11092810B8091800B8093820B94
:20CDE00014C16D847E848F8498886091880C7091890C80918A0C90918B0CA40193010E94E3
:20CE000004C56093880C7093890C80938A0C90938B0CF8012585368547855089C184D28429
:20CE2000E384F484C216D306E406F506A4F481899289A389B48982179307A407B5075CF46D
:20CE400085899689A789B08D82179307A407B50714F481E036C083E790E0289EF001299EE7
:20CE6000F00D389EF00D1124E25BFB4F21893289438954892C153D054E055F055CF4858980
:20CE80009689A789B08D8C159D05AE05BF0514F4128218C083E790E0289EF001299EF00D83
:20CEA000389EF00D1124E25BFB4F85899689A789B08D82179307A407B50714F482E001C084
:20CEC00083E0828383E790E09C01229EC001239E900D329E900D11249C01225B3B4FD90174
:20CEE0001296EC91F0E0EE0FFF1FEE0FFF1FE80FF91FE25BFB4F81859285A385B485215979
:20CF00003F4FF90180839183A283B3832F563040D90118968C91482E5524C20180779070D4
:20CF2000892B09F456C029813A814B815C81ED80FE800F811885CA01B9010E947AC85B013F
:20CF40006C01C801B701A80197010E947AC89B01AC01C601B5010E9404C57B018C0164011F
:20CF60005301E894D7F846FE0EC029853A854B855C85CA01B9010E947AC89B01AC01C80167
:20CF8000B7010E9404C50E94E7C8962E872E782E692ED601C50175018D01692D782D872DD7
:20CFA000962D9501AD010E94CAC587FD04C0E92CF82C072D162D83E790E0289EF001299EE9
:20CFC000F00D389EF00D1124ED55FB4FC701D80106C0F901EB5AFF4FD401C301BF778083FA
:20CFE0009183A283B38383E790E0FC012E9EC0012F9E900D3E9E900D1124825B9B4FBE01C0
:20D000006F5F7F4F4A8D0E94F45FA1960FB6F894DEBF0FBECDBFCF91DF911F910F91FF907B
:20D02000EF90DF90CF90BF90AF909F908F907F906F905F904F903F902F9008952F923F922E
:20D040004F925F926F927F928F929F92AF92BF92CF92DF92EF92FF920F931F93DF93CF93FC
:20D06000CDB7DEB760970FB6F894DEBF0FBECDBF1B012C012D833E834F835887E986FA86FF
:20D080000B871C87AD86BE86CF86D88A0E946CC62091880B3091890B40918A0B50918B0BE3
:20D0A0000E947AC82091D70B3091D80B4091D90B5091DA0B0E9404C53B014C01CB01D40145
:20D0C0008093D70B9093D80BA093D90BB093DA0B6D817E818F8198850E946CC620918C0BE0
:20D0E00030918D0B40918E0B50918F0B0E947AC82091DB0B3091DC0B4091DD0B5091DE0B4C
:20D100000E9404C55B016C01CB01D6018093DB0B9093DC0BA093DD0BB093DE0BC801B7016D
:20D120000E946CC62091900B3091910B4091920B5091930B0E947AC82091DF0B3091E00B5A
:20D140004091E10B5091E20B0E9404C57B018C01CB01D8018093DF0B9093E00BA093E10B01
:20D16000B093E20BB301C4019501A6010E94D96B882309F49EC0211431044104510449F49C
:20D1800020E83FE443EC57E429833A834B835C830CC08091D70B9091D80BA091D90BB091CB
:20D1A000DA0B89839A83AB83BC832D813E814F815885211531054105510559F40F2EF0E870
:20D1C0002F2EFFE43F2EF3EC4F2EF7E45F2EF02D08C02090DB0B3090DC0B4090DD0B509024
:20D1E000DE0B89859A85AB85BC850097A105B10559F40F2EF0E86F2EFFE47F2EF3EC8F2E8A
:20D20000F7E49F2EF02D08C06090DF0B7090E00B8090E10B9090E20B00D000D00DB71EB77A
:20D220000F5F1F4F6091C70B7091C80B8091C90B9091CA0B2D853E854F855889620F731F73
:20D24000841F951F0E946CC62091940B3091950B4091960B5091970B0E947AC85B016C0150
:20D260008DA19EA1AFA1B8A5F80180839183A283B38369817A818B819C81A2019101840161
:20D2800073010E94BA720F900F900F900F9080E00E94986A89A5882311F00E94D31B0E94C0
:20D2A000E3C26093400470934104809342049093430460960FB6F894DEBF0FBECDBFCF91EA
:20D2C000DF911F910F91FF90EF90DF90CF90BF90AF909F908F907F906F905F904F903F902B
:20D2E0002F9008952F923F924F925F926F927F928F929F92AF92BF92CF92DF92EF92FF9294
:20D300000F931F93DF93CF93CDB7DEB720906A0C30906B0C40906C0C50906D0C6090BB0B18
:20D320007090BC0B8090BD0B9090BE0B660E771E881E991E6092E30B7092E40B8092E50B2C
:20D340009092E60B8091BF0B9091C00BA091C10BB091C20B820F931FA41FB51F8093E70B09
:20D360009093E80BA093E90BB093EA0B8091C30B9091C40BA091C50BB091C60B8E0D9F1DFF
:20D38000A01FB11F8093EB0B9093EC0BA093ED0BB093EE0B8091C70B9091C80BA091C90B98
:20D3A000B091CA0B8A0D9B1DAC1DBD1D8093EF0B9093F00BA093F10BB093F20B8D899E898E
:20D3C000AF89B88D80936A0C90936B0CA0936C0CB0936D0C8A8D60E00E94996520926A0C27
:20D3E00030926B0C40926C0C50926D0C80E00E94986A898D882311F00E94D31B0E94E3C2B2
:20D4000060934004709341048093420490934304CF91DF911F910F91FF90EF90DF90CF90CE
:20D42000BF90AF909F908F907F906F905F904F903F902F9008958091000C85FD57C02091A2
:20D440003A0C30913B0C40913C0C50913D0C8091E30B9091E40BA091E50BB091E60B28179A
:20D4600039074A075B0744F42093E30B3093E40B4093E50B5093E60B20913E0C30913F0C90
:20D480004091400C5091410C8091E70B9091E80BA091E90BB091EA0B281739074A075B079D
:20D4A00044F42093E70B3093E80B4093E90B5093EA0B2091420C3091430C4091440C509129
:20D4C000450C8091EB0B9091EC0BA091ED0BB091EE0B281739074A075B0744F42093EB0B66
:20D4E0003093EC0B4093ED0B5093EE0B0895EF92FF920F931F936093F30B7093F40B8093C2
:20D50000F50B9093F60B2093F70B3093F80B4093F90B5093FA0BE092FB0BF092FC0B009319
:20D52000FD0B1093FE0B1F910F91FF90EF9008954F925F926F927F929F92AF92BF92CF9234
:20D54000DF92EF92FF920F931F93DF93CF9300D000D0CDB7DEB7982E6091BB0B7091BC0B22
:20D560008091BD0B9091BE0B0E946CC62091880B3091890B40918A0B50918B0B0E947AC8BA
:20D580007B018C016091BF0B7091C00B8091C10B9091C20B0E946CC620918C0B30918D0BBB
:20D5A00040918E0B50918F0B0E947AC85B016C016091C30B7091C40B8091C50B9091C60B77
:20D5C0000E946CC62091900B3091910B4091920B5091930B0E947AC869837A838B839C83E7
:20D5E00029813A814B815C81C901DA018093D30B9093D40BA093D50BB093D60BC801B701CD
:20D6000020917A0C30917B0C40917C0C50917D0C0E9403C52B013C01CB01D3018093CB0B6C
:20D620009093CC0BA093CD0BB093CE0BC601B50120917E0C30917F0C4091800C5091810CFA
:20D640000E9403C57B018C01CB01D8018093CF0B9093D00BA093D10BB093D20B992011F1DD
:20D66000C201D3018093D70B9093D80BA093D90BB093DA0BC701D8018093DB0B9093DC0B35
:20D68000A093DD0BB093DE0B29813A814B815C81C901DA018093DF0B9093E00BA093E10B66
:20D6A000B093E20B0F900F900F900F90CF91DF911F910F91FF90EF90DF90CF90BF90AF9034
:20D6C0009F907F906F905F904F90089580E00E94986A8091CB0B9091CC0BA091CD0BB09175
:20D6E000CE0B80938D0C90938E0CA0938F0CB093900C8091CF0B9091D00BA091D10BB09106
:20D70000D20B8093910C9093920CA093930CB093940C8091D30B9091D40BA091D50BB091C5
:20D72000D60B8093950C9093960CA093970CB093980C6091C70B7091C80B8091C90B909135
:20D74000CA0B0E946CC62091E7013091E8014091E9015091EA010E947AC86093990C7093D7
:20D760009A0C80939B0C90939C0C0895382F2091FF0B822F90E045E0969587954A95E1F77B
:20D7800081703817A9F0332319F0822F806202C0822F8F7D8093FF0B332319F082E996E0E2
:20D7A00002C087EA96E00E943A2A80E00E94986A089581E008959F92AF92BF92CF92DF9286
:20D7C000EF92FF920F931F93CF93DF930EE81FE0C80166E676E140E00E94BB98C8010E942E
:20D7E00091B6E0904E0CF0904F0C0091500C1091510C8091420C9091430CA091440CB091C1
:20D80000450CE81AF90A0A0B1B0B88279927DC018E199F09A00BB10B8093C30B9093C40BA2
:20D82000A093C50BB093C60B00D000D000D0EDB7FEB73196EE0CFF1C001F111F80910302C7
:20D8400090910402A0910502B0910602CDB7DEB789839A83AB83BC83992493949482958260
:20D8600060E070E080E090E020E030E040E050E0AA24BB2465010E94726980914E0C9091CC
:20D880004F0CA091500CB091510C8093C30B9093C40BA093C50BB093C60BCDB6DEB6089465
:20D8A000C11CD11C2091E3013091E4014091E5015091E601CA01B9010E9404C50E9439C653
:20D8C0007B018C016091030270910402809105029091060220E030E040E450E40E94D1C561
:20D8E000F60160837183828393839482158260E070E080E090E020E030E040E050E0AA2404
:20D90000BB2465010E947269CDB6DEB60894C11CD11C2091E3013091E4014091E5015091F5
:20D92000E601CA01B9010E9404C520E030E040E050EC0E947AC80E9439C67B018C01609125
:20D94000030270910402809105029091060220E030E040E450E40E94D1C5E601688379830C
:20D960008A839B839C829D8260E070E080E090E020E030E040E050E0AA24BB2465010E94CA
:20D98000726980914E0C90914F0CA091500CB091510C8093C30B9093C40BA093C50BB09381
:20D9A000C60BEDB7FEB736960FB6F894FEBF0FBEEDBFDF91CF911F910F91FF90EF90DF904D
:20D9C000CF90BF90AF909F9008959F92AF92BF92CF92DF92EF92FF920F931F93CF93DF93BF
:20D9E0000EE81FE0C8016DE676E140E00E94BB98C8010E9491B620914A0C30914B0C409108
:20DA00004C0C50914D0C80913E0C90913F0CA091400CB091410C281B390B4A0B5B0B8827B1
:20DA20009927DC01821B930BA40BB50B8093BF0B9093C00BA093C10BB093C20B00D000D025
:20DA400000D0EDB7FEB73196220F331F441F551F8091FF0190910002A0910102B0910202CF
:20DA6000CDB7DEB789839A83AB83BC83992493949482958260E070E080E090E0EE24FF2451
:20DA80008701AA24BB2465010E94726980914A0C90914B0CA0914C0CB0914D0C8093BF0B8F
:20DAA0009093C00BA093C10BB093C20B0DB71EB70F5F1F4F6091DF017091E0018091E1014E
:20DAC0009091E20120E030E040EA50E40E947AC80E9439C66B017C016091FF017091000272
:20DAE000809101029091020220E030E040E450E40E94D1C5F801608371838283938394824C
:20DB0000158260E070E080E090E0A7019601EE24FF248701AA24BB2465010E947269CDB6FF
:20DB2000DEB60894C11CD11C2091DF013091E0014091E1015091E201CA01B9010E9404C551
:20DB400020E030E040EA50EC0E947AC80E9439C67B018C016091FF017091000280910102B9
:20DB60009091020220E030E040E450E40E94D1C5E601688379838A839B839C829D8260E06A
:20DB800070E080E090E0A8019701EE24FF248701AA24BB2465010E9472690DB71EB70F5FD0
:20DBA0001F4F6091DF017091E0018091E1019091E2010E9439C69B01AC018091FF01909131
:20DBC0000002A0910102B0910202F80180839183A283B3839482158260E070E080E090E052
:20DBE000EE24FF2487010E94726980914A0C90914B0CA0914C0CB0914D0C8093BF0B9093E9
:20DC0000C00BA093C10BB093C20B8DB79EB706960FB6F8949EBF0FBE8DBFDF91CF911F91AE
:20DC20000F91FF90EF90DF90CF90BF90AF909F9008959F92AF92BF92CF92DF92EF92FF9267
:20DC40000F931F930EE81FE0C80164E776E140E00E94BB98C8010E9491B66091460C709105
:20DC6000470C8091480C9091490C20913A0C30913B0C40913C0C50913D0C621B730B840BAA
:20DC8000950B22273327A901261B370B480B590B2093BB0B3093BC0B4093BD0B5093BE0B13
:20DCA00000D000D000D0EDB7FEB73196660F771F881F991F2091FB013091FC014091FD0130
:20DCC0005091FE01ADB7BEB711962D933D934D935C931497992493949482958220E030E0B9
:20DCE00040E050E0EE24FF248701AA24BB2465010E9472698091460C9091470CA091480C2B
:20DD0000B091490C8093BB0B9093BC0BA093BD0BB093BE0B0DB71EB70F5F1F4F6091DB0161
:20DD20007091DC018091DD019091DE0120E030E040EA50E40E947AC80E9439C66B017C013A
:20DD40006091FB017091FC018091FD019091FE0120E030E040E450E40E94D1C5F80160832D
:20DD600071838283938394821582C701B60120E030E040E050E0EE24FF248701AA24BB249E
:20DD800065010E947269CDB6DEB60894C11CD11C2091DB013091DC014091DD015091DE0189
:20DDA000CA01B9010E9404C520E030E040EA50EC0E947AC80E9439C67B018C016091FB0182
:20DDC0007091FC018091FD019091FE0120E030E040E450E40E94D1C5D6016D937D938D936F
:20DDE0009C93139714969C92149715969C92C801B70120E030E040E050E0EE24FF24870150
:20DE0000AA24BB2465010E9472690DB71EB70F5F1F4F6091DB017091DC018091DD01909142
:20DE2000DE010E9439C62091FB013091FC014091FD015091FE01F80120833183428353835D
:20DE40009482158220E030E040E050E0EE24FF2487010E9472698091460C9091470CA09173
:20DE6000480CB091490C8093BB0B9093BC0BA093BD0BB093BE0B8DB79EB706960FB6F89468
:20DE80009EBF0FBE8DBF1F910F91FF90EF90DF90CF90BF90AF909F9008952F923F924F9213
:20DEA0005F926F927F928F929F92AF92BF92CF92DF92EF92FF920F931F93DF93CF93CDB7EB
:20DEC000DEB72B970FB6F894DEBF0FBECDBF9B878A872091B90B2987DC018C91222309F014
:20DEE000A7C083FF34C01A962D913D914D915C911D978091870B882351F0CA01B90123E370
:20DF000033E34BEC51E40E947AC89B01AC01CA01B9012091F30B3091F40B4091F50B5091AC
:20DF2000F60B0E9403C5DC019B01AC012093CB0B3093CC0B4093CD0B5093CE0BCB018093E7
:20DF4000D70B9093D80BA093D90BB093DA0BEA85FB85808184FF32C026853785408951892B
:20DF60008091870B882351F0CA01B90123E333E34BEC51E40E947AC89B01AC01CA01B90153
:20DF80002091F70B3091F80B4091F90B5091FA0B0E9403C5DC019B01AC012093CF0B30936F
:20DFA000D00B4093D10B5093D20BCB018093DB0B9093DC0BA093DD0BB093DE0BAA85BB8592
:20DFC0008C9185FFDBC052962D913D914D915C9155978091870B882351F0CA01B90123E3C0
:20DFE00033E34BEC51E40E947AC89B01AC01CA01B9012091FB0B3091FC0B4091FD0B5091B4
:20E00000FE0B0E9403C5DC019B01AC012093D30B3093D40B4093D50B5093D60BCB018093DE
:20E02000DF0B9093E00BA093E10BB093E20BA6C083FF34C0E090D70BF090D80B0091D90B93
:20E040001091DA0BEA85FB8522853385448555858091870B882351F0CA01B90123E333E319
:20E060004BEC51E40E947AC89B01AC01C801B7010E9404C5DC019B01AC012093D70B30939D
:20E08000D80B4093D90B5093DA0BCB018093CB0B9093CC0BA093CD0BB093CE0BAA85BB85D9
:20E0A0008C9184FF34C0E090DB0BF090DC0B0091DD0B1091DE0B1E962D913D914D915C9101
:20E0C00051978091870B882351F0CA01B90123E333E34BEC51E40E947AC89B01AC01C801C6
:20E0E000B7010E9404C5DC019B01AC012093DB0B3093DC0B4093DD0B5093DE0BCB0180932E
:20E10000CF0B9093D00BA093D10BB093D20BEA85FB85808185FF32C0E090DF0BF090E00BCD
:20E120000091E10B1091E20B22893389448955898091870B882351F0CA01B90123E333E392
:20E140004BEC51E40E947AC89B01AC01C801B7010E9404C5DC019B01AC012093DF0B3093B4
:20E16000E00B4093E10B5093E20BCB018093D30B9093D40BA093D50BB093D60B2091D70B9C
:20E180003091D80B4091D90B5091DA0B29833A834B835C832090DB0B3090DC0B4090DD0B55
:20E1A0005090DE0B8091DF0B9091E00BA091E10BB091E20B8D839E83AF83B887CA01B9011D
:20E1C00020917A0C30917B0C40917C0C50917D0C0E9404C52091DB013091DC014091DD01B8
:20E1E0005091DE010E947AC820E030E040E05FE30E9404C50E94A7C63B014C01C201B10191
:20E2000020917E0C30917F0C4091800C5091810C0E9404C52091DF013091E0014091E1015B
:20E220005091E2010E947AC820E030E040E05FE30E9404C50E94A7C65B016C016D817E8194
:20E240008F8198852091E3013091E4014091E5015091E6010E947AC820E030E040E05FE381
:20E260000E9404C50E94A7C67B018C01C401B3010E9439C66093E30B7093E40B8093E50B2B
:20E280009093E60BC601B5010E9439C66093E70B7093E80B8093E90B9093EA0BC801B701D1
:20E2A0000E9439C66093EB0B7093EC0B8093ED0B9093EE0BAA85BB858C9186FF4AC1809186
:20E2C000270283FD46C15696ED90FD900D911C9159976090E7017090E8018090E901909082
:20E2E000EA01C801B701A40193010E947AC89B01AC018091870B882351F0CA01B90123E332
:20E3000033E34BEC51E40E947AC89B01AC01CA01B9010E9439C65B016C01B985BB2321F42E
:20E320008091BA0B882359F1E0917502F091760264A575A586A597A520E030E046E153E439
:20E340000E94CAC587FD0BC0C801B7019F7720E030E040E253E40E94D8C718161CF4AA24F0
:20E36000BB2465018091C70B9091C80BA091C90BB091CA0B8A0D9B1DAC1DBD1DF2C0E09151
:20E380007502F091760264A575A586A597A520E030E046E153E40E94CAC587FD26C0809169
:20E3A000C70B9091C80BA091C90BB091CA0BA6019501281B390B4A0B5B0BCA01B9010E94D6
:20E3C0006CC67B018C01E89417F9C401B30120E030E040E253E40E947AC89B01AC01C8019E
:20E3E000B7010E94D8C7181644F4A092C70BB092C80BC092C90BD092CA0BA092EF0BB092DA
:20E40000F00BC092F10BD092F20BAA85BB858D919C91119790FF3FC08091870BC0906E0CF7
:20E42000D0906F0C8823D1F05A966D917D918D919C915D972FE737EB4AE85BE30E947AC8CE
:20E440007B018C01B601882777FD8095982F0E946CC69B01AC01C801B70113C0B601882726
:20E4600077FD8095982F0E946CC6EA85FB85228D338D448D558D0E947AC82EE333EC4EE223
:20E4800059E30E947AC860936A0C70936B0C80936C0C90936D0C69817A818B819C81A201A1
:20E4A0009101ED80FE800F8118850E94D96B882391F48091EF0B9091F00BA091F10BB09107
:20E4C000F20B8093C70B9093C80BA093C90BB093CA0B80E025C0AA85BB852D913C91C9013C
:20E4E00088739070892BD1F426FD02C060E017C060E02091EF0B3091F00B4091F10B509157
:20E50000F20B8091C70B9091C80BA091C90BB091CA0B281739074A075B0709F061E0862FEB
:20E520002B960FB6F894DEBF0FBECDBFCF91DF911F910F91FF90EF90DF90CF90BF90AF9049
:20E540009F908F907F906F905F904F903F902F9008958091C70B9091C80BA091C90BB09149
:20E56000CA0B8093EF0B9093F00BA093F10BB093F20B4BCF2F923F924F925F926F927F929C
:20E580008F929F92AF92BF92CF92DF92EF92FF920F931F93DF93CF93CDB7DEB73B014C01E9
:20E5A00019012A0120E83FE443EC57E40E94CAC5882341F46090CB0B7090CC0B8090CD0BEB
:20E5C0009090CE0BC201B10120E83FE443EC57E40E94CAC5882341F42090CF0B3090D00B02
:20E5E0004090D10B5090D20BC801B70120E83FE443EC57E40E94CAC5882341F4E090D30B3D
:20E60000F090D40B0091D50B1091D60B6092CB0B7092CC0B8092CD0B9092CE0B2092CF0B96
:20E620003092D00B4092D10B5092D20BE092D30BF092D40B0093D50B1093D60BC401B301AF
:20E6400020917A0C30917B0C40917C0C50917D0C0E9404C53B014C01C201B10120917E0CD4
:20E6600030917F0C4091800C5091810C0E9404C51B012C01C401B30120E83FE443EC57E4C1
:20E680000E94CAC58823F1F0C401B3012091DB013091DC014091DD015091DE010E947AC8C6
:20E6A00020E030E040E05FE30E9404C50E94A7C60E9439C66093E30B7093E40B8093E50BF7
:20E6C0009093E60BC201B10120E83FE443EC57E40E94CAC58823F1F0C201B1012091DF0159
:20E6E0003091E0014091E1015091E2010E947AC820E030E040E05FE30E9404C50E94A7C631
:20E700000E9439C66093E70B7093E80B8093E90B9093EA0BC801B70120E83FE443EC57E448
:20E720000E94CAC58823F1F0C801B7012091E3013091E4014091E5015091E6010E947AC8FD
:20E7400020E030E040E05FE30E9404C50E94A7C60E9439C66093EB0B7093EC0B8093ED0B3E
:20E760009093EE0BC601B50120E83FE443EC57E40E94CAC58823B1F0C601B5012091E701D8
:20E780003091E8014091E9015091EA010E947AC80E9439C66093EF0B7093F00B8093F10BC9
:20E7A0009093F20B6D897E898F89988D20E83FE443EC57E40E94CAC5882361F08D899E8900
:20E7C000AF89B88D80936A0C90936B0CA0936C0CB0936D0C81E061E00E949965CF91DF9120
:20E7E0001F910F91FF90EF90DF90CF90BF90AF909F908F907F906F905F904F903F902F90A7
:20E8000008953F924F925F926F927F928F929F92AF92BF92CF92DF92EF92FF920F931F938A
:20E82000582E462E342E6090CB0B7090CC0B8090CD0B9090CE0BA090CF0BB090D00BC09089
:20E84000D10BD090D20BE090D30BF090D40B0091D50B1091D60B8091000C81608093000CE2
:20E86000552011F00E94196E442011F00E94E56C332011F00E94DB6B552041F06090560C6D
:20E880007090570C8090580C9090590C442041F0A0905E0CB0905F0CC090600CD090610CB9
:20E8A000332041F0E090660CF090670C0091680C1091690C81E00E94986A00D000D080912E
:20E8C000FB019091FC01A091FD01B091FE01EDB7FEB781839283A383B483C401B301A601C0
:20E8E00095010F2EF0E8AF2EFFE4BF2EF3ECCF2EF7E4DF2EF02D0E94BA721092CE0F0F90F3
:20E900000F900F900F900E9436191F910F91FF90EF90DF90CF90BF90AF909F908F907F9012
:20E920006F905F904F903F9008952F923F924F925F926F927F928F929F92AF92BF92CF92E3
:20E94000DF92EF92FF920F931F93362FF42FA22F17012801882329F4662319F4E1E0E4271C
:20E9600001C0E0E060906A0C70906B0C80906C0C90906D0CEE2339F4882329F460E87FE467
:20E9800083EC97E40AC060918D0C70918E0C80918F0C9091900CEE2339F4332329F420E87C
:20E9A0003FE443EC57E40AC02091910C3091920C4091930C5091940CEE2369F4FF2359F485
:20E9C0000F2EF0E8EF2EFFE4FF2EF3EC0F2FF7E41F2FF02D08C0E090950CF090960C009106
:20E9E000970C1091980CAA2359F40F2EF0E8AF2EFFE4BF2EF3ECCF2EF7E4DF2EF02D08C0AA
:20EA0000A090990CB0909A0CC0909B0CD0909C0C00D000D0EDB7FEB7218232824382548251
:20EA20000E94BA7260926A0C70926B0C80926C0C90926D0C0F900F900F900F901F910F9136
:20EA4000FF90EF90DF90CF90BF90AF909F908F907F906F905F904F903F902F9008951F9345
:20EA6000182F9091FF0B90FF42C0882309F43FC042C091609093FF0B5E9A5E9A159A0E948B
:20EA8000EA3E112341F560E070E080E090E040E020E00E94F73E60E070E080E090E041E00C
:20EAA00020E00E94F73E60E070E080E090E040E00E94303B8EE89FE06CE876E140E00E9490
:20EAC000BB988EE89FE00E9491B68091000C88608093000C10C08EE89FE06BE776E140E053
:20EAE0000E94BB988EE89FE00E9491B604C08091000C83FFBECF1F910895EF92FF920F9352
:20EB00001F930E94B61B8EE89FE00E94B5990E94E3C29B01AC018091810B882349F0209327
:20EB200040043093410440934204509343043CC08091400490914104A0914204B091430490
:20EB400079018A01E81AF90A0A0B1B0B8091440490914504A0914604B09147040097A10569
:20EB6000B10549F08E159F05A007B10720F480E00E942F7505C08091000C877F8093000C3F
:20EB80008091D1019091D201A091D301B091D4010097A105B10541F08E159F05A007B107B9
:20EBA00018F481E00E942F751F910F91FF90EF9008952F923F924F925F926F927F928F9210
:20EBC0009F92AF92BF92CF92DF92EF92FF920F931F93DF93CF93CDB7DEB728970FB6F8943D
:20EBE000DEBF0FBECDBF8091DB019091DC01A091DD01B091DE018D839E83AF83B8872090B3
:20EC0000560C3090570C4090580C5090590CC201B1012091520C3091530C4091540C509140
:20EC2000550C0E9404C59B01AC016D817E818F8198850E947AC80E9439C660933A0C7093E4
:20EC40003B0C80933C0C90933D0CA090DF01B090E001C090E101D090E20160905E0C7090A6
:20EC60005F0C8090600C9090610CC401B30120915A0C30915B0C40915C0C50915D0C0E9443
:20EC800004C59B01AC01C601B5010E947AC80E9439C660933E0C70933F0C8093400C909353
:20ECA000410C8091E3019091E401A091E501B091E60189839A83AB83BC83E090660CF090D5
:20ECC000670C0091680C1091690CC801B7012091620C3091630C4091640C5091650C0E94A1
:20ECE00004C59B01AC0169817A818B819C810E947AC80E9439C66093420C7093430C8093C9
:20ED0000440C9093450C6D817E818F819885A20191010E947AC80E9439C66093460C709313
:20ED2000470C8093480C9093490CC601B501A40193010E947AC80E9439C660934A0C70931A
:20ED40004B0C80934C0C90934D0C69817A818B819C81A80197010E947AC80E9439C66093AE
:20ED60004E0C70934F0C8093500C9093510CAA24BB24F501E552FE4FE080F18002811381DD
:20ED800098E8C92E9BE0D92ECA0CDB1C60E070E080E89FE3A80197010E94D1C5D6016D93E3
:20EDA0007D938D939C93139788E9C82E8BE0D82ECA0CDB1CF501E95FFD4FC801B7012081F9
:20EDC0003181428153810E947AC80E943EC6F6016083718382839383B8EACB2EBBE0DB2E38
:20EDE000CA0CDB1CF501E95EFD4FC801B70120813181428153810E947AC80E943EC6D601F1
:20EE00006D937D938D939C931397E4E0F0E0AE0EBF1EF0E1AF16B10409F0ABCFC0900702A5
:20EE2000A09008026090090220900A02E0901702F09018020091190210911A026C2D7A2D15
:20EE4000862D922DA80197010E94CAC587FD06C08C2D9A2DA62DB22D7C018D016D817E815A
:20EE60008F819885A80197010E947AC89B01AC0160E070E080E090E40E94D1C50E94E7C80A
:20EE80009B01AC01C801B7010E947AC86093320C7093330C8093340C9093350CC0900F0239
:20EEA000A09010026090110220901202E0901F02F090200200912102109122026C2D7A2D5D
:20EEC000862D922DA80197010E94CAC587FD06C08C2D9A2DA62DB22D7C018D0169817A81E2
:20EEE0008B819C81A80197010E947AC89B01AC0160E070E080E090E40E94D1C50E94E7C88E
:20EF00009B01AC01C801B7010E947AC86093360C7093370C8093380C9093390C8091FF0BEE
:20EF20008D7F8093FF0B28960FB6F894DEBF0FBECDBFCF91DF911F910F91FF90EF90DF9006
:20EF4000CF90BF90AF909F908F907F906F905F904F903F902F90089588E10FB6F8948093A2
:20EF60006000109260000FBE579A3E9A239A3D9A3F9A229A569A5E9A569A5E9A0D9A159A4A
:20EF80000C9A149A3A98429A3B98439A3C98449A249A2C98559A5D980E94AA1880E090E073
:20EFA000A8E4B2E480936A0C90936B0CA0936C0CB0936D0C84E690E090936F0C80936E0CA0
:20EFC0009093710C8093700C20E030E040E050E02093DF0B3093E00B4093E10B5093E20BC8
:20EFE0002093DB0B3093DC0B4093DD0B5093DE0B2093D70B3093D80B4093D90B5093DA0B8D
:20F00000109248041092490410924A0410924B041092C70B1092C80B1092C90B1092CA0B5C
:20F020001092C30B1092C40B1092C50B1092C60B1092BF0B1092C00B1092C10B1092C20B54
:20F040001092BB0B1092BC0B1092BD0B1092BE0B80E090E0A0EAB1E48093720C9093730CE8
:20F06000A093740CB093750C8AE999E9A9E9BEE38093760C9093770CA093780CB093790C37
:20F0800020937E0C30937F0C4093800C5093810C20937A0C30937B0C40937C0C50937D0CCC
:20F0A00088E893E1A0E0B0E08093260C9093270CA093280CB093290C81E0809328021092A2
:20F0C000840C1092850C1092860C1092870C2093880C3093890C40938A0C50938B0C80936F
:20F0E000FF0B80E090E0AAE7B3E48093520C9093530CA093540CB093550C80E090E0A4E68A
:20F10000B3E480935A0C90935B0CA0935C0CB0935D0C80E090E0A0E7B3E48093620C90937C
:20F12000630CA093640CB093650C2093560C3093570C4093580C5093590C20935E0C30936F
:20F140005F0C4093600C5093610C2093660C3093670C4093680C5093690C10928C0C0E94DF
:20F160000A2C4091D5015091D6016091D7017091D80183E294E00E94824D85E593E00E948E
:20F18000282A8EE89FE00E944AC20E945D500E940F410E9437350E94D9750E9424190E94BA
:20F1A000AB180E94C74C80E00E94BD3F82EF9CE00E94137E08950E94B82808950E94AC7738
:20F1C0000895FC0189E181831482148E13A216A2E05CFF4F108233961082B9961082339661
:20F1E000108236971192119210828091000C8D7F8093000C0895FC01E759FF4F1192119222
:20F2000010828091000C8D7F8093000C8091010C887F8093010C8FE28093E30F1092E40FC4
:20F2200010921B100895FC01E659FF4F8081EA56F040882351F0E759FF4F81E0808380917A
:20F24000010C82608B7F8093010C0895DA01FB0190E02EE28C91803229F0983009F4219340
:20F260008C9181939F5F9B3011F01196F3CF1082CF01089582EF9CE00E94E17808950F9304
:20F280001F93CF93DF93EC018B01C659DF4F8881CA56D0408823C1F0C759DF4F1882C95686
:20F2A000D040CE01805C9F4F0E946789CE01B80141E00E944B95882319F08FE49EE002C081
:20F2C00081E69EE00E94282ADF91CF911F910F9108950F931F93CF93DF93EC018B01C659D8
:20F2E000DF4F8881CA56D0408823E9F0C759DF4F1882C956D040CE01805C9F4F0E946789E1
:20F30000CE01B8010E948C94882331F4CE01B8010E949A94882319F082E39EE002C08FE3B0
:20F320009EE00E94282ADF91CF911F910F9108950F931F93CF93DF939C01EC01C559DF4FA0
:20F340008881882381F08901005C1F4FC8010E94D287C8010E946789188280E29EE00E94F9
:20F36000282A1092CE0FDF91CF911F910F910895EF92FF920F931F93CF93DF93EC017B015C
:20F38000C659DF4F8881CA56D040882349F18E01005C1F4FC8010E946789C759DF4F188266
:20F3A000C956D040CE0160E00E947189C801B70146E50E949094882319F48AEF9DE00DC086
:20F3C0008EE89FE063E976E140E00E94BB98C559DF4F81E088838EE09EE0B7010E941B2A3D
:20F3E000DF91CF911F910F91FF90EF900895CF93DF93EC01C659DF4F8881CA56D040882350
:20F40000A1F0CF59DF4F488159816A817B8188ED9DE00E94DA29FE01729162915291429139
:20F420008BEE93E00E94B12904C08AEE9DE00E94282ADF91CF910895BF92CF92DF92EF92A6
:20F44000FF920F931F93DF93CF93CDB7DEB76D970FB6F894DEBF0FBECDBF8C01D62EC72E09
:20F46000B42E06591F4FF80180810A561040882309F468C007591F4FF8011082095610405B
:20F4800080E4E82EF12CE00EF11E1C821982C7010E946789DE011196F801B3968DE101907E
:20F4A0000D928150E1F7C701BE016F5F7F4F4D2D5C2D21E00E941D948823F1F18D2D9C2D7A
:20F4C0006FE270E00E94E8179C01009721F48D2D9C2D9C0102C02F5F3F4FBB2091F485EAD4
:20F4E0009DE0B9010E94102A0D5A1F4FF80140815181628173810355104082EB9DE00E948D
:20F50000B1290F591F4FF80110821182128213820E501040F80180819181A281B381065F7E
:20F520001F4FF80180839183A283B38389EB9DE00E94282A81E007C0BB2021F487EC9DE005
:20F540000E94282A80E06D960FB6F894DEBF0FBECDBFCF91DF911F910F91FF90EF90DF9070
:20F56000CF90BF900895EF92FF920F931F93DF93CF93CDB7DEB76D970FB6F894DEBF0FBE2E
:20F58000CDBF8C0119821C8287E89DE00E94282AC80160E00E9471890B5F1F4F7E010894A1
:20F5A000E11CF11CC701B8010E94BA86C70160E040E00E94929687E99DE00E94282A6D9608
:20F5C0000FB6F894DEBF0FBECDBFCF91DF911F910F91FF90EF900895CF92DF92EF92FF9235
:20F5E0000F931F93CF93DF937C018B01EA011CC0F7018081992787FD90950E94FAC96C01DF
:20F60000F8018081992787FD90950E94FAC92197C816D90621F0FC2DF81B8F2F08C008943E
:20F62000E11CF11C0F5F1F4F209711F780E0DF91CF911F910F91FF90EF90DF90CF9008952C
:20F64000DF92EF92FF920F931F93CF93DF937C01EB0104C00894E11CF11C2196F701D0802D
:20F66000DD2081F08D2D992787FD90950E94FAC98C018881992787FD90950E94FAC9081711
:20F68000190741F38D2D992787FD90950E94FAC9182F8881992787FD90950E94FAC9181B3D
:20F6A000812FDF91CF911F910F91FF90EF90DF900895CF92DF92EF92FF920F931F93DF93B6
:20F6C000CF93CDB7DEB7C456D0400FB6F894DEBF0FBECDBF7C019B0180E490E0E80EF91E44
:20F6E000D7011C92E0ECFFEFEE0EFF1EDB014D915C9111979EE7C92E9FEFD92EC422D52274
:20F70000E0E8F0E0CE2ADF2ADA82C98254FF34C012968D919C9113979C838B8357FD02C082
:20F7200044E00CC0FB01A3A9B4A9FD0101900020E9F73197EA1BFB0BED8345E0D9018C9146
:20F7400081FF0AC0FE01E40FF11D16968D919C911797928381834E5FF901808182FF1FC099
:20F76000FE01E40FF11DD90118968D919C911997928381834E5F13C041FD02C042E004C087
:20F78000FB0186818B8343E0D9018C9182FF07C0FE01E40FF11D18968C9181834F5FF9017F
:20F7A000808183FF0DC0BE01640F711D82859385A485B585FB0181839283A383B4834C5F9A
:20F7C000D9018C9184FF0FC0BE01640F711D1E968D919D910D90BC91A02DFB018183928354
:20F7E000A383B4834C5FD9018C9185FF0FC0BE01640F711D52968D919D910D90BC91A02D0C
:20F80000FB0181839283A383B4834C5FD9018C9186FF0FC0BE01640F711D56968D919D9188
:20F820000D90BC91A02DFB0181839283A383B4834C5FD9018D919C91119790FF0FC0BE010A
:20F84000640F711D5A968D919D910D90BC91A02DFB0181839283A383B4834C5FD9018D919F
:20F860009C91119791FF07C0FE01E40FF11D5E968C9181834F5FF9018081918192FF0DC02E
:20F88000BE01640F711D878D90A1A1A1B2A1FB0181839283A383B4834C5FD9018D919C918C
:20F8A000119793FF0FC0BE01640F711D93968D919D910D90BC91A02DFB0181839283A38318
:20F8C000B4834C5FD90112968C91129780FF0FC0BE01640F711D97968D919D910D90BC918D
:20F8E000A02DFB0181839283A383B4834C5FD90112968C91129781FF0FC0BE01640F711DC7
:20F900009B968D919D910D90BC91A02DFB0181839283A383B4834C5FD9018D919C911197C9
:20F9200097FF35C0D3966D917C91D49794FF1BC0FB0101900020E9F73197E61BF70B3E2F2A
:20F94000242F9E2FDE0111960AC08D01020F111DFB018191BF01F80180832F5F9150992375
:20F96000A1F7430F14C020E030E0DE011196842F820F8D01080F111DFB018191BF01F80155
:20F9800080832F5F3F4F2031310589F7405F142F20E030E0A0E0B0E0BE016F5F7F4F1FC005
:20F9A000512F163108F055E1FB01952F8191280F311D2F3F310510F02F5F3040A20FB31FD6
:20F9C000AF3FB10510F0AF5FB040915079F75150852F90E05F5F0196680F791F151B1123A7
:20F9E000F9F6BE016F5F7F4FFB01E40FF11D20834F5FFB01E40FF11DA083F0E8CF16D104BD
:20FA000029F48FEC95E00E942D2A07C04F5FC701805C9F4F50E00E94E38C80E490E0E80ECE
:20FA2000F91ED7018C91882321F081E79DE00E94282ACC59DF4F0FB6F894DEBF0FBECDBF8B
:20FA4000CF91DF911F910F91FF90EF90DF90CF900895FC0180915C0D882379F0E759FF4FF4
:20FA600010828091010C897F8093010C80EA96E10E94282A81E00E942F750895EF92FF9283
:20FA80000F931F93CF93DF93EC0180915C0D8823B9F18091010C8B7F8093010C662361F15F
:20FAA0006091EB017091EC018091ED019091EE0120E030E040E05FE30E947AC87B018C010D
:20FAC00081E061E040E021E00E9495746091F3017091F4018091F5019091F6012DEC3CEC7D
:20FAE0004CE45FE30E947AC87B018C0180E060E041E020E00E949574C759DF4F81E0888381
:20FB0000DF91CF911F910F91FF90EF9008954F925F926F927F928F929F92AF92BF92CF92F1
:20FB2000DF92EF92FF920F931F93FC0180915C0D882309F469C0E759FF4F10828091010C68
:20FB400084608093010C662309F45EC00E94E7280E94666B00D000D04DB65EB60894411C29
:20FB6000511C6090560C7090570C8090580C9090590C60915E0C70915F0C8091600C909105
:20FB8000610C20915A0C30915B0C40915C0C50915D0C0E9404C55B016C016091DF0B709126
:20FBA000E00B8091E10B9091E20B20E030E040E050E40E9404C57B018C016091EB01709199
:20FBC000EC018091ED019091EE0120E030E040E05FE30E947AC8F2016083718382839383EE
:20FBE000C401B301A60195010F2EF0E8AF2EFFE4BF2EF3ECCF2EF7E4DF2EF02D0E94BA72DE
:20FC00000F900F900F900F901F910F91FF90EF90DF90CF90BF90AF909F908F907F906F9052
:20FC20005F904F900895FF920F931F93CF93DF93EC018C0106591F4FF80110826FE144E05A
:20FC40000E947C8A882329F484E69DE00E94282A26C0FF24F394F801F0828091010C81605F
:20FC60008093010CCE0160E00E947189CE0160E071E041E00E941C7A882389F08AEB96E1F0
:20FC80000E94282AF8018081882349F0C759DF4FF8828091010C82608B7F8093010CDF9130
:20FCA000CF911F910F91FF900895FC01E759FF4F1082E956F040CF010E94137E0895CF93DA
:20FCC000DF93DC01EB01BA0180E090E020E2FE01E80FF91F208301968B309105C1F747E0E4
:20FCE00030E023C0282F8E3219F0E8EEF8E108C04A3049F14AE038E017C03196981719F12D
:20FD000094919923D1F7431720F0803210F08F3708F02FE5822F81568A3108F42052FE019C
:20FD2000E30FF11D20833F5F11968C91882311F08F32C1F6FB01B183A08390E0888180321C
:20FD400019F091E001C090E0892FDF91CF9108958D3010F046E002C0482F4695249A2C9A58
:20FD6000279A259A2698809164008B7F80936400242F30E0C9019595879580658CBD40FF6F
:20FD800002C080E004C080E0463009F081E08DBD0895FF920F931F93CF93DF938B010E947F
:20FDA000E3C2EB01FF24FA9409C00E94E3C26C1B7D0B6017710710F080E008C0FEBC0DB450
:20FDC00007FEFDCF8EB58F3F81F781E0DF91CF911F910F91FF9008950F931F938C01FC013E
:20FDE00082810E94A87EF801808160E00E9497C41F910F910895FF920F931F93DF93CF935B
:20FE0000CDB7DEB72A970FB6F894DEBF0FBECDBF8C01F62E2F83388749875A870E94EC7EE2
:20FE2000C8016CE271E00E94C97EFE0137969E012F5F3F4F86E0D9011D928A95E9F78F2D40
:20FE40008064898383818A8382818B8381818C838F818D83D901F90190E069E0AE014A5F7A
:20FE60005F4F308120E0990F892F832787FD96272F5F283011F0330FF6CF3196E417F5072C
:20FE800081F7990F91609E839E01295F3F4F8C918EBD0DB407FEFDCF1196A217B307B9F7B7
:20FEA000BCE0FB1631F48FEF8EBD0DB407FEFDCF8EB59FEF2FEF2EBD0DB407FEFDCF8EB566
:20FEC00087FF07C0992319F4F801838305C09150F2CFD80113968C932A960FB6F894DEBF57
:20FEE0000FBECDBFCF91DF911F910F91FF900895FC01808161E00E9497C48FEF8EBD0DB497
:20FF000007FEFDCF0895CF93DF93EC010E94EC7ECE0168E572E00E94C97E882389F08DEFAF
:20FF20008EBD0DB407FEFDCFCE0168E572E00E94C97E882329F0CE010E94787F81E006C03A
:20FF400082E18983CE010E94787F80E0DF91CF910895AF92BF92CF92DF92EF92FF920F93E5
:20FF60001F93CF93DF93EC015A016B017801890167E320E030E040E050E00E94FB7ECE01B0
:20FF800067E1A80197010E94FB7E882311F089E013C08C81833039F0E9E0AA0CBB1CCC1CAE
:20FFA000DD1CEA95D1F7CE0169E1A60195010E94FB7E882339F087E08983CE010E94787FE1
:20FFC00080E004C0CE010E94787F81E0DF91CF911F910F91FF90EF90DF90CF90BF90AF90AA
:20FFE00008950F931F93CF93DF938C01EA0140E050E0A0E0B0E0252F3327FE01EA0FFB1FA4
:020000040001F9
:20000000808190E028273927220F331F2851394EF90185919491542F442748275927119684
:20002000F2E0A030BF0739F76EBD0DB407FEFDCF88818EBDE98182E090E00DB407FEFDCF49
:20004000EEBD22E08030920731F0FE01E80FF91FE0810196F2CF0DB407FEFDCF5EBD0DB454
:2000600007FEFDCF4EBD0DB407FEFDCF8FEF8EBD0DB407FEFDCF8EB5F80183838F718530C0
:2000800011F481E007C083E1F8018183C8010E94787F80E0DF91CF911F910F9108950F93B1
:2000A0001F93CF93DF93EC018B010E94EC7ECE0168E572E00E94C97E882361F0CE016CEFB8
:2000C000A8010E94F17F882329F0CE010E94787F81E006C085E18983CE010E94787F80E0D8
:2000E000DF91CF911F910F910895CF92DF92EF92FF920F931F93CF93DF93EC017A018B0143
:2001000069018C81833039F029E0EE0CFF1C001F111F2A95D1F7CE0168E1A80197010E949D
:20012000FB7E882311F086E023C0CE016EEFA6010E94F17F8823E9F0CE0168E572E00E94D8
:20014000C97E882311F487E113C0CE016DE020E030E040E050E00E94FB7E882341F48FEF78
:200160008EBD0DB407FEFDCF8EB5882379F086E18983CE010E94787F80E0DF91CF911F9190
:200180000F91FF90EF90DF90CF900895CE010E94787F81E0F2CF8091830F80FF3EC04091CB
:2001A0007F0F5091800F6091810F7091820F8091880F9091890F2FE73DE00E947580882358
:2001C00071F18091830F81FF23C04091840F5091850F6091860F7091870F411551056105AF
:2001E0007105B1F080917F0F9091800FA091810FB091820F480F591F6A1F7B1F8091880F6C
:200200009091890F2FE73DE00E947580882339F08091830F8E7F8093830F81E0089580E0D4
:200220000895CF93DF93EC010E94EC7ECE016CE020E030E040E050E00E94FB7E882339F0EA
:2002400083E08983CE010E94787F80E004C0CE010E94787F81E0DF91CF910895CF93DF9399
:20026000EC019A01AB018C81833039F069E0220F331F441F551F6A95D1F7CE0162E10E9443
:20028000FB7E882339F085E08983CE010E94787F80E004C0CE010E94787F81E0DF91CF917B
:2002A0000895BF92CF92DF92EF92FF920F931F93CF93DF93EC016B017A010E94E3C28B019D
:2002C000BB24BA9409C00E94E3C2601B710B6D52714010F081E160C0BEBC0DB407FEFDCFEC
:2002E0008EB58B838F3F79F38E3F11F08FE054C0D7011197E114F104D9F08FEF8EBD20E026
:2003000030E09FEF0BC00DB407FEFDCF8EB5F601E20FF31F80839EBD2F5F3F4F2A173B07A8
:2003200090F30DB407FEFDCF8EB5AC0DBD1D8C931B828FEF8EBD0DB407FEFDCF3EB58FEF4A
:200340008EBD0DB407FEFDCF2EB5A0E0B0E060E070E016C04B2F5527F601E60FF71F80816E
:2003600090E048275927440F551F4851594EFA0185919491BA2FAA27A827B9276F5F7F4FDC
:200380006E157F0538F3932F80E030E0822B932B8A179B0739F08BE18983CE010E94787F42
:2003A00080E004C0CE010E94787F81E0DF91CF911F910F91FF90EF90DF90CF90BF90089568
:2003C000EF92FF920F931F938C017B010E94EC7EC801B70140E052E00E9451811F910F910B
:2003E000FF90EF900895CF92DF92EF92FF920F931F93CF93DF93EC017A018B0169018C81DB
:20040000833039F059E0EE0CFF1C001F111F5A95D1F7CE0161E1A80197010E94FB7E882394
:2004200039F084E08983CE010E94787F80E006C0CE01B60140E052E00E945181DF91CF9179
:200440001F910F91FF90EF90DF90CF900895DF92EF92FF920F931F937B018C01D42E8091E0
:200460007F0F9091800FA091810FB091820F8E159F05A007B107E1F00E94CB80882311F19A
:20048000D2FC0CC08091880F9091890FB801A7012FE73DE00E94F3818823A1F01092830F47
:2004A000E0927F0FF092800F0093810F1093820F83E0D8228091830F8D298093830F2FE763
:2004C0003DE002C020E030E0C9011F910F91FF90EF90DF9008956F927F928F929F92AF9254
:2004E000BF92CF92DF92EF92FF920F931F93CF93DF935C01142F7093890F6093880FDC01FD
:2005000057961C9282E090E0A0E0B0E0F50180839183A283B3831092830F8FEF9FEFAFEF18
:20052000BFEF80937F0F9093800FA093810FB093820F1092840F1092850F1092860F1092DF
:20054000870F442321F466247724430144C0453008F022C160E070E080E090E040E00E94AA
:200560002782EC01009709F417C1412F50E041505040FA01B4E0EE0FFF1FBA95E1F7E80FF0
:20058000F91FE254FE4F8081EE5BF14090E08F779070892B09F000C1E653FE4F80819181C8
:2005A000A281B38184369105A105B10508F4F4C0A4E0440F551FAA95E1F7C40FD51FCA5342
:2005C000DE4F688079808A809B80611471048104910409F4E1C0C401B30140E00E94278262
:2005E000EC01009709F4D8C08B859C858050924009F0D2C06889662309F4CEC0EE85FF8588
:20060000309709F4C9C08D85882309F4C5C0D50152966C93529714968C9314971D961C92D3
:2006200001E010E008C04F5FD5011D964C934150483008F0B1C0D5011D964C911D971496D5
:200640008C9190E09801042E02C0220F331F0A94E2F78217930739F78E899F89009721F03C
:200660009C0140E050E004C02CA13DA14EA15FA1D50115962D933D934D935C9318975296B8
:200680008C91882341F02093840F3093850F4093860F5093870F6F01EE24FF24C60CD71C79
:2006A000E81CF91CF501C38AD48AE58AF68A09891A89118F008F70E080E090E025813681B0
:2006C000478150850E9450C96C0D7D1D8E1D9F1DD5015A966D937D938D939C935D97F5E05A
:2006E000000F111FFA95E1F701501E4F012F11270695980140E050E0260F371F481F591F40
:20070000F50126873787408B518B8B899C89009721F07C0100E010E004C0E8A0F9A00AA113
:200720001BA1C401B301621B730B840B950B6E0D7F1D801F911FD5011D960C901D9704C057
:2007400096958795779567950A94D2F7F5016187728783879487653FFFE07F07F0E08F0778
:20076000F0E09F0720F48CE057968C9315C0655F7F4F8040904018F480E1F5010AC08CA522
:200780009DA5AEA5BFA5F501828F938FA48FB58F80E2878B81E001C080E0DF91CF911F914A
:2007A0000F91FF90EF90DF90CF90BF90AF909F908F907F906F90089542600E9427820895AC
:2007C0008F929F92AF92BF92CF92DF92EF92FF920F931F93CF93DF93EC016A017B0148010C
:2007E0005901423051056105710508F44BC089859A85AB85BC850196A11DB11D84179507FC
:20080000A607B70708F43EC08F89803129F4252F362F472F55270BC08032A1F59A01AB0188
:2008200097E056954795379527959A95D1F78B899C89AD89BE89280F391F4A1F5B1FCA0108
:20084000B90141E00E94DC839C010097D9F08F89803149F4F601F070EE0FFF1FE20FF31F44
:20086000918280820DC0F601EF77F070EE0FFF1FEE0FFF1FE20FF31F80829182A282B38232
:2008800081E001C080E0DF91CF911F910F91FF90EF90DF90CF90BF90AF909F908F90089561
:2008A000CF92DF92EF92FF920F931F93CF93DF93EC017A018B01690142305105610571052A
:2008C00008F453C089859A85AB85BC850196A11DB11D84179507A607B70708F446C08F898C
:2008E000803129F45527412F302F2F2D0BC08032E1F59A01AB0167E0569547953795279553
:200900006A95D1F78B899C89AD89BE89280F391F4A1F5B1FCA01B90140E00E94DC839C01A5
:20092000009719F18F89803159F4F701F070EE0FFF1FE20FF31F80819181A0E0B0E00EC099
:20094000F701EF77F070EE0FFF1FEE0FFF1FE20FF31F80819181A281B381BF70F60180830D
:200960009183A283B38381E001C080E0DF91CF911F910F91FF90EF90DF90CF900895AF92AC
:20098000BF92CF92DF92EF92FF920F931F93DF93CF9300D000D0CDB7DEB76C017A018B01CD
:2009A00082E090E0A0E0B0E0F60180839183A283B3835E010894A11CB11CC601B801A7013F
:2009C00095010E945084882341F1C601B801A70100E010E020E030E00E94E0838823E9F09D
:2009E000E980FA800B811C81F6018789803151F4F8EFEF16FFEFFF06F0E00F07F0E01F0733
:200A0000E0F209C088EFE8168FEFF8068FEF08078FE0180790F281E001C080E00F900F90ED
:200A20000F900F90CF91DF911F910F91FF90EF90DF90CF90BF90AF9008952F923F924F92DE
:200A40005F926F927F928F929F92AF92BF92CF92DF92EF92FF920F931F93DF93CF93CDB71F
:200A6000DEB72F970FB6F894DEBF0FBECDBF1C014A875B876C877D873F872E87DC01199606
:200A80008D919D910D90BC91A02D0196A11DB11D8E839F83A887B987F901008111812281DE
:200AA0003381011511052105310549F0480159010894811C911CA11CB11C1D8210C0D1016D
:200AC0008D909D90AD90BC901D828A859B85AC85BD850197A105B10511F491E09D83750102
:200AE00064014424552432018E010F5F1F4FF10181859285A385B485481659066A067B06F4
:200B000008F090C08E819F81A885B9858C159D05AE05BF0550F4F2E08F2E912CA12CB12CFF
:200B2000E2E0CE2ED12CE12CF12CC101B701A60198010E945084882309F474C089819A819F
:200B4000AB81BC81A70196012F5F3F4F4F4F5F4F0097A105B10519F049015A010DC02819D6
:200B600039094A095B098A859B85AC85BD85281739074A075B0759F00894411C511C611C7C
:200B8000711C0894C11CD11CE11CF11CB0CFC101A601B7010FEF1FEF2FEF3FE00E94E0836A
:200BA000882399F43FC02601370108944108510861087108C101B301A201970186010E94A5
:200BC000E083882379F1730162018C149D04AE04BF0448F3AE85BF854D915D916D917C9187
:200BE000411551056105710539F0C101950184010E94E0838823B1F0EE85FF85808291820A
:200C0000A282B382FD81FF2359F00894811C911CA11CB11CD1018D929D92AD92BC921397CB
:200C200081E001C080E02F960FB6F894DEBF0FBECDBFCF91DF911F910F91FF90EF90DF9089
:200C4000CF90BF90AF909F908F907F906F905F904F903F902F900895CF93DF93EC019C01F4
:200C6000295F3F4F8D819E8141E050E060E070E00E941D858823A1F08F89988DA98DBA8D16
:200C80000097A105B10559F48F819885A985BA858F8B988FA98FBA8F89818068898381E059
:200CA000DF91CF910895CF92DF92EF92FF920F931F93DF93CF9300D000D0CDB7DEB77C0185
:200CC000FC018789908DA18DB28D89839A83AB83BC8300E010E06E010894C11CD11C498178
:200CE0005A816B817C81D70115968D919C91169796010E945084882379F1D7011596ED9192
:200D0000FC9116978481080F111DB0E100301B0718F529813A814B815C818789803131F46B
:200D2000285F3F4F40405040D0F205C0285F3F4F4F4F5F40A0F2C801A0E0B0E019E0880FBA
:200D4000991FAA1FBB1F1A95D1F7F701838B948BA58BB68B81E001C080E00F900F900F90CC
:200D60000F90CF91DF911F910F91FF90EF90DF90CF900895CF93DF93EC01FB018B818823C7
:200D8000D1F57E836D8387898031C9F582E08B831F8A188E198E1A8E808D918DA0E0B0E0D4
:200DA00025E0880F991FAA1FBB1F2A95D1F78B8B9C8BAD8BBE8B0FC083E08B83828D938D88
:200DC000A48DB58D8F8B988FA98FBA8FCE010E945386882381F081E089831F82188619862D
:200DE0001A861B861C861D861E861F86188A198A1A8A1C8201C080E0DF91CF91089580325D
:200E0000D1F7DACF6F927F928F929F92AF92BF92CF92DF92EF92FF920F931F93CF93DF935F
:200E2000EC017A018B012B81222309F489C08B899C89AD89BE8984179507A607B70708F433
:200E40007FC08EC0EB86FC860D871E871F82188619861A860DC0E114F1040105110551F443
:200E60001F82188619861A861B861C861D861E8681E067C02B853C854D855E85ED81FE81CF
:200E8000858590E00996215030404040504039014A01082E04C096948794779467940A94E0
:200EA000D2F72F5F3F4F4F4F5F4F0894E108F108010911095701680104C0D694C794B794CA
:200EC000A7948A95D2F70894E11CF11C011D111DA614B704C804D90428F021153105410515
:200EE000510549F48F89988DA98DBA8D8F839887A987BA8716C0A618B708C808D90811C02E
:200F00004F81588569857A858D819E8194010E9450840894A108B108C108D108882331F48F
:200F20000FC037E0832E912C8C0E9D1EA114B104C104D10429F7EB86FC860D871E8798CF51
:200F400080E0DF91CF911F910F91FF90EF90DF90CF90BF90AF909F908F907F906F900895AE
:200F6000223009F078CF6ECFCF93DF93EC01462F6F85788989899A890E942782AC010097B3
:200F800019F420E030E00AC08C81282F30E065E0220F331F6A95E1F7240F351FC901DF9196
:200FA000CF9108950F931F93CF93DF938C01FC0183818823F1F1818187FF38C0C80161E067
:200FC0000E94B487EC010097A1F18881853E89F1F8018381823040F483899489A589B6895F
:200FE0008C8F9D8FAE8FBF8FF8018789908D9B8F8A8F8789908DA18DB28DCD01AA27BB279B
:201000009D8B8C8BE0917D0DF0917E0D309751F0BE016A5E7F4FCE0148960995888D998DA7
:201020009B8B8A8BF80181818F7781830E94CB8004C081E0F801808380E0DF91CF911F9182
:201040000F9108956F927F928F929F92AF92BF92CF92DF92EF92FF920F931F93DF93CF9351
:2010600000D000D0CDB7DEB77C015A016B01DC0113968C911397813009F091C011968C9167
:2010800081FF8DC0A0C00097A105B10511F481E087C0F7016384748485849684C701B6010A
:2010A000A5010E940287882309F479C0D70115968D919C911697A114B104C104D10489F482
:2010C00057964D915D916D917C915A970E94BF84882309F464C0F701178A108E118E128E34
:2010E00044C0D70117964D915D916D917C911A979E012F5F3F4F0E945084882309F44FC0F7
:20110000D7011596ED91FC91169749815A816B817C818789803149F4483FBFEF5B07B0E0E1
:201120006B07B0E07B0748F020C0483F8FEF58078FEF68078FE07807C0F4CF010E94BF846B
:20114000882369F1D70117964D915D916D917C911A9715968D919C9116970FEF1FEF2FEFB0
:201160003FE00E94E0838823D1F0F701A38AB48AC58AD68A818180688183C7010E94D2871C
:20118000882369F0B601A5016A147B048C049D0410F4B401A301C7010E94028701C080E04F
:2011A0000F900F900F900F90CF91DF911F910F91FF90EF90DF90CF90BF90AF909F908F90DB
:2011C0007F906F900895F70183899489A589B68984179507A607B70708F055CFE0CF1F93B7
:2011E000CF93DF93EC01142FE62FF0E080917F0F9091800FA091810FB091820F8F87988BEB
:20120000A98BBA8B6C83B5E0EE0FFF1FBA95E1F7E158F24F2489358940E050E0A901332756
:2012200022272F8B388F498F5A8F828D938DA0E0B0E0282B392B4A2B5B2B2F8B388F498FD9
:201240005A8F838590E088719070009751F4848D958DA68DB78D8B8B9C8BAD8BBE8B81E08F
:201260000CC0409751F5CE010E945386882321F41B8A1C8A1D8A1E8A84E08B83812F8F70C0
:2012800089831F82188619861A861B861C861D861E8614FF18C0CE0140E050E060E070E0A0
:2012A0000E942288882379F408C04B895C896D897E89CE010E94028702C01B8280E0DF9123
:2012C000CF911F91089515FDF0CF81E0F8CF0F931F938C010E94D287F80113821F910F91AE
:2012E0000895CF93DF93EC01662331F0A396D0937C0DC0937B0DA3978EA1882321F0CE01F2
:2013000083960E946789CE0183962596BE010E94BA86DF91CF910895CF93DF93EC0140E090
:2013200050E060E070E00E942288882369F0CE0161E00E94B487FC01009731F085EE808385
:201340001B820E94CB8001C080E0DF91CF910895BF92CF92DF92EF92FF920F931F93CF938A
:20136000DF93EC01B62E1C82198248830E94E3C26B01888161E00E941AC4888161E00E94BD
:2013800097C42698259A279A089A8BE08A830E94A87E80E09FEF9EBD0DB407FEFDCF8F5F09
:2013A0008A30C9F709C00E94E3C26C197D09615D774010F081E06FC0CE0160E020E030E074
:2013C00040E050E00E94FB7E813069F7CE016BE321E030E040E050E00E94FB7E813011F046
:2013E0008AE159C01FEFCE0168E02AEA31E040E050E00E94FB7E853011F481E00DC080E06C
:201400001EBD0DB407FEFDCF9EB58F5F8430C1F79B839A3A31F482E08C838C81823051F426
:201420000DC00E94E3C26C197D09615D7740D8F282E031C0EE24FF2487010FC0E12CF12C45
:20144000012D60E4162F09C00E94E3C26C197D09615D774010F08AE01EC0CE0167E320E0E4
:2014600030E040E050E00E94FB7ECE0169E2A80197010E94FB7E882339F78C81823029F5C3
:20148000CE016AE320E030E040E050E00E94FB7E882331F088E08983CE010E94787F21C02C
:2014A0008FEF8EBD0DB407FEFDCF8EB5807C803C11F483E08C8380E09FEF9EBD0DB407FE50
:2014C000FDCF2EB58F5F8330C1F7CE010E94787F8EE08B1518F488E1898303C0BA8281E0AD
:2014E00001C080E0DF91CF911F910F91FF90EF90DF90CF90BF9008950F931F93CF93DF93BB
:20150000EC01262F642F422F0E94A8898823C9F08E010B5F1F4FC801BE0141E00E946B82AF
:20152000882339F4C801BE0140E00E946B82882341F0CE0161E00E947189882319F081E0FF
:2015400001C080E0DF91CF911F910F9108953F924F925F926F927F928F929F92AF92BF9214
:20156000CF92DF92EF92FF920F931F93DF93CF93CDB7DEB72A970FB6F894DEBF0FBECDBF3E
:201580003C01162F072F5A874987DC0111968C91119781FFFAC182FF17C053964D915D9151
:2015A0006D917C9156971B968D919D910D90BC91A02D84179507A607B70731F0C3010E9456
:2015C0000287882309F4E1C1812F902F9C0138872F83E985FA85FE83ED839BC1D301159602
:2015E000ED91FC911697DA01C90119E0B695A795979587951A95D1F794809A949822AFEFB5
:20160000AA2EA1E0BA2EA222B322992009F052C0A114B10409F04EC0D30117964D915D916E
:201620006D917C911A97411551056105710571F1CF019E012F5F3F4F0E945084882309F45B
:20164000A4C129813A814B815C81D3011596ED91FC9116978789803149F4283FBFEF3B078B
:20166000B0E04B07B0E05B0748F019C0283FEFEF3E07EFEF4E07EFE05E0788F4D301179697
:201680002D933D934D935C931A9714C0F3018789908DA18DB28D0097A105B10531F4C301FC
:2016A0000E942C86882331F470C1F30187839087A187B287D30113968C91139715960D91D2
:2016C0001C9116978230B9F41B96CD90DD90ED90FC901E97E9E0F694E794D794C794EA9505
:2016E000D1F7F801828D938DA48DB58DC80ED91EEA1EFB1E20C0D80114966C9170E080E089
:2017000090E0F301278130854185528522503040404050400E9450C96B017C01F8018685D1
:201720009785A089B189C80ED91EEA1EFB1EC90CD11CE11CF11CA114B104C9F42D813E81DC
:2017400020503240E8F5D3011B962D913D914D915C911E9753968D919D910D90BC91A02D4D
:20176000281739074A075B0710F045E001C041E0C701B6010E942782009709F406C140E0EB
:2017800052E04A195B094D805E804415550508F42A019C012A0D3B1DC9016F817885A20145
:2017A0000E94AA17A40CB51CB0E0AB16B2E0BB0609F093C00E94CB80882309F08EC0E5C0D1
:2017C000ED81FE81E050F44060F580917F0F9091800FA091810FB091820F8C159D05AE058B
:2017E000BF0571F48FEF9FEFAFEFBFEF80937F0F9093800FA093810FB093820F1092830F4A
:201800008091880F9091890FB701A6012F8138850E947580882309F4B8C0412C72E0572EA0
:201820005CC0D3011596ED91FC911697848189193E803694831508F4382E032D10E020E00C
:2018400030E08091880F9091890FB701A6010E94A97F882309F499C00F8118854601570121
:201860002CC080917F0F9091800FA091810FB091820F88169906AA06BB0671F48FEF9FEF7B
:20188000AFEFBFEF80937F0F9093800FA093810FB093820F1092830F8091880F9091890F7D
:2018A000B8010E944F8000501E4F0894811C911CA11CB11C882309F468C0882D8C1983150F
:2018C00080F28091880F9091890F0E94837F882309F45BC0532C550C4424920140E050E0A3
:2018E000F30183859485A585B685820F931FA41FB51F83879487A587B6872F813885240D68
:20190000351D38872F838D819E81841995099E838D83D3011B962D913D914D915C911E97DA
:20192000ED81FE81EF2B09F059CE53968D919D910D90BC91A02D82179307A407B50740F4C6
:20194000D30153962D933D934D935C9356970BC080917D0D90917E0D892B59F0E985FA8582
:20196000EF2B39F0D30111968C911197806811968C93F301818183FF05C0C3010E94D2873A
:20198000882319F049855A8505C081E0D3018C934FEF5FEFCA012A960FB6F894DEBF0FBEFB
:2019A000CDBFCF91DF911F910F91FF90EF90DF90CF90BF90AF909F908F907F906F905F90C6
:2019C0004F903F9008950E94A78A08953F924F925F926F927F928F929F92AF92BF92CF9252
:2019E000DF92EF92FF920F931F93DF93CF93CDB7DEB72A970FB6F894DEBF0FBECDBF3C01DE
:201A000058874F83DC0113968C911397882309F439C111968C9180FF35C14FC1F401EC19E3
:201A2000FD09F887EF837C836B839301295F3F4F3E832D838F8198859A8389831BC1D301A1
:201A40001B962D913D914D915C911E97F901F170FA87E9871596ED91FC91169749015A0175
:201A600019E0B694A794979487941A95D1F734803A94382013968C91823049F4C28CD38CEF
:201A8000E48CF58CC80CD91CEA1CFB1C46C089859A85892B01F53320F1F4211531054105A8
:201AA000510551F4F3018789908DA18DB28D87839087A187B2870FC0D30117964D915D915F
:201AC0006D917C911A97CF012D813E810E945084882309F4D7C0F30105811681D8011496C4
:201AE0006C9170E080E090E0278130854185528522503040404050400E9450C96B017C0139
:201B0000F80186859785A089B189C80ED91EEA1EFB1EC30CD11CE11CF11C29853A85232BD3
:201B200099F489819A818050924070F020917F0F3091800F4091810F5091820FC216D306DE
:201B4000E406F50609F0D8C0C701B60140E00E942782009709F496C040E052E0E985FA85FC
:201B60004E1B5F0B49805A804415550508F42A0129853A85280F391F8B819C81B901A20193
:201B80000E94AA175BC08091880F9091890FB701A6012B813C810E94F381882309F472C0AE
:201BA000412CE2E05E2E4AC0BA80B694D30113968C911397823049F01596ED91FC9116974A
:201BC000848183198B1508F4B82EC216D306E406F50670F02B0D311D411D511DC216D306E9
:201BE000E406F50628F40E94CB80882309F44AC08091880F9091890FB701A6010E942E8134
:201C0000882309F43FC0EB80FC8000E00AC0B7010E94E081E0E0F2E0EE0EFF1E882391F1F9
:201C20000F5F8091880F9091890F0B1580F30E941181882339F15B2C550C44242B813C8180
:201C4000240D351D3C832B83920140E050E0F30183859485A585B685820F931FA41FB51F5D
:201C600083879487A587B68729813A81241935093A83298389819A81892B09F0E0CE4F813D
:201C8000588502C04FEF5FEFCA012A960FB6F894DEBF0FBECDBFCF91DF911F910F91FF9098
:201CA000EF90DF90CF90BF90AF909F908F907F906F905F904F903F900895D30153968D90D9
:201CC0009D90AD90BC9056971B96CD90DD90ED90FC901E97EF81F8859F0140E050E0D50175
:201CE000C4018C199D09AE09BF09281739074A075B0708F093CE97CE89819A81805094409C
:201D000008F052CF40CFDF93CF930F92CDB7DEB7BE016F5F7F4F41E050E00E94E68C0197B5
:201D200019F02FEF3FEF03C08981282F30E0C9010F90CF91DF910895EF92FF920F931F93DE
:201D4000CF93DF93EC018B81823038F1EB84FC840D851E85CE010E94838E97FD1EC08B85B3
:201D60009C85AD85BE854F96A11DB11D8B879C87AD87BE8785E016950795F794E7948A95DD
:201D8000D1F72E2D30E02F70307005E0220F331F0A95E1F72158324F02C020E030E0C9015C
:201DA000DF91CF911F910F91FF90EF900895CF93DF93EC018B81843071F5CE0140E050E052
:201DC00060E070E00E94028710C0CE010E949C8EFC01009701F180818823A1F0853E29F03E
:201DE0008E3219F0838583FF16C02B853C854D855E858B899C89AD89BE89281739074A070E
:201E00005B0718F381E08B83898182608983CE010E948C8901C080E0DF91CF910895BF9289
:201E2000CF92DF92EF92FF920F931F93CF93DF93EC01B42E690178018B81823008F44AC020
:201E4000CE0140E050E060E070E00E94028710E0A895CE010E949C8EFC010097E9F1808171
:201E60008823D1F1853011F0853E89F783858F738F3071F1E114F10459F11B144CF51B15FD
:201E80003CF1F70180819181A281B3810097A105B105F1F42B853C854D855E8520523040D3
:201EA00040405040812F992787FD909565E0880F991F6A95E1F7A0E0B0E0281B390B4A0BA2
:201EC0005B0B2083318342835383F601108302C01F5FBECF81E001C080E0DF91CF911F9151
:201EE0000F91FF90EF90DF90CF90BF900895DF92EF92FF920F931F93CF93DF938C01EB0156
:201F00007A01D22E8D819E81F801968385838381882329F56115710559F521C0A701E5E0AA
:201F2000440F551FEA95E1F760E070E0CE010E9402878823A1F0CE010E949C8EFC0100978E
:201F400071F08081882359F0853E49F08E3239F06E2D6F70C8014D2D0E94EF8801C080E04F
:201F6000DF91CF911F910F91FF90EF90DF90089527FFD4CFF4CFCF92DF92EF92FF920F9315
:201F80001F93CF93DF936C018A010115110511F0F8011082FF24F394A895C6010E949C8E91
:201FA000EC01009709F47DC04881442319F4C0E0D0E077C0453049F3453E39F38B85282FD8
:201FC00030E0C9018F7390700F97A9F50115110519F38A8D9B8D892BF9F6842F8F71E1F241
:201FE0008330D4F6FDE08F02D00111241D97F801EA0FFB1F898180838B8181838D81828300
:202000008F818383898584838E858583888986838A8987838C8980878E898187888D8287EA
:202020008C8D83878E8D8487FF2009F4B5CFED841586FF24B1CFC90186709070892B09F09B
:20204000A4CF4E3221F489818E3209F09ECFC90188719070009719F0409709F09DCFAE01FA
:2020600001151105F1F0FF20B9F4FE0190E06BE070E0892F90E09C01359527959695982F40
:20208000882797958795982F920F8191980F6150704079F7E91629F082EF9CE0B8010E94F7
:2020A0002679CE01DF91CF911F910F91FF90EF90DF90CF9008952F923F924F925F926F92B4
:2020C0007F928F929F92AF92BF92CF92DF92EF92FF920F931F93DF93CF93CDB7DEB7C054D2
:2020E000D0400FB6F894DEBF0FBECDBF9EAF8DAF6B01942E752E2FAF21960FAF21971C8286
:202100001D821E821F82FB0185819681EDADFEAD96838583CB0140E050E060E070E00E9412
:202120000287FFADEF2EFF2430E4232E312C2E203F20F6FF40C0A92DB72DFD01019000205D
:20214000E9F73197E9196624E93014F46624639420E08E2F6DE00E946FC9911121E08E2F65
:202160006DE00E946FC9822E880E28C0A895F60183859485A585B6854F97A109B10925E001
:20218000B695A795979587952A95D1F7AFE0BA2EB8228DE99CE0692D772D0E94207B882384
:2021A00091F4FFADF7FDA3C18DAD9EAD6B2D4F2F0E94EF889DC1662488248A94F4E04F2EDF
:2021C000512C4C0E5D1EC601B8014DE95CE0282D82010E94BB8F8C01009741F6232809F454
:2021E00086C1E1FE84C1C601BE01635E7F4F482D9E012F5F3F4F82010E940F8F8C819D8141
:20220000AE81BF810097A105B10519F0332433941FC0F6018381823009F084C1838594854A
:20222000A585B685E5E0B695A79597958795EA95D1F780509240A040B04008F473C157C1A4
:202240008097A109B1098C839D83AE83BF833324A92CB72CF6018181826081834C815D81C8
:202260006E817F81C6010E9402876620D1F5892D972D6EE270E00E94BE178C0176E0E72EA8
:20228000F12CEA0CFB1C009771F0CE010896B80144E050E00E94D9171C86C701E016F106B9
:2022A00020F0C80102C01886C701F82EF9188E01035F1F4FC801692D772D4F2D50E00E9436
:2022C000AA17F801EF0DF11D1082C80167E071E00E94B317C801BE01685F7F4F0E94B31752
:2022E00006C0CE010D96692D772D0E94D2178E01035E1F4FCE010D96B801AE014E5F5F4F4E
:202300000E945F7E9924F801AE01485D5F4F892D90E09C01359527959695982F8827979570
:202320008795982E920E8191980EE417F50779F7D5010D900020E9F71197AA19182D0DE1EB
:20234000E02EF12CEC0EFD1EB0E22B2E0FE0482C552447FC50946A2E772452C0212F30E0AA
:202360004DE050E0249FC001259F900D349F900D11248D50F701422D11924A95E9F708A721
:202380002415350511F090E001C090E4912B9D8F682F70E0D501A60FB71FFE017E9620E0E1
:2023A00030E0C901860F971FAF014E5F5F4F681679061CF48FEF9FEF04C08C91992787FDAF
:2023C000909591838083FA01243019F4FE01BB9604C02A3011F4FE01F9962F5F3F4F1196A1
:2023E0002D303105F1F69AA6C601B70140E250E00E94A78A97FD7BC0C6010E94D28711508D
:20240000112309F0ABCF80E2F70111928A95E9F7CE010D96B701AE014E5F5F4F0E945F7E66
:202420002196FFAD2197FF2311F480E201C080E188A781E298E29EA78DA720E038E03CA756
:202440002BA798AB8FA79EAB8DAB3CAB2BAB8E01035E1F4FC601B80140E250E00E94A78AF0
:2024600097FD45C0C6010E94D28780E2F80111928A95E9F7332011F085EE8D8F00E010E051
:20248000E82CFF24E7FCF094ADE1AA2EB12CAC0EBD1E0DC0C601B50140E250E00E94A78A57
:2024A0000F5F1F4F97FD23C0C6010E94D2878981992787FD90958E199F090817190754F3BF
:2024C0008C819D81AE81BF81F5E0B695A79597958795FA95D1F7E80EF91EFFADFF778DADFE
:2024E0009EADB601A7012F2F0E94778F01C080E0C05CDF4F0FB6F894DEBF0FBECDBFCF911A
:20250000DF911F910F91FF90EF90DF90CF90BF90AF909F908F907F906F905F904F903F9098
:202520002F900895839489828A94F60183859485A585B6850097A105B10509F081CE87CEF2
:20254000CF92DF92EF92FF920F931F93DF93CF93CDB7DEB7A0970FB6F894DEBF0FBECDBFD8
:202560007C016B01DB0113968C91823008F480C0C70123EC01E00E945B90882309F478C0BD
:20258000FE01319680E2DF011D928A95E9F78EE28983FE01329620E2CE010C962193E8171C
:2025A000F907E1F780E18C8720E038E0388F2F8B81E298E29A8F898F9C8B8B8B388B2F8762
:2025C0009A8B898BC701BE016F5F7F4F40E250E00E94A78A97FD4CC0C7010E94D2878EE2A7
:2025E0008A83F60183818250823028F41C8E1B8E1E8A1D8A12C0D60157968D919C915897C1
:202600009C8F8B8F57968D919D910D90BC91A02DCD01AA27BB279E8B8D8BC7018E010F5FFE
:202620001F4FB80140E250E00E94A78A97FD20C0C7010E94D28780E2F80111928A95E9F71A
:20264000C701B80140E250E00E94A78A97FD10C0C7010E94D28784E0D70113968C931397FF
:2026600011968C911197806811968C9381E001C080E0A0960FB6F894DEBF0FBECDBFCF91E1
:20268000DF911F910F91FF90EF90DF90CF9008952F923F924F925F926F927F928F929F9239
:2026A000AF92BF92CF92DF92EF92FF920F931F93DF93CF93CDB7DEB7C154D0400FB6F894ED
:2026C000DEBF0FBECDBFFC012B016A0139010CAF1DAFEBAE19821C821E8E19A2D9011C92EE
:2026E0006115710509F48EC08381882309F08AC0FA0180818F32D1F403C00894C11CD11C06
:20270000D6018C918F32C9F3F20183818250823068F08E01025E1F4F65817681C8010E94D0
:20272000BA86882309F46EC0480101C042015E010894A11CB11C2296BFAEAEAE2297C501B1
:20274000AEAE9FAF5EE1252E312C2C0E3D1E41C04E2D4C19042F112707FD1095C301B601DB
:20276000A8010E94AA17060D171DD8011C92F70181818823D9F1C501B401A30121E000E010
:202780000E945B90882351F4FBADFF23D9F1C501B401A3010E94A0928823A1F184149504C7
:2027A00019F0C4010E94678922968EAD9FAD2297A816B90621F4C101322D292F02C03EAD09
:2027C0002FAD67010894C11CD11C4501832F922F5C01C6016FE270E00E94BE177C01009746
:2027E00009F0B6CFC301B6010E94D2178CAD9DAD9C01D901F4018DE101900D928150E1F71F
:2028000081E001C080E0CF5BDF4F0FB6F894DEBF0FBECDBFCF91DF911F910F91FF90EF9069
:20282000DF90CF90BF90AF909F908F907F906F905F904F903F902F9008958F929F92AF9254
:20284000BF92CF92DF92EF92FF920F931F93DF93CF93CDB7DEB7E9970FB6F894DEBF0FBEC7
:20286000CDBF6C01F22E1D8E18A2EDE18E2E912C8C0E9D1E5E010894A11CB11C950184019E
:20288000EE240E944893882361F08981882311F481E007C0C601B401A5012F2D00E00E94CB
:2028A0005B90E9960FB6F894DEBF0FBECDBFCF91DF911F910F91FF90EF90DF90CF90BF901C
:2028C000AF909F908F9008950F931F93DF93CF93CDB7DEB76D970FB6F894DEBF0FBECDBF42
:2028E0009C01AB0119821C828E010F5F1F4FC801B90122E00E941D94882319F0C8010E94F4
:202900008C896D960FB6F894DEBF0FBECDBFCF91DF911F910F91089583960E94649408954B
:20292000FB01242F60917B0D70917C0DAF010E941D9408950F931F93DF93CF93CDB7DEB764
:202940006D970FB6F894DEBF0FBECDBF19821C828E010F5F1F4FC80141E00E94909488232D
:2029600019F0C8010E94D78E6D960FB6F894DEBF0FBECDBFCF91DF911F910F910895DF9206
:20298000EF92FF920F931F93DF93CF93CDB7DEB76D970FB6F894DEBF0FBECDBF9C01FB0100
:2029A000D42E19821C8280818F3241F48181882329F4C901642F0E94718922C089010D5D4C
:2029C0001F4F7E010894E11CF11CC701B801AF0121E00E941D94882391F08C81823078F08C
:2029E000D801F7018DE101900D928150E1F7DD2021F010937C0D00937B0D81E001C080E0E8
:202A00006D960FB6F894DEBF0FBECDBFCF91DF911F910F91FF90EF90DF9008958F929F92E0
:202A2000AF92BF92CF92DF92EF920F931F93DF93CF93CDB7DEB7E9970FB6F894DEBF0FBE35
:202A4000CDBF6C01E22E1D8E18A2FDE18F2E912C8C0E9D1E5E010894A11CB11C95018401BB
:202A60000E944893882329F0C601B401A5010E94A092E9960FB6F894DEBF0FBECDBFCF91F9
:202A8000DF911F910F91EF90DF90CF90BF90AF909F908F900895DF93CF93CDB7DEB76D97BF
:202AA0000FB6F894DEBF0FBECDBFFB01242F19821C82BC016D5D7F4FCE010196AF010E943A
:202AC0000E956D960FB6F894DEBF0FBECDBFCF91DF9108952F923F924F925F926F927F9226
:202AE0008F929F92AF92BF92CF92DF92EF92FF920F931F93DF93CF93CDB7DEB76D970FB604
:202B0000F894DEBF0FBECDBF6B01542E49013801CB0140E050E060E070E00E940287AA241D
:202B2000BB241E010894211C311C452C4394C8C0A895F5018385082F10E008711070011530
:202B4000110509F4E6C00031110509F0B9C0E1C00031110509F068C0F1E0F51508F4B0C0B3
:202B60008114910491F4552041F089EB9CE00E9424298BEE93E00E94A1298DE99CE00E9435
:202B800024298BEE93E00E94282A19821C82552031F089EB9CE06AE071E00E94B31789EBCE
:202BA0009CE06DE97CE00E94B317F60123853485458556852F5130404040504085E056952E
:202BC0004795379527958A95D1F77901C101B601A90121E00E94778F882351F0C101B10104
:202BE000442D940183010E946A95882309F077C00894E11CF11C05E0EE0CFF1C0A95E1F7B8
:202C0000A70160E070E0C6010E94028789EB9CE06FE270E00E94E817FC01009711F0108231
:202C20004FC01092B90C4CC08114910481F1E9EBFCE001900020E9F78F0101501040095BA0
:202C40001C40F02E402F552747FD509589EB9CE0B4010E94EC7A882399F510160CF4F39453
:202C60006F2D772767FD7095680D791D8DE99CE00E94207B882321F56114710481F1D30186
:202C8000F6018DE101900D928150E1F728C0552041F089EB9CE00E9424298BEE93E00E94FB
:202CA000A1298DE99CE00E942429F501448D558D668D778D8DE594E00E94EB290E945D1A14
:202CC000C601B5014DE95CE020E000E010E00E94BB8F5C01009709F02BCF80E001C081E0E0
:202CE0006D960FB6F894DEBF0FBECDBFCF91DF911F910F91FF90EF90DF90CF90BF90AF9000
:202D00009F908F907F906F905F904F903F902F9008958DE99CE06CE071E00E94C9170097B6
:202D200079F216CF0F931F93DF93CF93CDB7DEB76D970FB6F894DEBF0FBECDBF8C0119828F
:202D40001C8240E050E060E070E00E9402871092B90C89EB9CE0F801948F838FDE011196BF
:202D60008DE101900D928150E1F7C801BE016F5F7F4F40E020E030E000E010E00E946A9547
:202D80006D960FB6F894DEBF0FBECDBFCF91DF911F910F9108959C01F999FECF32BD21BD63
:202DA000F89A80B50895089580FF02C05A9A01C05A9881FF02C05B9A01C05B9882FF02C0FC
:202DC000409A01C0409883FF02C0419A01C04198129A000000000000000000000000129871
:202DE00000000000000000000000000008959F92AF92BF92CF92DF92EF92FF920F931F933B
:202E0000DF93CF93CDB7DEB727970FB6F894DEBF0FBECDBF7C01C42E922E77FD03C0DD2459
:202E2000E0E006C0709561957F4FDD24D394E1E01F828E01095F1F4F86EFA82E8FEFB82E65
:202E4000262FCB016AE070E00E9490C9862F972FBC01205D6A9DC0016B9D900D7A9D900DE6
:202E60001124280FD8012E938D01D3946115710539F7EE2361F0F7018181E82FF0E0E057C1
:202E8000FF4E9DE290838F5FD70111968C93B5E0BC1528F412C0F80192928F01D394DC146F
:202EA000D0F30BC0E82FF0E0E057FF4E90838F5FD70111968C930F5F1F4FF80190819923D8
:202EC00029F0D70111968C918C3160F327960FB6F894DEBF0FBECDBFCF91DF911F910F9109
:202EE000FF90EF90DF90CF90BF90AF909F9008956F927F928F929F92AF92BF92CF92DF92D4
:202F0000EF92FF920F931F93DF93CF93CDB7DEB72D970FB6F894DEBF0FBECDBF4C016A019B
:202F20007B01622E77FD03C000E077240BC0F094E094D094C094C11CD11CE11CF11C01E0A3
:202F4000772473941D869DE0A92EB12CAC0EBD1E1C2DC701B6012AE030E040E050E00E9492
:202F6000C5C9C901DA016C017D01105DC701B60126EF3FEF4FEF5FEF0E9450C9160FF501A2
:202F800012935F010F5FC114D104E104F10401F7772059F0F4018181E82FF0E0E057FF4E00
:202FA0009DE290838F5FF4018183FBE0F61534F41BC0F50142935F010F5F05C0262D3327A4
:202FC00027FD309540E2802F90E0821793078CF30BC0E82FF0E0E057FF4E90838F5FF401E9
:202FE00081830894A11CB11CF5019081992321F0F40181818C3168F32D960FB6F894DEBF13
:203000000FBECDBFCF91DF911F910F91FF90EF90DF90CF90BF90AF909F908F907F906F9071
:2030200008954F925F927F928F929F92AF92BF92CF92DF92EF92FF920F931F93DF93CF9320
:2030400000D000D0CDB7DEB72C016A017B01122F702ECB01BA0120E030E040E050E00E943B
:20306000CAC588239CF4F2018181E82FF0E0E057FF4E9DE290838F5FF20181838C3108F0FA
:2030800066C0F7FAF094F7F8F0941150E72DF0E0EE0FFF1FEE0FFF1FEC5FF44E259135919E
:2030A00045915491C701B6010E9404C54B015C010E943EC66B017C01C201B701A601212FC1
:2030C0000E947897F2019181943108F040C0772049F0E92FF0E0E057FF4E8EE280839F5FD0
:2030E000F2019183C701B6010E946AC69B01AC01C501B4010E9403C5F20111811C3138F54B
:20310000772029F17A9420E030E040E251E40E947AC869837A838B839C830E943EC6E12FD9
:20312000F0E0E057FF4E605D608360531F5FF201118370E0882777FD8095982F0E946CC6C0
:203140009B01AC0169817A818B819C81D3CF0F900F900F900F90CF91DF911F910F91FF904B
:20316000EF90DF90CF90BF90AF909F908F907F905F904F900895CF93DF93DC01442331F073
:20318000ED01C05CDF4F80E090E005C08091000C84FFF6CF19C0382FFB01E80FF91F2491FD
:2031A000222331F029933F5F01968031910599F7A30FB11DA05CBF4F1C92442329F0809118
:2031C000000C80618093000CDF91CF910895CF93DF93FC01DB01442329F0EF01C05CDF4F0F
:2031E00080E008C08091000C84FFF7CF14C099938F5F11969C91992311F08031C1F7E80F62
:20320000F11DE05CFF4F1082442329F08091000C80618093000CDF91CF910895CF92DF92A8
:20322000FF920F931F93CF93DF93EC01EA81EE2309F493C0F0E03496EE0FFF1FE80FF91F58
:2032400020813181C9010596FC01C590D490F9018491823009F081C08091010C082F10E0C0
:2032600029C0E52FF0E0EE0FFF1FEC0DFD1D259134912B5F3F4FF901849125503040882321
:2032800031F040E090E080239123892B09F041E02A5F3F4FF9018491442339F0882399F06E
:2032A00090E080239123892B71F0AC0FBD1F515013965C938A81A82FB0E0FE01EA0FFB1FDE
:2032C0005381552371F6FE01EA0FFB1F8289581708F4528B8A81A82FB0E0FE01EA0FFB1F52
:2032E000F28863815F2D70E026C0E52FF0E0EE0FFF1FEC0DFD1D259134912B5F3F4FF9010F
:20330000849125503040882331F040E090E080239123892B09F041E02A5F3F4FF90184910C
:20332000442339F0882331F090E080239123892B09F07F5F5F5F5617C0F28F2D90E003963D
:20334000870F911D262F30E08217930734F4AC0FBD1F635052966C93BDCFDF91CF911F912C
:203360000F91FF90DF90CF90089508950895CF93DF93EC01F89488818A70C1F48881886083
:203380008883789488A599A5892B61F00E94E3C26AA77BA78CA79DA719A618A6F8948881A3
:2033A00081608883F8948881885088837894DF91CF9108951F9340917102509172028FE076
:2033C000403A580730F5E9E2F2E020E030E08081918184179507B8F4828193814817590776
:2033E00090F4F901EE0FFF1FEE0FFF1FE20FF31FE75DFD4F148187EA99E1612F70E00E9484
:20340000C429812F06C02F5F3F4F359628303105F1F61F910895AF92BF92CF92DF92EF92BB
:20342000FF920F931F93CF93DF93EC01B62E8091000C84FF05C08F7E8093000C0C94C1AB65
:203440000E94E3C22AA93BA94CA95DA97B018C01E21AF30A040B150BA80197016AAB7BABC6
:203460008CAB9DAB223331054105510528F422E330E040E050E014C02D3201E0300700E0FA
:20348000400700E0500760F080E090E0A0E8BFE38EAB9FABA8AFB9AF2CE231E040E050E0B3
:2034A0006CE271E080E090E0621B730B840B950B0E946AC620E030E04AE753E40E94D1C5F1
:2034C0007B018C0120E030E048EC52E40E947AC8A80197010E947AC8A80197010E947AC83B
:2034E00020E030E040E85FE30E9404C56EAB7FAB88AF99AF8A818823D1F40E94E3C268A358
:2035000079A38AA39BA38B81B7FE09C08F5F8B83843010F40C94C1AB1B820C94C1AB882386
:2035200011F483E001C081508B830C94C1AB90E0FC013496EE0FFF1FEC0FFD1F408151817B
:20354000FA01339625913491FA017491359605911491FE01E80FF91F6381723009F081C058
:203560008C8D9D8D892B09F0A6C0B7FE3FC02FC0822F8F5F8383E82FF0E0EE0FFF1FE00FBC
:20358000F11F459154914B5F5F4FFA01249145505040222349F060E030E08091010C90E0D7
:2035A00028233923232B09F061E04A5F5F4FFA012491662371F0222309F44EC030E080917A
:2035C000010C90E028233923232B19F445C0A22FB0E08A81FE01E80FF11D2381822F90E032
:2035E00001968A179B070CF4C3CF36C0662369F533C081508383E82FF0E0EE0FFF1FE00FC7
:20360000F11F459154914B5F5F4FFA01249145505040222349F060E030E08091010C90E056
:2036200028233923232B09F061E04A5F5F4FFA012491662351F0222379F030E08091010CAE
:2036400090E028233923232B39F08A81FE01E80FF11D8381882369F6CE010E940E990C9407
:20366000C1AB713009F5B7FE06C08091AD10681730F46F5F03C0662311F0615063838A8196
:20368000FE01E80FF11D82894381481750F090E00396242F30E08217930714F00C94C1AB09
:2036A0004350428B0C94C1AB733029F4FA0131968591949102C08C8D9D8DFC01ED5EF34061
:2036C000EC36F10510F00C94B3ABEA5BFF4FEE0FFF1F0590F491E02D099483E0FB2DF802DD
:2036E000C001112420914B04820F911D60E00E94E11B0C94B3AB00D000D00F926B2D772742
:2037000067FD7095872F972F2091FB013091FC014091FD015091FE01EDB7FEB721833283F8
:203720004383548321E0258320E030E040E050E0EE24FF248701AA24BB2465010E941E68EB
:203740000F900F900F900F900F900E9436190C94B3AB00D000D00F922B2D332727FD309583
:20376000432F532F8091FF0190910002A0910102B0910202EDB7FEB781839283A383B483D9
:2037800081E0858360E070E080E090E0EE24FF248701AA24BB2465010E941E680F900F902A
:2037A0000F900F900F900E9436190C94B3AB00D000D00F92EB2CFF24E7FCF0940F2D1F2DD3
:2037C0008091030290910402A0910502B0910602EDB7FEB781839283A383B48381E08583F3
:2037E00060E070E080E090E020E030E040E050E0AA24BB2465010E941E680F900F900F90F1
:203800000F900F900E9436190C94B3AB00D000D00F920DB71EB70F5F1F4F6B2D772767FD2B
:203820007095872F972F0E946CC62091DB013091DC014091DD015091DE010E947AC820E0B5
:2038400030E040EA50E40E947AC80E9439C62091FB013091FC014091FD015091FE01F80162
:20386000208331834283538321E0248320E030E040E050E0EE24FF248701AA24BB2465017E
:203880000E941E680F900F900F900F900F900E9436190C94B3AB00D000D00F920DB71EB71C
:2038A0000F5F1F4F6B2D772767FD7095872F972F0E946CC62091DF013091E0014091E10157
:2038C0005091E2010E947AC820E030E040EA50E40E947AC80E9439C69B01AC018091FF01F3
:2038E00090910002A0910102B0910202F80180839183A283B38381E0848360E070E080E069
:2039000090E0EE24FF248701AA24BB2465010E941E680F900F900F900F900F900E94361933
:203920000C94B3AB00D000D00F92CDB6DEB60894C11CD11C6B2D772767FD7095872F972FB0
:203940000E946CC62091E3013091E4014091E5015091E6010E947AC820E030E040EA50E487
:203960000E947AC80E9439C67B018C018091030290910402A0910502B0910602F601808301
:203980009183A283B38381E0848360E070E080E090E020E030E040E050E0AA24BB2465017D
:2039A0000E941E680F900F900F900F900F900E9436190C94B3AB00D000D000D00DB71EB7CC
:2039C0000F5F1F4F6B2D772767FD7095872F972F0E946CC62091E7013091E8014091E9011E
:2039E0005091EA010E947AC80E9439C65B016C0180E090E0A0E0B0E4F80180839183A28394
:203A0000B38381E08483158260E070E080E090E020E030E040E050E0EE24FF2487010E9452
:203A200072690DB71EB70A5F1F4F0FB6F8941EBF0FBE0DBF0E9436190C94B3AB8091000C68
:203A400080628093000C00D000D00F92EB2CFF24E7FCF0940F2D1F2D8091030290910402BE
:203A6000A0910502B0910602EDB7FEB781839283A383B48381E0858360E070E080E090E02D
:203A800020E030E040E050E0AA24BB2465010E941E680F900F900F900F900F900E9436197F
:203AA0008091000C8F7D8093000C0C94B3AB8091000C80628093000C00D000D00F92CDB6DE
:203AC000DEB60894C11CD11C6B2D772767FD7095872F972F0E946CC62091E3013091E401C2
:203AE0004091E5015091E6010E947AC80E9439C67B018C018091030290910402A091050244
:203B0000B0910602F60180839183A283B38381E0848360E070E080E090E020E030E040E0FB
:203B200050E0AA24BB2465010E941E680F900F900F900F900F900E9436198091000C8F7DE5
:203B40008093000C0C94B3AB0E94E3C2609340047093410480934204909343048091B80BEB
:203B60001B144CF48E3714F00C94B3AB8F5F8093B80B0C94B3AB833814F40C94B3AB8150BB
:203B80008093B80B0C94B3AB609196017091970180919801909199010E9439C66E31710515
:203BA00014F460E070E0EB2CFF24E7FCF094E60EF71EF1E0EF16F10419F42EE130E00DC0FF
:203BC0000EE1E016F1041CF420E030E006C097012937310514F028E730E0B901882777FDF7
:203BE0008095982F0E946CC640E00E94303B0C94B3AB60914F0170915001809151019091D3
:203C000052010E9439C66A3A710514F460E070E0EB2CFF24E7FCF094E60EF71E11E0E1166C
:203C2000F10419F42AEA30E00EC02AEAE216F1041CF420E030E007C0970181E0253038071B
:203C400014F024E031E0B901882777FD8095982F0E946CC640E020E00E94F73E0C94B3ABC9
:203C600040916E0C50916F0CB7FE0BC02B2D332727FD309589E190E0821B930B48175907AE
:203C800084F08B2D992787FD9095840F951F893191053CF0E1E0853F9E072CF084EF91E0A2
:203CA00002C089E190E00E94D4180C94B3ABB7FE15C08B2D992787FD909549E150E09A013C
:203CC000281B390B8091700C9091710C8217930728F45093710C4093700C20C0EB2CFF241A
:203CE000E7FCF0948091700C9091710CE80EF91EF092710CE092700CF9E1EF16F10418F458
:203D000089E190E007C005EFE01601E0F00630F084EF91E09093710C8093700C6091700CA1
:203D20007091710C8FEF93E00E94C4290C94B3ABE090D101F090D2010091D3011091D40117
:203D4000C801B70128EE33E040E050E00E94A3C9E61AF70A080B190BB7FE22C06B2D772756
:203D600067FD7095872F972F20E63AEE40E050E00E9450C990958095709561957F4F8F4F44
:203D80009F4FE616F7060807190750F41092D1011092D2011092D3011092D4010C94B3ABF5
:203DA0006B2D772767FD7095872F972F20E63AEE40E050E00E9450C96E0D7F1D801F911F49
:203DC0006093D1017093D2018093D3019093D40161507F4C8949904010F40C94B3AB80E0E9
:203DE0009FECA9E9B0E08093D1019093D201A093D301B093D4010C94B3ABE0904404F090E6
:203E000045040091460410914704C801B70128EE33E040E050E00E94A3C9E61AF70A080B76
:203E2000190BB7FE22C06B2D772767FD7095872F972F20E63AEE40E050E00E9450C990954E
:203E40008095709561957F4F8F4F9F4FE616F7060807190750F410924404109245041092D5
:203E60004604109247040C94B3AB6B2D772767FD7095872F972F20E63AEE40E050E00E94D2
:203E800050C96E0D7F1D801F911F6093440470934504809346049093470461507F4C894903
:203EA000904010F40C94B3AB80E09FECA9E9B0E08093440490934504A0934604B093470451
:203EC0000C94B3ABB7FE19C06CE98B2D8602B0011124882777FD8095982F0E946CC69B016C
:203EE000AC0160910702709108028091090290910A020E94CAC588233CF164E69B2D960214
:203F0000B0011124882777FD8095982F0E946CC620910702309108024091090250910A029A
:203F20000E9404C57B018C0160930702709308028093090290930A0220E030E040E050E057
:203F40000E94CAC588232CF480E090E0A0E0B0E00EC0C801B70120E030E44CE156E40E9419
:203F6000D8C7181664F480E090E4ACE1B6E48093070290930802A0930902B0930A020E94A9
:203F8000D9750C94B3ABB7FE1BC06B2D772767FD7095709561957F4F882777FD8095982FDE
:203FA0000E946CC69B01AC0160910B0270910C0280910D0290910E020E94CAC5882324F195
:203FC0006B2D772767FD7095872F972F0E946CC620910B0230910C0240910D0250910E0294
:203FE0000E9404C57B018C0160930B0270930C0280930D0290930E0220E030E040E050E087
:204000000E94CAC588232CF480E090E0A0E0B0E00EC0C801B70120E030E44CE156E40E9458
:20402000D8C7181664F480E090E4ACE1B6E480930B0290930C02A0930D02B0930E020E94D8
:20404000D9750C94B3ABB7FE19C06CE9EB2DE602B0011124882777FD8095982F0E946CC678
:204060009B01AC0160910F027091100280911102909112020E94CAC588233CF164E6FB2D0E
:20408000F602B0011124882777FD8095982F0E946CC620910F023091100240911102509115
:2040A00012020E9404C57B018C0160930F0270931002809311029093120220E030E040E0D2
:2040C00050E00E94CAC588232CF480E090E0A0E0B0E00EC0C801B70120E030E44CE156E40A
:2040E0000E94D8C7181664F480E090E4ACE1B6E480930F0290931002A0931102B093120208
:204100000E94D9750C94B3ABB7FE19C06CE90B2D0602B0011124882777FD8095982F0E9407
:204120006CC69B01AC0160911702709118028091190290911A020E94CAC588233CF164E623
:204140001B2D1602B0011124882777FD8095982F0E946CC6209117023091180240911902B5
:2041600050911A020E9404C57B018C0160931702709318028093190290931A0220E030E028
:2041800040E050E00E94CAC588232CF480E090E0A0E0B0E00EC0C801B70120E030E44CE163
:2041A00056E40E94D8C7181664F480E090E4ACE1B6E48093170290931802A0931902B09309
:2041C0001A020E94D9750C94B3ABB7FE19C06CE92B2D2602B0011124882777FD8095982F8D
:2041E0000E946CC69B01AC0160911B0270911C0280911D0290911E020E94CAC588233CF1FB
:2042000064E68B2D8602B0011124882777FD8095982F0E946CC620911B0230911C024091DD
:204220001D0250911E020E9404C57B018C0160931B0270931C0280931D0290931E0220E044
:2042400030E040E050E00E94CAC588232CF480E090E0A0E0B0E00EC0C801B70120E030E4BF
:204260004CE156E40E94D8C7181664F480E090E4ACE1B6E480931B0290931C02A0931D0252
:20428000B0931E020E94D9750C94B3ABB7FE19C06CE99B2D9602B0011124882777FD80956C
:2042A000982F0E946CC69B01AC0160911F027091200280912102909122020E94CAC5882390
:2042C0003CF164E6EB2DE602B0011124882777FD8095982F0E946CC620911F0230912002F9
:2042E00040912102509122020E9404C57B018C0160931F027093200280932102909322029B
:2043000020E030E040E050E00E94CAC588232CF480E090E0A0E0B0E00EC0C801B70120E012
:2043200030E44CE156E40E94D8C7181664F480E090E4ACE1B6E480931F0290932002A09394
:204340002102B09322020E94D9750C94B3ABB7FE30C06B2D772767FD7095872F972F0E9483
:204360006CC62DEC3CEC4CEC5DEB0E947AC820E030E040E85FE30E9404C59B01AC01609147
:20438000720C7091730C8091740C9091750C0E94CAC5882374F480E090E0A0E8BFE380939B
:2043A000720C9093730CA093740CB093750C0C94B3AB6B2D772767FD7095872F972F0E94AB
:2043C0006CC62DEC3CEC4CEC5DE30E947AC82091720C3091730C4091740C5091750C0E944A
:2043E00004C57B018C016093720C7093730C8093740C9093750C20E030E040E85FE30E94A5
:20440000CAC5882374F480E090E0A0E8BFE38093720C9093730CA093740CB093750C0C94B6
:20442000B3ABC801B7012DEC3CEC47EC52E40E94D8C7181614F00C94B3AB8DEC9CECA7ECEE
:20444000B2E48093720C9093730CA093740CB093750C0C94B3ABB7FE30C06B2D772767FDDF
:204460007095872F972F0E946CC62DEC3CEC4CEC5DEB0E947AC82DEC3CEC4CEC5DE30E94E7
:2044800004C59B01AC016091760C7091770C8091780C9091790C0E94CAC5882374F48DEC1B
:2044A0009CECACECBDE38093760C9093770CA093780CB093790C0C94B3AB6B2D772767FDEA
:2044C0007095872F972F0E946CC62DEC3CEC4CEC5DE30E947AC82091760C3091770C4091A2
:2044E000780C5091790C0E9404C57B018C016093760C7093770C8093780C9093790C2DEC0B
:204500003CEC4CEC5DE30E94CAC5882374F48DEC9CECACECBDE38093760C9093770CA09310
:20452000780CB093790C0C94B3ABC801B7012DEC3CEC47EC52E40E94D8C7181614F00C94F3
:20454000B3AB8DEC9CECA7ECB2E48093760C9093770CA093780CB093790C0C94B3ABB7FE66
:204560002AC02B2D332727FD309565E070E0621B730B882777FD8095982F0E946CC69B01B7
:20458000AC016091FB017091FC018091FD019091FE010E94CAC5882374F480E090E0A0EAB6
:2045A000B0E48093FB019093FC01A093FD01B093FE010C94B3AB6B2D772767FD7095872F72
:2045C000972F0E946CC62091FB013091FC014091FD015091FE010E9404C57B018C016093C0
:2045E000FB017093FC018093FD019093FE0120E030E040EA50E40E94CAC5882374F480E07A
:2046000090E0A0EAB0E48093FB019093FC01A093FD01B093FE010C94B3ABC801B70120E0EB
:2046200030E04AE754E40E94D8C7181614F00C94B3AB80E090E0AAE7B4E48093FB01909365
:20464000FC01A093FD01B093FE010C94B3ABB7FE2AC02B2D332727FD309565E070E0621BA0
:20466000730B882777FD8095982F0E946CC69B01AC016091FF017091000280910102909177
:2046800002020E94CAC5882374F480E090E0A0EAB0E48093FF0190930002A0930102B09333
:2046A00002020C94B3AB6B2D772767FD7095872F972F0E946CC62091FF01309100024091C4
:2046C0000102509102020E9404C57B018C016093FF0170930002809301029093020220E049
:2046E00030E040EA50E40E94CAC5882374F480E090E0A0EAB0E48093FF0190930002A093AF
:204700000102B09302020C94B3ABC801B70120E030E04AE754E40E94D8C7181614F00C9444
:20472000B3AB80E090E0AAE7B4E48093FF0190930002A0930102B09302020C94B3ABB7FEBA
:204740002AC02B2D332727FD309561E070E0621B730B882777FD8095982F0E946CC69B01D9
:20476000AC01609103027091040280910502909106020E94CAC5882374F480E090E0A0E8B2
:20478000BFE38093030290930402A0930502B09306020C94B3AB6B2D772767FD7095872F5E
:2047A000972F0E946CC6209103023091040240910502509106020E9404C57B018C016093BA
:2047C000030270930402809305029093060220E030E040E85FE30E94CAC588236CF480E070
:2047E00090E0A0E8BFE38093030290930402A0930502B0930602B7C7C801B70120E030E04A
:204800004AE754E40E94D8C718160CF0ACC780E090E0AAE7B4E48093030290930402A093E4
:204820000502B09306029FC7B7FE29C02B2D332727FD309561E070E0621B730B882777FDD8
:204840008095982F0E946CC69B01AC016091EB017091EC018091ED019091EE010E94CAC554
:2048600088236CF480E090E0A0E8BFE38093EB019093EC01A093ED01B093EE0174C76B2DFE
:20488000772767FD7095872F972F0E946CC62091EB013091EC014091ED015091EE010E9445
:2048A00004C57B018C016093EB017093EC018093ED019093EE0120E030E040E85FE30E9428
:2048C000CAC588236CF480E090E0A0E8BFE38093EB019093EC01A093ED01B093EE0143C7D8
